:1020000095EF11F0FFFFFFFF468260EF1CF0FFFF2E
:10201000FFFFFFFFFFFFFFFF4680D8CF15F0E8CF9F
:1020200016F0E0CF17F0D9CF18F0DACF19F0F2A4FC
:102030001CEF10F01EEF10F089EF11F0F10ED76ECB
:10204000690ED66EC2B227EF10F029EF10F022EF22
:1020500010F0D890C432C332D890C432C3320001D9
:1020600095A135EF10F037EF10F03BEF10F0C3CF34
:10207000FEF044EF10F0000EA825D96EDA6A050EC6
:10208000DA22C3CFDFFFA82B01018E51D8B44BEF6A
:1020900010F04DEF10F072EF10F038503910D8B446
:1020A00054EF10F056EF10F05BEF10F03806D8A0A8
:1020B00039067DEF10F0B051D8B461EF10F063EF46
:1020C00010F06EEF10F04250D8A469EF10F06BEFF3
:1020D00010F06EEF10F0010E00019E6F0101B06B69
:1020E0007DEF10F038503910D8B479EF10F07BEF55
:1020F00010F07DEF10F056EF10F0000172517311E7
:10210000D8B485EF10F087EF10F08AEF10F0720767
:10211000D8A07307B0EC68F0000195A192EF10F021
:1021200094EF10F098EF10F0090EC26E9AEF10F0D5
:102130002D0EC26EC28227EF11F00101745175118C
:10214000D8B4A5EF10F0A7EF10F066EF11F0740708
:10215000D8A0750766EF11F0B651D8B4B2EF10F001
:10216000B4EF10F066EF11F0B60766EF11F0010161
:10217000E951EA11D8B4BFEF10F0C1EF10F066EFEB
:1021800011F0E907D8A0EA0766EF11F00101B85194
:10219000D8B4CDEF10F0CFEF10F066EF11F0B80724
:1021A00066EF11F00101E151E211D8B4DAEF10F05D
:1021B000DCEF10F066EF11F0E107D8A0E20766EF60
:1021C00011F074517511D8B4E8EF10F0EAEF10F087
:1021D00066EF11F07407D8A0750766EF11F05AEC9E
:1021E0006BF066EF11F070517111D8B4FAEF10F086
:1021F000FCEF10F066EF11F07007D8A0710766EFE2
:1022000011F0F751F811D8B408EF11F00AEF11F0FE
:1022100066EF11F0F707D8A0F80766EF11F001019B
:10222000B951D8B416EF11F018EF11F066EF11F0B4
:10223000B90766EF11F00101B651D8B422EF11F0E1
:1022400024EF11F066EF11F0B60766EF11F095512B
:10225000000AD8B49DEF10F0010AD8B4ACEF10F02A
:10226000030AD8B4B7EF10F0010AD8B4C6EF10F0E3
:10227000070AD8B4D2EF10F0010AD8B466EF11F013
:10228000030AD8B4E1EF10F0010AD8B466EF11F0F8
:102290000F0AD8B4EFEF10F0010AD8B466EF11F0CE
:1022A000030AD8B4F3EF10F0010AD8B466EF11F0C6
:1022B000070AD8B401EF11F0010AD8B40FEF11F0FA
:1022C000030AD8B41BEF11F066EF11F00001952B53
:1022D0000F0E95174204D8A470EF11F072EF11F0B1
:1022E00086EF11F076517711D8A479EF11F07BEFDA
:1022F00011F084EF11F074517511D8B482EF11F020
:1023000084EF11F086EF11F01F0EA81777EC26F07E
:10231000F29419C0DAFF18C0D9FF17C0E0FF16C049
:10232000E8FF15C0D8FF46901000FBEF4EF0008884
:1023300088888888888888888888888A8D8F9192FC
:1023400093939494959596969797989899999A9A25
:102350009B9B9C9C9C9D9D9D9E9E9E9E9F9F9FA0A7
:10236000A0A0A1A1A1A2A2A2A3A3A3A4A4A4A5A545
:10237000A5A6A6A6A7A7A7A8A8A8A9A9AAAAAAABDE
:10238000ABABACACADADAEAEAFAFB0B0B0B1B1B267
:10239000B2B2B3B3B3B4B4B5B5B5B6B6B7B7B8B8EF
:1023A000B9B9BABABABBBBBCBCBDBDBEBEBFBFBF6C
:1023B000C0C0C1C1C2C2C3C3C4C4C5C5C6C6C7C7E5
:1023C000C8C8C9C9CACACBCBCCCDCDCECFD0D2D349
:1023D000D4D5D7D8DDE2E2E2E2E2E2E2E2E2E2E212
:1023E000E2E2E2E2E2E2E2E2E2E2E2E2E2E2E2E2CD
:1023F000E2E2E2E2E2E2E2E2E2E2E2E2E2E2E2E2BD
:10240000E2E2E2E2E2E2E2E2E2E2E2E2E2E2E2E2AC
:10241000E2E2E2E2E2E2E2E2E2E2E2E2E2E2E2E29C
:10242000E2E2E2E2E2E2E2E2E2E2E2E2E2E2E22D41
:10243000003000340038003C0043004B005700627D
:102440000070007E008F00A000B000C000D600EE3B
:10245000000601230145016A019501C201F401272B
:10246000026402A302DC02100336034C0358035E2D
:10247000036203313233343536373839182C572953
:102480002329E028524946467C31140057415645DD
:10249000666D74201000000001000100225600004B
:1024A00044AC0000020010006461746150311400FB
:1024B0000000F123FB44756028747D7E9E7E897444
:1024C0000E61BF45D024E900EFDCCABB24A03A8CE2
:1024D000A6814381188B5B9E7EB951DA2EFE302295
:1024E0007143415F6273367EDB7E46753B624447D3
:1024F0008E26BB02B1DE56BD5BA1038DF081098142
:102500005E8A319DFBB794D85BFC6E20E341075E89
:102510009772E87D127FFC756363C54849288E0475
:1025200074E0E5BE97A2D18D4182D580AB890B9C2A
:102530007CB6DAD689FAAA1E5240C95CC571947D70
:10254000427FAD768664434A032A5F0639E278C04B
:10255000D8A3A68E9982A880FD88EB9A00B521D5D4
:10256000B8F8E51CBD3E865BED70397D6C7F577712
:10257000A365BC4BBA2B3108FFE30FC21EA5818FA8
:10258000F78282805688D09988B36BD3E6F61E1BFB
:10259000253D3E5A1070D87C8E7FFB77BB66324D4E
:1025A0006F2D020AC6E5A8C368A661905B836380AD
:1025B000B587BB9815B2B7D116F555198A3BF158B6
:1025C0002C6F707CAB7F9978CE67A44E222FD30BF3
:1025D00090E745C5B7A74891C6834A801A87AA974E
:1025E000A5B006D045F38B17EC39A057436E027C9B
:1025F000C07F3179DC681150D230A30D5AE9E5C6AD
:102600000AA93492388438808686A09639AF57CE8E
:1026100076F1C1154A384A56546D8D7BCF7FC27909
:10262000E4697B518032720F25EB87C863AA25933A
:10263000B0842C80F7859A95D2ADAACCA7EFF4137D
:10264000A636F054606C127BD77F4D7AE66AE05272
:102650002B344011F2EC2DCABFAB1D942E85278080
:102660006F859B946FAC01CBD9ED2712FF3491534A
:10267000656B917AD97FD27AE36B4154D3350E13CF
:10268000C0EED5CB20AD1A95B3852980EE84A093FA
:1026900010AB5AC90CEC591056332E52666A097A9F
:1026A000D47F507BDB6C9D557937DB148EF080CD69
:1026B00085AE1C963E8631807384AC92B6A9B6C7AF
:1026C0003FEA8A0EA931C75060697A79C87FC87B12
:1026D000CC6DF6561B39A6165DF22ECFEFAF2497C0
:1026E000CF864080FE83BD9160A814C675E8BB0C00
:1026F000FA2F5B4F5668E678B67F3A7CB86E495839
:10270000BB3A70182DF4DED05CB1329867875580E3
:102710009083D4900FA776C4ABE6EA0A492EEB4D1E
:1027200045674B789D7FA57C9F6F9859583C3A1A16
:10273000FEF591D2CEB24599058872802883F08F3C
:10274000C2A5DBC2E2E41A09952C784C3066AA7760
:102750007E7F097D7F70E25AF13D011CCFF746D4A0
:1027600044B45D9AA9889480C782138F7AA443C128
:102770001BE34807DF2A004B15650377587F677D09
:102780005A71285C883FC71DA1F9FDD5BDB57A9B5C
:102790005389BE806C823B8E37A3AEBF56E177056E
:1027A00026298449F56355762B7FBF7D2F72695D9D
:1027B0001B418C1F72FBB7D73BB79D9C048AEE80F0
:1027C0001882698DF9A11DBE92DFA5036C2705480B
:1027D000CF62A275F77E107EFD72A55EAA424F21E0
:1027E00045FD72D9BCB8C59DBA8A2581CA819E8C27
:1027F000BFA08FBCD0DDD201AF258246A561E874B1
:10280000BD7E5A7EC673DC5F3644112317FF30DB72
:1028100041BAF29E778B62818381D88B8B9F05BBF7
:102820000FDC41542B554D4C413D310D0A00000049
:10283000000000000041542B474D520D0A000000DB
:10284000000000000000000041542B5542544C4E43
:102850003D0000000000000000000041542B5542E4
:10286000544C454346473D312C33320D0A00415408
:102870002B5542544C454346473D322C36340D0AC5
:102880000041542B5542544C453D320D0A00000086
:102890000000000041542B554453433D312C300D72
:1028A0000A00000000000041542B554453433D31C1
:1028B0002C360D0A000000000000415426570D0A76
:1028C0000000000000000000000000000041542B48
:1028D000435057524F46460D0A00000000000000CA
:1028E00009024300020100C0320904000001020293
:1028F0000100052400100104240202052406000141
:1029000005240100010705810308000209040100F4
:10291000020A0000000705020240000007058202CB
:1029200040000034034300440043002000520053A1
:10293000002D00320033003200200045006D00758C
:10294000006C006100740069006F006E002000449C
:102950000065006D006F0034034D00690063007274
:10296000006F00630068006900700020005400657B
:1029700000630068006E006F006C006F00670079F4
:1029800000200049006E0063002E004E6220646546
:102990002064656661757420527820636F6D706C79
:1029A00065786520646520303020612000446566CC
:1029B00061757420696E646973706F2077617463E8
:1029C00068646F67203E203130252E0052615A2006
:1029D0006A6F75726E616C206576656E656D656E89
:1029E00074732C2020206465200052615A20636F8C
:1029F0006D70746575722061637469766174696F56
:102A00006E732C2064652000436F6E73756C746167
:102A100074696F6E206A6F75726E616C2C20202055
:102A2000202064652000436F6E73756C7461746957
:102A30006F6E2065746174206D6F64756C652C20F9
:102A400064652000436F6E73756C746174696F6E9A
:102A500020706172616D65747265732C20206465ED
:102A60002000526570726F6772616D6D6174696F7D
:102A70006E206669726D776172652C206465200036
:102A8000436F6E66696775726174696F6E206D65FC
:102A90007373616765732C20202064652000436F89
:102AA0006E66696775726174696F6E2070617261BC
:102AB0006D65747265732C206465200041542B553C
:102AC0004D52533D3233303430302C322C382C318F
:102AD0002C312C310D0A0044656661757420435217
:102AE00043206D6573736167657320617564696FF9
:102AF0002E0044656661757420636F75706C616744
:102B00006520636F6D706C6578652E004465666145
:102B1000757420636865636B73756D206669726D8B
:102B2000776172652E00466F6E6374696F6E6E65B5
:102B30006D656E74207374616E646172642E0044FE
:102B40006566617574207265636570746575722061
:102B5000726164696F2E00446566617574206465F6
:102B600074656374696F6E2070686173652E0044CC
:102B700065666175742043524320706172616D65B2
:102B8000747265732E00526564656D61727261675F
:102B900065207761746368646F672E00436F6E749D
:102BA000726F6C6520617564696F204E4F4B206EAB
:102BB0000044656661757420636861696E652061B3
:102BC0007564696F2E0041542B52554E20222461AA
:102BD00075746F72756E24220D00120100020200DE
:102BE0000008D8040A000001010200017370702679
:102BF000626C650D006174206920330D00617420E2
:102C00006920340D002D76342E32342D0041544F7E
:102C1000310D0A004D0D0A00040309044D6573755A
:102C20007265204853005331302D000D0A002200F8
:102C300000FF7BC0F3F022C1EFF023C1F0F024C10C
:102C4000F1F025C1F2F0000E2F6E000E306E000E76
:102C5000316E2FC01AF030C01BF031C01CF0000ED6
:102C60001D6E030E1E6EE9EC62F0000E326E030E56
:102C7000336E0001F46B32C01AF033C01BF0000E4B
:102C80001D6E3D0E1C6EEBEC6AF01AC032F01BC0DC
:102C900033F032503310D8B450EF16F052EF16F034
:102CA0005EEF16F03350030802E13250FF08D8B04F
:102CB0005CEF16F05EEF16F07CEF16F0FFC3F5F058
:102CC000000E326E040E336E32C020F033C021F09D
:102CD000C4EC6AF020C032F021C033F032C01AF0E8
:102CE00033C01BF0000E1D6E3D0E1C6EEBEC6AF047
:102CF0001AC032F01BC033F03350030802E13250E7
:102D00000008D8B086EF16F088EF16F091EF16F0B5
:102D10002FEEFFF03250D9263350DA22DF50000177
:102D2000F56F324A332A32C020F033C021F0C4ECB0
:102D30006AF020C032F021C033F09EEF1AF05AEC56
:102D40005EF0CAEF1BF032C0D9FF33C0DAFF0D0EC0
:102D5000DE18D8B4AEEF16F0B0EF16F0C7EF16F0ED
:102D6000010E0101A16F32C023F033C024F0080E20
:102D7000256E000E266EF8EC51F023C026F124C01B
:102D800027F125C028F126C029F1CAEF1BF0010167
:102D9000A16BCAEF1BF032C0D9FF33C0DAFF4F0E70
:102DA000DE18D8B4D6EF16F0D9EF16F0010EDAEF30
:102DB00016F0000E896F040E3226000E332232C048
:102DC000D9FF33C0DAFF730EDE18D8A4EAEF16F08D
:102DD000EDEF16F0010EEEEF16F0000E8A6FCAEF5F
:102DE0001BF032C0D9FF33C0DAFF4F0EDE18D8B463
:102DF000FCEF16F0FFEF16F0010E00EF17F0000EDB
:102E0000886FDBEF16F0010EBDEC64F0235001017A
:102E1000A06FCAEF1BF0010EBDEC64F0235001015E
:102E20009F6FCAEF1BF032C0D9FF33C0DAFF4F0EDD
:102E3000DE18D8B41EEF17F021EF17F0010E22EFC5
:102E400017F0000E876FCAEF1BF032C0D9FF33C0F6
:102E5000DAFF4F0EDE18D8B430EF17F033EF17F06B
:102E6000010E34EF17F0000E01019E6FCAEF1BF048
:102E700032C0D9FF33C0DAFF4F0EDE18D8B443EFAB
:102E800017F046EF17F0010E47EF17F0000E866FB0
:102E9000CAEF1BF032C0D9FF33C0DAFF4F0EDE1885
:102EA000D8B455EF17F058EF17F0010E59EF17F09F
:102EB000000E01019D6FCAEF1BF0010EBDEC64F026
:102EC00023500001856FCAEF1BF0010EBDEC64F0CA
:102ED00023500001846FCAEF1BF0010EBDEC64F0BB
:102EE00023500001836FCAEF1BF0010EBDEC64F0AC
:102EF00023500001826FCAEF1BF0010EBDEC64F09D
:102F000023500001816FCAEF1BF0010EBDEC64F08D
:102F100023500001806FCAEF1BF0010EBDEC64F07E
:102F2000235000017F6FCAEF1BF0010EBDEC64F06F
:102F3000235000017E6FCAEF1BF08A51D8B4A3EF73
:102F400017F0A5EF17F0B3EF17F0010EBDEC64F02A
:102F500023C062F124C063F1000E0101616F000E15
:102F6000606FCAEF1BF0640EBDEC64F023C060F12B
:102F700024C061F1000E0101636F000E626FCAEFA1
:102F80001BF08A51D8B4C7EF17F0C9EF17F0D7EF8D
:102F900017F0010EBDEC64F023C06AF024C06BF0A2
:102FA000000E0001696F000E686FCAEF1BF0640E1F
:102FB000BDEC64F023C068F024C069F0000E00018D
:102FC0006B6F000E6A6FCAEF1BF0640EBDEC64F00D
:102FD00023C05EF124C05FF1CAEF1BF032C0D9FFFD
:102FE00033C0DAFF4F0EDE18D8B4F9EF17F0FCEF5C
:102FF00017F0010EFDEF17F0000E01019C6FCAEFF4
:103000001BF032C0D9FF33C0DAFF4F0EDE18D8B440
:103010000CEF18F00FEF18F0010E10EF18F0000E83
:1030200001019B6FCAEF1BF0010EBDEC64F0235051
:1030300001019A6FCAEF1BF0010EBDEC64F0235042
:103040000101996FCAEF1BF0010EBDEC64F0235033
:103050000101986FCAEF1BF0010EBDEC64F0235024
:103060000101976FCAEF1BF0010EBDEC64F0235015
:103070000101966FCAEF1BF0010EBDEC64F0235006
:103080000101956FCAEF1BF0010EBDEC64F02350F7
:103090000101946FCAEF1BF0010EBDEC64F02350E8
:1030A0000101936FCAEF1BF08A51D8B45AEF18F0A0
:1030B0005CEF18F06AEF18F0010EBDEC64F023C06D
:1030C0005CF124C05DF1000E0101596F000E586FD4
:1030D000CAEF1BF0640EBDEC64F023C058F124C0AD
:1030E00059F1000E01015D6F000E5C6FCAEF1BF01D
:1030F0008A51D8B47EEF18F080EF18F08EEF18F0F8
:10310000010EBDEC64F023C05AF124C05BF1000E47
:103110000101576F000E566FCAEF1BF0640EBDEC35
:1031200064F023C056F124C057F1000E01015B6F1B
:10313000000E5A6FCAEF1BF032C023F033C024F0E8
:10314000010E256EFDEC50F023C032F024C033F0A8
:10315000CAEF1BF032C023F033C024F0020E256EFC
:10316000FDEC50F023C032F024C033F0CAEF1BF066
:1031700032C023F033C024F0030E256EFDEC50F076
:1031800023C032F024C033F0CAEF1BF032C023F06A
:1031900033C024F0040E256EFDEC50F023C032F055
:1031A00024C033F0CAEF1BF032C023F033C024F048
:1031B000050E256EFDEC50F023C032F024C033F034
:1031C000CAEF1BF032C023F033C024F0060E256E88
:1031D000FDEC50F023C032F024C033F0CAEF1BF0F6
:1031E00032C023F033C024F0070E256EFDEC50F002
:1031F00023C032F024C033F0CAEF1BF032C023F0FA
:1032000033C024F0080E256EFDEC50F023C032F0E0
:1032100024C033F0CAEF1BF032C023F033C024F0D7
:10322000090E256EFDEC50F023C032F024C033F0BF
:10323000CAEF1BF032C023F033C024F00A0E256E13
:10324000FDEC50F023C032F024C033F0CAEF1BF085
:10325000000E246EB40E236EF5C025F0330E266EDC
:103260005BEC62F0640E00012303F3CFEDF0F4CFCA
:10327000EEF02403F350EE27EDC0DFF1EEC0E0F1F5
:10328000CAEF1BF0F5C01AF0330E1B6E010EFFECF7
:103290006BF001018B6FCAEF1BF0F5C01AF0330E13
:1032A0001B6E010EFFEC6BF001018A6FCAEF1BF081
:1032B000F5C01AF0330E1B6E010EFFEC6BF001012E
:1032C0008C6FCAEF1BF0F5C01AF0330E1B6E000EA8
:1032D000FFEC6BF00101916FCAEF1BF00A0E6FEC6F
:1032E0005AF00001ED6FED51236E246AF5C025F010
:1032F000340E266E5BEC62F023506FEC5AF0000146
:10330000F96FCAEF1BF0000E246E000E236EF5C09D
:1033100025F0350E266E5BEC62F0235000017D6FC8
:10332000CAEF1BF0000E246E000E236EF5C025F0D0
:10333000350E266E5BEC62F0235000017C6FCAEF05
:103340001BF0F5C01AF0350E1B6E000EFFEC6BF093
:1033500000017B6FCAEF1BF0000E246E020E236E7D
:10336000F5C025F0350E266E5BEC62F023500001AF
:10337000C76FCAEF1BF0350EF519D8A4C2EF19F0CC
:10338000C4EF19F0CAEF1BF032C0D9FF33C0DAFF27
:103390000D0EDE18D8B4CFEF19F0D1EF19F0CAEF47
:1033A0001BF032C023F033C024F0060E256E010E50
:1033B000266EF8EC51F023C022F124C023F125C081
:1033C00024F126C025F1CAEF1BF0F5C01AF0350E26
:1033D0001B6E000EFFEC6BF000017A6FCAEF1BF062
:1033E000000E246E000E236EF5C025F0350E266EFD
:1033F0005BEC62F023500001796FCAEF1BF0F5C05F
:103400001AF0350E1B6E000EFFEC6BF00101906F91
:10341000CAEF1BF0000E246E000E236EF5C025F0DF
:10342000350E266E5BEC62F0235001018F6FCAEF00
:103430001BF0F5C01AF0350E1B6E010EFFEC6BF0A1
:103440000001786FCAEF1BF07851D8A42AEF1AF068
:103450002CEF1AF0CAEF1BF0020E786FCAEF1BF0C8
:10346000F5C01AF0350E1B6E000EFFEC6BF001017B
:103470008E6FCAEF1BF0020E246E300E236EF5C065
:1034800025F0350E266E5BEC62F023C0DDF124C022
:10349000DEF1CAEF1BF0000E246E000E236EF5C0A5
:1034A00025F0350E266E5BEC62F023500101DD271E
:1034B0002450DE23CAEF1BF0F5C01AF0350E1B6E48
:1034C000000EFFEC6BF001018D6FCAEF1BF0F5C031
:1034D0001AF0350E1B6E010EFFEC6BF00101EF6F61
:1034E000CAEF1BF0F5C01AF0350E1B6E010EFFEC93
:1034F0006BF00101EE6FCAEF1BF0F5C01AF0350E4C
:103500001B6E010EFFEC6BF00101ED6FCAEF1BF0BB
:10351000F5C01AF0350E1B6E010EFFEC6BF00101C9
:10352000EC6FCAEF1BF0F5C01AF0350E1B6E010EE2
:10353000FFEC6BF00101EB6FCAEF1BF00001F451DF
:10354000000AD8B4CAEF1BF0010AD8B49FEF16F0F6
:10355000030AD8B4A3EF16F0010AD8B4CBEF16F0E3
:10356000070AD8B4F1EF16F0010AD8B403EF17F048
:10357000030AD8B40BEF17F0010AD8B413EF17F011
:103580000F0AD8B425EF17F0010AD8B438EF17F0B6
:10359000030AD8B4CAEF1BF0010AD8B44AEF17F0F7
:1035A000070AD8B45DEF17F0010AD8B465EF17F039
:1035B000030AD8B46DEF17F0010AD8B475EF17F00D
:1035C0001F0AD8B47DEF17F0010AD8B485EF17F0C1
:1035D000030AD8B48DEF17F0010AD8B495EF17F0AD
:1035E000070AD8B49DEF17F0010AD8B4C1EF17F05D
:1035F000030AD8B4E5EF17F0010AD8B4EEEF17F0DC
:103600000F0AD8B4CAEF1BF0010AD8B401EF18F0C2
:10361000030AD8B414EF18F0010AD8B41CEF18F05C
:10362000070AD8B424EF18F0010AD8B42CEF18F028
:10363000030AD8B434EF18F0010AD8B43CEF18F0FC
:103640003F0AD8B444EF18F0010AD8B44CEF18F090
:10365000030AD8B454EF18F0010AD8B478EF18F080
:10366000070AD8B49CEF18F0010AD8B4AAEF18F0F2
:10367000030AD8B4B8EF18F0010AD8B4C6EF18F0AE
:103680000F0AD8B4D4EF18F0010AD8B4E2EF18F05A
:10369000030AD8B4F0EF18F0010AD8B4FEEF18F01E
:1036A000070AD8B40CEF19F0010AD8B41AEF19F0D0
:1036B000030AD8B428EF19F0010AD8B442EF19F080
:1036C0001F0AD8B44DEF19F0010AD8B458EF19F019
:1036D000030AD8B4CAEF1BF0010AD8B4CAEF1BF032
:1036E000070AD8B463EF19F0010AD8B46EEF19F0E5
:1036F000030AD8B483EF19F0010AD8B492EF19F095
:103700000F0AD8B4A1EF19F0010AD8B4ACEF19F040
:10371000030AD8B4BBEF19F0010AD8B4E5EF19F0E9
:10372000070AD8B4F0EF19F0010AD8B4FFEF19F086
:10373000030AD8B40AEF1AF0010AD8B419EF1AF044
:103740007F0AD8B424EF1AF0010AD8B430EF1AF087
:10375000030AD8B43BEF1AF0010AD8B44BEF1AF0C1
:10376000070AD8B45CEF1AF0010AD8B467EF1AF070
:10377000030AD8B472EF1AF0010AD8B47DEF1AF038
:103780000F0AD8B488EF1AF0010AD8B493EF1AF0F0
:10379000CAEF1BF00001F42B490EF465D2EF1BF0C9
:1037A000D4EF1BF03BEF16F00101E051926FDEBF4A
:1037B000DEEF1BF0DCEF1BF0E4EF1BF0000EDE6F22
:1037C000000EDD6F11EF1CF0CD0E0001D06FCC0E9E
:1037D000D16FCC0ED26F3F0ED36FDDC11AF0DEC1B8
:1037E0001BF0000E1BBEFF0E1C6E1D6E010E02ECC8
:1037F0003DF01AC0CCF01BC0CDF01CC0CEF01DC0F7
:10380000CFF0A7EC28F0CCC0E5F0CDC0E6F0CEC0FC
:10381000E7F0CFC0E8F0F3EC4DF0E5C0DDF1E6C035
:10382000DEF100017B05D8A418EF1CF01AEF1CF0A4
:103830005EEF1CF0795101012227000E232324237F
:1038400025232351070B00018B6F8B51D8B42BEF2D
:103850001CF02DEF1CF02EEF1CF08B070A0E8B03D3
:10386000F3508B6F876B01019C6B0001F351D8B44F
:103870003CEF1CF03EEF1CF057EF1CF0EF51010144
:10388000221915E10001F0510101231910E1000195
:10389000F151010124190BE10001F2510101251937
:1038A000D8B455EF1CF057EF1CF05FEF1CF0EA0E98
:1038B0000101E26F600EE16F5FEF1CF0416A1200E0
:1038C000D9CF09F0DACF0AF0F3CF0BF0F4CF0CF038
:1038D000A0A26DEF1CF06FEF1CF01EEF1DF0A1A277
:1038E00074EF1CF076EF1CF01EEF1DF00101B451D7
:1038F000D8A47DEF1CF07FEF1CF0FAEF1CF08CAE2B
:1039000084EF1CF088EF1CF0016A012A89EF1CF09B
:10391000016A013201328C5001187F0B01188C6E44
:103920000001B551D8A497EF1CF099EF1CF0A4EF5B
:103930001CF02EC142F12FC143F130C144F131C11D
:1039400045F1200EB56FB407010142A1AAEF1CF0AA
:10395000ACEF1CF0CEEF1CF0E80E7B6ECC0E7A6E56
:10396000D89045334433433342330001B507B55152
:10397000D8A4BDEF1CF0BFEF1CF0E4EF1CF0050E67
:10398000B419D8A4C6EF1CF0C8EF1CF0E4EF1CF08B
:10399000D10E7B6E5C0E7A6EE4EF1CF0F40E7B6E43
:1039A000840E7A6EB52B020EB519D8A4DAEF1CF08E
:1039B000DCEF1CF0E4EF1CF0D89045334433433384
:1039C0004233B56B0001B5070001B551D8A4EBEF48
:1039D0001CF0EDEF1CF01DEF1DF0B451D8A4F3EF77
:1039E0001CF0F5EF1CF01DEF1DF0010E0101B46F8E
:1039F0001DEF1DF083AEFFEF1CF001EF1DF008EF8F
:103A00001DF08C9EA092A190A0808D981DEF1DF0BE
:103A10008CAE0DEF1DF011EF1DF0016A012A12EFBF
:103A20001DF0016A013201328C5001187F0B011820
:103A30008C6EE80E7B6ECC0E7A6EA192A0A023EF66
:103A40001DF025EF1DF0EDEF1FF0A1A02AEF1DF0F6
:103A50002CEF1DF0EDEF1FF0CF6ACE6AB7CF0DF05F
:103A6000B8CF0EF0590E0D5C020E0E58D8A03BEFE9
:103A70001DF03DEF1DF0D8EF1FF0100E0D5C0E0E87
:103A80000E58D8B046EF1DF048EF1DF0D8EF1FF0EC
:103A9000CA0E0D5C080E0E58D8B051EF1DF053EF52
:103AA0001DF061EF1DF00001FF2F79EF1DF0D890A0
:103AB0002E322D322C322B322E9E020EFF6F79EFDA
:103AC0001DF0020E0001FF19D8A469EF1DF06BEF85
:103AD0001DF073EF1DF0D8902E322D322C322B3288
:103AE0002E8E79EF1DF0020EFF6F2B682C682D686B
:103AF0002E68FF05D8B47FEF1DF081EF1DF0DFEFDA
:103B00001FF09051D8A487EF1DF089EF1DF091EFC1
:103B10001DF04050D8B48FEF1DF091EF1DF093EFE2
:103B20001DF00101A52B00017B51D8B49AEF1DF0C7
:103B30009CEF1DF0D5EF1EF02B28D8B4A2EF1DF09E
:103B4000A4EF1DF0D5EF1EF0000E01012215016E4D
:103B5000FF0E2315026EFF0E2415036EFF0E2515B2
:103B6000046E000E2B14056EFF0E2C14066EFF0E55
:103B70002D14076EFF0E2E14086E015005180DE16E
:103B8000025006180AE10350071807E1045008180C
:103B9000D8A4CDEF1DF0CFEF1DF0D5EF1EF02B50C8
:103BA000070B016E026A620E0124D96E020E02201A
:103BB000DA6EDF2A2B50070B016E026A000E012419
:103BC000D96E010E0220DA6EDF6A9DEC69F0010108
:103BD0003E512B180DE13F512C180AE140512D1890
:103BE00007E141512E18D8A4F8EF1DF0FAEF1DF0AF
:103BF000C7EF1EF000017A51D8B401EF1EF003EFB9
:103C00001EF075EF1EF02BC001F0070E0116D8B4A0
:103C10000CEF1EF00EEF1EF0C7EF1EF02BAC13EFF3
:103C20001EF015EF1EF02CEF1EF04204D8B41BEF6F
:103C30001EF01DEF1EF02CEF1EF02B50070B8D6FAA
:103C4000D8908D33C7518D5DD8A029EF1EF02BEF92
:103C50001EF02CEF1EF08D6B2BAE31EF1EF033EF0C
:103C60001EF03DEF1EF04450D8B439EF1EF03BEF8C
:103C70001EF03DEF1EF0010E9C6F2BA642EF1EF0D2
:103C800044EF1EF067EF1EF02BA849EF1EF04BEF3C
:103C90001EF059EF1EF02B50070B016E026AD80E72
:103CA0000124D96E020E0220DA6E460EDF6EC7EFD7
:103CB0001EF02B50070B016E026AD80E0124D96E3C
:103CC000020E0220DA6E660EDF6EC7EF1EF02B507A
:103CD000070B016E026AD80E0124D96E020E022073
:103CE000DA6E300EDF6EC7EF1EF02BC001F0070E4C
:103CF0000116D8A47EEF1EF080EF1EF0C7EF1EF075
:103D00008C6B0101A36B2BC001F0380E0116D8B4E7
:103D10008CEF1EF08EEF1EF0B0EF1EF02B50300B2C
:103D200000018D6F8D3B0F0E8D17C7518D5DD8A093
:103D30009CEF1EF09EEF1EF09FEF1EF08D6B445027
:103D4000D8B4A5EF1EF0A7EF1EF0A9EF1EF0010EEC
:103D50009C6FAF0E0101E26FC80EE16FBFEF1EF066
:103D60002BAEB5EF1EF0B7EF1EF0BAEF1EF0010E4E
:103D700000018C6F000E0101E26F000EE16F000187
:103D80007951640DF3500101E127F450E2232BC077
:103D90003EF12CC03FF12DC040F12EC041F12B6807
:103DA0002C682D682E68DFEF1FF0000E2B14016EBB
:103DB000FF0E2C14026EFF0E2D14036EFF0E2E1438
:103DC000046E330E021809E1A80E03180110041046
:103DD000D8A4EDEF1EF0EFEF1EF02BEF1FF02B68D5
:103DE0009DEC69F001018E51D8B4F9EF1EF0FBEFA4
:103DF0001EF024EF1FF0B051D8B401EF1FF003EF15
:103E00001FF01CEF1FF038503910D8B40AEF1FF024
:103E10000CEF1FF01EEF1FF0700E385C030E3958C8
:103E2000D8B015EF1FF017EF1FF01EEF1FF0010EB7
:103E300000019E6F1EEF1FF0010EB06F030E396E72
:103E4000C00E386E27EF1FF0010E00019E6FFEC0FE
:103E5000B3F1C7EF1EF00101A105D8A432EF1FF0A6
:103E600034EF1FF04DEF1FF026512B180DE12751B5
:103E70002C180AE128512D1807E129512E18D8A431
:103E800044EF1FF046EF1FF04DEF1FF09DEC69F07F
:103E9000010E00019C6FC7EF1EF0A751D8B453EF7D
:103EA0001FF055EF1FF08BEF1FF02B28D8B45BEFFE
:103EB0001FF05DEF1FF08BEF1FF0000E3615016E47
:103EC000FF0E3715026EFF0E3815036EFF0E391503
:103ED000046E000E2B14056EFF0E2C14066EFF0EE2
:103EE0002D14076EFF0E2E14086E015005180DE1FB
:103EF000025006180AE10350071807E10450081899
:103F0000D8A485EF1FF087EF1FF08BEF1FF09DEC1B
:103F100069F0CFEF1EF0A651D8B491EF1FF093EFE8
:103F20001FF0C7EF1FF02B28D8B499EF1FF09BEFBD
:103F30001FF0C7EF1FF0000E3215016EFF0E331594
:103F4000026EFF0E3415036EFF0E3515046E000E63
:103F50002B14056EFF0E2C14066EFF0E2D14076E2B
:103F6000FF0E2E14086E015005180DE102500618C0
:103F70000AE10350071807E104500818D8A4C3EF5A
:103F80001FF0C5EF1FF0C7EF1FF087EF1FF0A5C1AF
:103F900001F01F0E0116D8A4D0EF1FF0D2EF1FF0D2
:103FA000D6EF1FF09DEC69F0DFEF1FF0DFEF1FF0A1
:103FB0000101A56B020E0001FF6FCFEF1EF00101A2
:103FC000F52BF551D8A4E7EF1FF0E9EF1FF0EAEF6A
:103FD0001FF0F52B010EB61AA190A3AAF2EF1FF065
:103FE000F4EF1FF07FEF21F0A4AAF9EF1FF0FBEF31
:103FF0001FF07FEF21F09CA200EF20F002EF20F0F5
:1040000004EF20F09C989C889CA409EF20F00BEF13
:1040100020F00DEF20F09C989C88AACF0FF0030EA3
:104020000001936516EF20F018EF20F0E4EF20F088
:1040300001019105D8A41FEF20F021EF20F07BEFC4
:1040400020F0330E0F18D8A428EF20F02AEF20F02C
:104050007BEF20F0FE0E3624D96E0C0E3720DA6E80
:10406000300EDE18D8A437EF20F039EF20F07BEFC8
:1040700020F0FF0E3624D96E0C0E3720DA6E300E8B
:10408000DE18D8A446EF20F048EF20F07BEF20F0B8
:10409000000E3624D96E0D0E3720DA6E410EDE1872
:1040A000D8A455EF20F057EF20F07BEF20F0010E61
:1040B0003624D96E0D0E3720DA6E380EDE18D8A4ED
:1040C00064EF20F066EF20F07BEF20F0020E362444
:1040D000D96E0D0E3720DA6E330EDE18D8A473EFCA
:1040E00020F075EF20F07BEF20F0010EAD6F000E99
:1040F000376E000E366E050E00019319D8A483EFBB
:1041000020F085EF20F0D4EF20F0FE0E3624D96E9B
:104110000C0E3720DA6E6E0EDE18D8A492EF20F067
:1041200094EF20F0D4EF20F0FF0E3624D96E0C0E61
:104130003720DA6E650EDE18D8A4A1EF20F0A3EFC9
:1041400020F0D4EF20F0000E3624D96E0D0E37206B
:10415000DA6E630EDE18D8A4B0EF20F0B2EF20F0D4
:10416000D4EF20F0010E3624D96E0D0E3720DA6E12
:10417000740EDE18D8A4BFEF20F0C1EF20F0D4EF0A
:1041800020F0020E3624D96E0D0E3720DA6E5D0E49
:10419000DE18D8A4CEEF20F0D0EF20F0D4EF20F03E
:1041A000000E376E000E366E030E3624D96E0D0EDD
:1041B0003720DA6E0FC0DFFF364A372A000E396E1D
:1041C000020E386E70EF21F0030E3624D96E0D0EFC
:1041D0003720DA6E0FC0DFFF364A372A2B0E0F1852
:1041E000D8A4F5EF20F0F7EF20F0FDEF20F0000E5F
:1041F000376E000E366E70EF21F003CDE8FF530AE4
:10420000D8A405EF21F007EF21F070EF21F004CDE5
:10421000E8FF540AD8A40FEF21F011EF21F070EF5E
:1042200021F005CDE8FF410AD8A419EF21F01BEFDA
:1042300021F070EF21F006CDE8FF520AD8A423EF59
:1042400021F025EF21F070EF21F007CDE8FF540AAF
:10425000D8A42DEF21F02FEF21F070EF21F008CD41
:10426000E8FF550AD8A437EF21F039EF21F070EFBD
:1042700021F009CDE8FF500AD8A441EF21F043EF27
:1042800021F070EF21F00ACDE8FF0D0AD8A44BEF22
:1042900021F04DEF21F070EF21F00BCDE8FF0A0A7D
:1042A000D8A455EF21F057EF21F070EF21F0935192
:1042B000D8A45DEF21F05FEF21F063EF21F0010E54
:1042C000936F70EF21F0020E9319D8A46AEF21F0DA
:1042D0006CEF21F070EF21F0030E936F70EF21F07F
:1042E000180E365C010E3758D8A079EF21F07BEF1D
:1042F00021F07FEF21F0000E376E000E366EA3A87E
:1043000084EF21F086EF21F0B8EF21F0A4A88BEF25
:1043100021F08DEF21F0B8EF21F0EB0E01016825BF
:10432000D96E0B0E6921DA6EDF50D8B49AEF21F006
:104330009CEF21F0B3EF21F0180E685D010E695972
:10434000D8B0A5EF21F0A7EF21F0B3EF21F0EB0EED
:104350006825D96E0B0E6921DA6EDF50A96E684BA5
:10436000692BB8EF21F0A398000E696F000E686FFB
:104370000CC0F4FF0BC0F3FF0AC0DAFF09C0D9FF7D
:1043800046921100000172517311D8A4CAEF21F0B6
:10439000CCEF21F034EF24F09E51D8B4D2EF21F0CD
:1043A000D4EF21F0DEEF21F09FEC6BF00009D8A4F0
:1043B000DCEF21F0DEEF21F009EF22F000019C514B
:1043C000D8A4E5EF21F0E7EF21F009EF22F0010199
:1043D000AF51D8A4EEEF21F0F0EF21F009EF22F079
:1043E000AE51D8A4F6EF21F0F8EF21F009EF22F05A
:1043F000AD51D8A4FEEF21F000EF22F009EF22F03A
:1044000000019D51D8B407EF22F009EF22F034EFFC
:1044100024F04450D8B40FEF22F011EF22F02CEF2B
:1044200024F0000170517111D8B419EF22F01BEF84
:1044300022F023EF22F09C51D8B421EF22F023EF99
:1044400022F02CEF24F08951D8B429EF22F02BEF81
:1044500022F033EF22F08751D8B431EF22F033EF5E
:1044600022F044EF22F08851D8B439EF22F03BEF2C
:1044700022F074EF22F001019C51D8A442EF22F007
:1044800044EF22F074EF22F08B8E00017B51D8B400
:104490004CEF22F04EEF22F067EF22F07B51D8B4C0
:1044A00054EF22F056EF22F074EF22F04150D8B4CE
:1044B0005CEF22F05EEF22F074EF22F0020E78192A
:1044C000D8A465EF22F067EF22F074EF22F09C5140
:1044D000D8A46DEF22F06FEF22F074EF22F0010EFE
:1044E000E86F050EBBEC2AF0000170517111D8A4E1
:1044F0007CEF22F07EEF22F081EF22F00101724B7F
:10450000732B4250D8A487EF22F089EF22F02FEFCF
:1045100023F000017B51D8B490EF22F092EF22F00B
:10452000ABEF22F07A51D8B498EF22F09AEF22F054
:10453000E5EF22F04150D8B4A0EF22F0A2EF22F034
:10454000B3EF22F0020E7819D8A4A9EF22F0ABEF56
:1045500022F02DEF23F0010E426E5EC1F7F05FC135
:10456000F8F027EF24F0010E426E5EC1F7F05FC154
:10457000F8F09E51D8B4BFEF22F0C1EF22F0D3EF94
:1045800022F0000E0101E26F140EE16F5EEC66F0A6
:104590001F0E2616000E271626500101E127275070
:1045A000E22327EF24F09D51D8B4D9EF22F0DBEFBE
:1045B00022F0DCEF22F08D6B0001B451020DF3CF3D
:1045C000E1F1F4CFE2F127EF24F09C51D8A4EBEF16
:1045D00022F0EDEF22F0FEEF22F04150D8B4F3EFDD
:1045E00022F0F5EF22F00CEF23F0020E7819D8A498
:1045F000FCEF22F0FEEF22F00CEF23F0010E426EF2
:104600005EC1F7F05FC1F8F00101A36BEA0EE26F43
:10461000600EE16F27EF24F04150D8A412EF23F091
:1046200014EF23F027EF24F09E51D8A41AEF23F0C3
:104630001CEF23F02DEF23F0010E0101A36F000109
:104640009D51D8B426EF23F028EF23F0DCEF22F0C1
:10465000010E0101A26FDCEF22F027EF24F04204EB
:10466000D8A435EF23F037EF23F027EF24F0000133
:1046700076517711D8A43FEF23F041EF23F055EFA7
:1046800023F074517511D8A448EF23F04AEF23F0BA
:1046900055EF23F070517111D8A451EF23F053EF6F
:1046A00023F055EF23F0010E966F7B51D8B45BEFEA
:1046B00023F05DEF23F0EAEF23F07A51D8B463EFF3
:1046C00023F065EF23F0A4EF23F070517111D8A40B
:1046D0006CEF23F06EEF23F0A4EF23F08D2BC75186
:1046E0008D5DD8A076EF23F078EF23F079EF23F0FB
:1046F0008D6B4150D8A47FEF23F081EF23F0BBEF07
:1047000023F09E51D8B487EF23F089EF23F09BEF7D
:1047100023F0000E0101E26F140EE16F5EEC66F013
:104720001F0E2616000E271626500101E1272750DE
:10473000E223BBEF23F00001B451020DF3CFE1F10E
:10474000F4CFE2F1BBEF23F09C51D8A4AAEF23F001
:10475000ACEF23F0B9EF23F09E51D8A4B2EF23F0D1
:10476000B4EF23F0BBEF23F0010E0101A36F9BEF29
:1047700023F062EC48F04150D8B4C1EF23F0C3EF0E
:1047800023F005EF24F0020E00017819D8A4CBEF36
:1047900023F0CDEF23F005EF24F09651D8A4D3EF0A
:1047A00023F0D5EF23F005EF24F0060EAA61DBEF2E
:1047B00023F0DDEF23F005EF24F070517111D8A440
:1047C000E4EF23F0E6EF23F005EF24F0020EAA2732
:1047D00005EF24F09651D8A4F0EF23F0F2EF23F088
:1047E00005EF24F0060EAA61F8EF23F0FAEF23F0AC
:1047F00005EF24F070517111D8A401EF24F003EFFC
:1048000024F005EF24F0E6EF23F000017051711160
:10481000D8A40DEF24F00FEF24F027EF24F062EC82
:1048200048F06AC1E2F06BC1E3F0F7EC57F0000129
:104830008951D8B41EEF24F020EF24F027EF24F0A4
:104840000101AA6BA96B5EC1F7F05FC1F8F0010E20
:104850000001716F2C0E706F00019E6B9D6B9C6B45
:104860000101AF6BAE6BAD6B0001715107E1C80E7A
:10487000705DD8B03EEF24F040EF24F041EF24F01B
:104880008B9E12000001D16F01012A29D8A44BEFA1
:1048900024F04DEF24F091EF24F0F70E1A6E010E84
:1048A0001B6E0A0E1C6E0D0E1D6E000E1F6E080E86
:1048B0001E6E06EC67F0F8C1D0F00F0E0001D017A5
:1048C0000101F751100DF3500001D02501012A6FAD
:1048D000FAC1D0F00F0E0001D0170101F951100DEF
:1048E000F3500001D02501012B6FFCC1D0F00F0E59
:1048F0000001D0170101FB51100DF3500001D0252C
:1049000001012C6FFEC1D0F00F0E0001D017010184
:10491000FD51100DF3500001D02501012D6F7DECEC
:104920006BF072C170F173C171F1030E00016E255D
:10493000D96E0D0E6F21DA6EDF6A030E1A6E0D0E40
:104940001B6E000E1D6E2D0E1C6EEBEC6AF0010E40
:104950001A240001D46F000E1B20D56FD4C01AF0AA
:10496000D5C01BF0000E1D6E3A0E1C6EEBEC6AF00B
:104970001AC0D6F01BC0D7F0D6C01AF0D7C01BF0B3
:10498000000E1D6E2D0E1C6EEBEC6AF01AC0D6F0F8
:104990001BC0D7F00001D64BD72BD605D711D8B402
:1049A000D4EF24F0D6EF24F0DDEF24F0D451D65D1F
:1049B000D06FD005D36FE0EF24F06E51EB0FD36FC3
:1049C000300E1A6E040E1B6ED4C01CF0D5C01DF044
:1049D000D3C01EF01F6A06EC67F0300E0001D3252D
:1049E000D96EDA6A040EDA22DF6AD86BF70ED825A0
:1049F000D96EDA6A010EDA226CC0E1FF6DC0E2FF07
:104A0000DFCFE7FF6C4B6D2BD82B070ED8650BEF74
:104A100025F00DEF25F0F6EF24F06CC0D9FF6DC046
:104A2000DAFF2D0EDF6E6C4B6D2BD86B6CC0D9FF8F
:104A30006DC0DAFF200EDF6E6C4B6D2BD82B030E92
:104A4000D86525EF25F027EF25F016EF25F0000EAD
:104A500024EC6DF06CC0D9FF6DC0DAFFDF6E000191
:104A60006C4B6D2BA55124EC6DF06CC0D9FF6DC063
:104A7000DAFFDF6E00016C4B6D2BA05124EC6DF062
:104A80006CC0D9FF6DC0DAFFDF6E00016C4B6D2B7F
:104A9000415024EC6DF06CC0D9FF6DC0DAFFDF6EC1
:104AA00000016C4B6D2B6CC0D9FF6DC0DAFF2D0E71
:104AB000DF6E6C4B6D2B6CC021F06DC022F070C1AD
:104AC00023F071C124F0050E256ED1EC5AF021C0FF
:104AD0006CF022C06DF06CC0D9FF6DC0DAFF2D0EF6
:104AE000DF6E00016C4B6D2BD6C0D9FFD7C0DAFF4B
:104AF000690EDE18D8A47FEF25F081EF25F0E1EFF5
:104B000025F0A65124EC6DF06CC0D9FF6DC0DAFF22
:104B1000DF6E00016C4B6D2BA45124EC6DF06CC06A
:104B2000D9FF6DC0DAFFDF6E00016C4B6D2BA35116
:104B300024EC6DF06CC0D9FF6DC0DAFFDF6E0001B0
:104B40006C4B6D2BA25124EC6DF06CC0D9FF6DC085
:104B5000DAFFDF6E00016C4B6D2BA15124EC6DF080
:104B60006CC0D9FF6DC0DAFFDF6E00016C4B6D2B9E
:104B70006CC0D9FF6DC0DAFFDF6A6CC01AF06DC07F
:104B80001BF0050E1C6E2C0E1D6E3AEC65F06CC011
:104B90001AF06DC01BF0B00E1C6E020E1D6E3AECCA
:104BA00065F06CC01AF06DC01BF0000E1D6E000E9B
:104BB0001C6EEBEC6AF01AC06CF01BC06DF061EF7C
:104BC00026F0A65124EC6DF06CC0D9FF6DC0DAFF61
:104BD000DF6E00016C4B6D2BA65124EC6DF06CC0A8
:104BE000D9FF6DC0DAFFDF6E00016C4B6D2BA45155
:104BF00024EC6DF06CC0D9FF6DC0DAFFDF6E0001F0
:104C00006C4B6D2BA35124EC6DF06CC0D9FF6DC0C3
:104C1000DAFFDF6E00016C4B6D2B010ED26FA251DB
:104C2000D8A415EF26F017EF26F020EF26F0A151BB
:104C3000D8A41DEF26F01FEF26F020EF26F0D26B50
:104C4000D25124EC6DF06CC0D9FF6DC0DAFFDF6E7D
:104C500000016C4B6D2B6CC0D9FF6DC0DAFFDF6AB1
:104C60006CC01AF06DC01BF0050E1C6E2C0E1D6E74
:104C70003AEC65F06CC01AF06DC01BF0000E1D6EB2
:104C8000000E1C6EEBEC6AF01AC06CF01BC06DF0ED
:104C90006CC0D9FF6DC0DAFF3F0EDF6E00016C4BB8
:104CA0006D2B6CC0D9FF6DC0DAFF3F0EDF6E6C4B11
:104CB0006D2B6CC0D9FF6DC0DAFF3F0EDF6E6C4B01
:104CC0006D2B4204D8A467EF26F069EF26F06BEF56
:104CD00026F0CEEC66F0D1C042F0000E0101E66F86
:104CE000030EE56F446A916BA090A1901200000141
:104CF000B251D8A47EEF26F080EF26F09FEF26F089
:104D00006EC110F06FC111F0070E126ED890113203
:104D10001032122E86EF26F01050B06F000E0101F7
:104D20006F6F000E6E6F0001A751D8B49AEF26F096
:104D30009CEF26F09FEF26F0010E0101B26F0001FB
:104D4000B151D8A4A6EF26F0A8EF26F0C7EF26F0C1
:104D50006CC110F06DC111F0070E126ED8901132B7
:104D60001032122EAEEF26F01050AF6F000E010180
:104D70006D6F000E6C6F0001A751D8B4C2EF26F022
:104D8000C4EF26F0C7EF26F0010E0101B26F00015B
:104D9000B251D8A4CEEF26F0D0EF26F09BEF28F04A
:104DA000B151D8A4D6EF26F0D8EF26F09BEF28F02B
:104DB000B051106E116AF951126E136A010E12266B
:104DC000000E13221050125C1350800A146E115002
:104DD000800A1458D8A0EFEF26F0F1EF26F0FAEF92
:104DE00026F001018705D8A4F8EF26F0FAEF26F0A7
:104DF000FEEF26F00001AE6B19EF27F0FF0E000169
:104E0000F925106E116AFF0E1122B051126E136A4D
:104E10001050125C1350800A146E1150800A1458FE
:104E2000D8B015EF27F017EF27F019EF27F0010E94
:104E3000AE6FAF51106E116AF951126E136A010E06
:104E40001226000E13221050125C1350800A146EAA
:104E50001150800A1458D8A030EF27F032EF27F015
:104E60003BEF27F001018805D8A439EF27F03BEF8D
:104E700027F03FEF27F00001AD6B5AEF27F0FF0E50
:104E80000001F925106E116AFF0E1122AF51126E4A
:104E9000136A1050125C1350800A146E1150800A6D
:104EA0001458D8B056EF27F058EF27F05AEF27F0F4
:104EB000010EAD6F01018905D8A461EF27F063EF02
:104EC00027F068EF27F0010E0001AE6F010EAD6F05
:104ED0000001AE05D8A46FEF27F071EF27F0E9EFDE
:104EE00027F0AD51D8A477EF27F079EF27F0E9EF5D
:104EF00027F07B51D8B47FEF27F081EF27F0C5EF83
:104F000027F0520EB319D8B488EF27F08AEF27F0B4
:104F1000C5EF27F04204D8B490EF27F092EF27F0C6
:104F2000C5EF27F04150D8A498EF27F09AEF27F06B
:104F3000C5EF27F07A51D8B4A0EF27F0A2EF27F001
:104F4000A5EF27F08D6BC5EF27F0010E7965ABEF6C
:104F500027F0ADEF27F0C5EF27F0FE0E7925010110
:104F6000E16FE26BFF0EE223060ED890E137E237E5
:104F7000E82EB5EF27F000018B510101E127000E6B
:104F8000E223010EA26FC5EF27F0520E0001B36FAE
:104F9000000E0101E86F0C0EE76F00019705D8A421
:104FA000D4EF27F0D6EF27F0D7EF27F08988040E4B
:104FB0004218D8B4DEEF27F0E0EF27F0E2EF27F059
:104FC0008D848D96020E0101EA6F580EE96FA6EFEF
:104FD00028F0AD05D8A4EFEF27F0F1EF27F017EF99
:104FE00028F0AE51D8A4F7EF27F0F9EF27F017EF2C
:104FF00028F0560EB36F000E0101E86F0C0EE76F3C
:1050000000019705D8A407EF28F009EF28F00AEF70
:1050100028F08988040E4218D8B411EF28F013EF55
:1050200028F0E2EF27F08D868D94E2EF27F0AE5165
:10503000D8A41DEF28F01FEF28F058EF28F0AD514D
:10504000D8A425EF28F027EF28F058EF28F0B65124
:10505000D8A42DEF28F02FEF28F030EF28F0899812
:105060000101E751E811D8B438EF28F03AEF28F001
:105070003FEF28F0E707D8A0E8074DEF28F0300E03
:105080000001B36F040E4218D8B449EF28F04BEF7B
:1050900028F04DEF28F08D948D960101EF51D8A4A2
:1050A00054EF28F056EF28F0A6EF28F0E2EF27F0B3
:1050B000AE05D8A45EEF28F060EF28F099EF28F055
:1050C000AD05D8A466EF28F068EF28F099EF28F036
:1050D000B651D8A46EEF28F070EF28F071EF28F0E9
:1050E00089980101E751E811D8B479EF28F07BEFF6
:1050F00028F080EF28F0E707D8A0E8078EEF28F027
:10510000300E0001B36F040E4218D8B48AEF28F0B5
:105110008CEF28F08EEF28F08D868D8401018C5164
:10512000D8A495EF28F097EF28F099EF28F0E2EF58
:1051300027F0A6EF28F0B151B219D8B4A2EF28F0A9
:10514000A4EF28F0A6EF28F0B26BB16B12000001BB
:10515000CF51800BD86FCF51CF25DA6FCEAFB3EFE1
:1051600028F0B5EF28F0B6EF28F0DA81DA51D8B49C
:10517000BCEF28F0BEEF28F0D1EF28F0DA29D8A450
:10518000C4EF28F0C6EF28F0CEEF28F0000ECC6F69
:10519000000ECD6F000ECE6F000ECF6FCE8FD9EF09
:1051A00028F0000ECC6F000ECD6F000ECE6F000EFB
:1051B000CF6FD351800BD81BD351D325D96FD2AF2A
:1051C000E4EF28F0E6EF28F0E7EF28F0D981D95195
:1051D000D8B4EDEF28F0EFEF28F002EF29F0D9294D
:1051E000D8A4F5EF28F0F7EF28F0FFEF28F0000E35
:1051F000D06F000ED16F000ED26F000ED36FD28F22
:105200000AEF29F0000ED06F000ED16F000ED26FA2
:10521000000ED36FD951D8B410EF29F012EF29F056
:105220001AEF29F0DA51D8A418EF29F01AEF29F073
:1052300024EF29F0000ECC6F000ECD6F000ECE6F64
:10524000000ECF6FBAEF2AF0D251CC03F3CFE3F0C8
:10525000F4CFE4F0E351DB6FDC6BDD6BDE6BE4512C
:10526000DF6FE06BE16BE26BD151CD03F3CFE3F085
:10527000F4CFE4F0E351DB27000EDC23DD23DE2353
:10528000E451DF27000EE023E123E223D051CE03D7
:10529000F3CFE3F0F4CFE4F0E351DB27000EDC239F
:1052A000DD23DE23E451DF27000EE023E123E223A8
:1052B000DDC0DEF0DCC0DDF0DBC0DCF0DB6BD0514C
:1052C000CD03F3CFE3F0F4CFE4F0E351DB27E45177
:1052D000DC23000EDD23000EDE23D151CC03F3CFFF
:1052E000E3F0F4CFE4F0E351DB27E451DC23000EDC
:1052F000DD23000EDE23DDC0DEF0DCC0DDF0DBC030
:10530000DCF0DB6BD051CC03F3CFE3F0F4CFE4F06F
:10531000E351DB27E451DC23000EDD23000EDE2306
:10532000D251CD03F3CFE3F0F4CFE4F0E351DF2724
:10533000E451E023000EE123000EE223D151CE031D
:10534000F3CFE3F0F4CFE4F0E351DF27E451E023BF
:10535000000EE123000EE223D251CE03F3CFE3F09F
:10536000F4CFE4F0E351D46FE451D56FD66BD76B33
:10537000D6C0D7F0D5C0D6F0D4C0D5F0D46BD451B8
:10538000DF27D551E023D651E123D751E223DBC0FB
:10539000D4F0DCC0D5F0DDC0D6F0DEC0D7F0190EF9
:1053A000D7EF29F0D890D733D633D533D433E82E7E
:1053B000D2EF29F0D451DF27D551E023D651E12394
:1053C000D751E223DDC0DEF0DCC0DDF0DBC0DCF075
:1053D000DB6BD951DAC0D4F0D56BD427000ED523BE
:1053E000820ED425E36FFF0ED521E46F0DEF2AF076
:1053F000D890DF37E037E137E237DEAF02EF2AF04F
:1054000004EF2AF005EF2AF0DF81D890DB37DC3794
:10541000DD37DE37E307D8A0E407E1AF12EF2AF06B
:1054200014EF2AF0F8EF29F0D96BDEAF1AEF2AF06B
:105430001CEF2AF040EF2AF0FF0EDB15D46FFF0EB1
:10544000DC15D56FFF0EDD15D66F7F0EDE15D76F1D
:10545000D451D511D611D711D8B431EF2AF033EF8A
:105460002AF037EF2AF0010ED96F40EF2AF0DFA1C2
:105470003CEF2AF03EEF2AF040EF2AF033EF2AF01B
:10548000D951D8B446EF2AF048EF2AF06CEF2AF051
:10549000010EDF27000EE023E123E223E2A153EF18
:1054A0002AF055EF2AF06CEF2AF0DFC0D4F0E0C00C
:1054B000D5F0E1C0D6F0E2C0D7F0D735D733D63338
:1054C000D533D433D4C0DFF0D5C0E0F0D6C0E1F09E
:1054D000D7C0E2F0E34BE42BE4BF77EF2AF0E451CE
:1054E00008E1E329D8A077EF2AF079EF2AF083EFDB
:1054F0002AF0000EDF6F000EE06F800EE16F7F0E6E
:10550000E26FB0EF2AF0E4BF90EF2AF0E45106E139
:10551000E305D8B08EEF2AF090EF2AF09BEF2AF047
:10552000000EDF6F000EE06F000EE16F000EE26F05
:10553000D86BB0EF2AF0E3C0DAF0FF0EDF17FF0EF2
:10554000E0177F0EE117000EE217DAA1AAEF2AF0AA
:10555000ACEF2AF0ADEF2AF0E18FD890DA31E26FAC
:10556000D851E213DFC0CCF0E0C0CDF0E1C0CEF006
:10557000E2C0CFF012000001ED6F300E0001EE6FBF
:105580000101B56BB46B000E2E6F000E2F6F000E75
:10559000306F000E316F00017B51D8B4D2EF2AF08A
:1055A000D4EF2AF072EF2BF0E851D8A4DAEF2AF00A
:1055B000DCEF2AF072EF2BF097EC46F022C12EF1CF
:1055C00023C12FF124C130F125C131F10101A251D4
:1055D000D8B4EDEF2AF0EFEF2AF0F1EF2AF02E8D9C
:1055E000A26B00017A51D8B4F8EF2AF0FAEF2AF052
:1055F0004DEF2BF04204D8A400EF2BF002EF2BF07C
:1056000041EF2BF070517111D8B409EF2BF00BEF73
:105610002BF041EF2BF04150D8A411EF2BF013EFFA
:105620002BF041EF2BF02EEF2BF001012E87460ED1
:105630000201D86F83EF2BF0180E01012E13660EB6
:105640000201D86F83EF2BF0280E01012E131FEFFC
:105650002BF0380E01012E131FEF2BF08D51000A95
:10566000D8B415EF2BF0010AD8B41CEF2BF0030AC5
:10567000D8B424EF2BF0010AD8B429EF2BF070EF47
:105680002BF04150D8B447EF2BF049EF2BF070EFDF
:105690002BF001012E8F83EF2BF00101A351D8B421
:1056A00054EF2BF056EF2BF058EF2BF02E8FA36B0F
:1056B0004204D8A45EEF2BF060EF2BF083EF2BF0C9
:1056C0002E870001D89079318D19D8A46AEF2BF07C
:1056D0006CEF2BF070EF2BF001012E8983EF2BF094
:1056E00083EF2BF00101A105D8A479EF2BF07BEF1C
:1056F0002BF083EF2BF026C12EF127C12FF128C10B
:1057000030F129C131F101012E512F113011311128
:10571000D8B48DEF2BF08FEF2BF05DEF2CF0A0EFD6
:105720002BF05FEC40F00001FE29D8B49AEF2BF08B
:105730009CEF2BF0A0EF2BF0EE07FEC0F4F1FE691A
:105740000101F4510001FE5DD8A0A9EF2BF0ABEFF1
:105750002BF0B3EF2BF0EE51D8A4B1EF2BF0B3EF59
:105760002BF091EF2BF0400E0101F46FEDC0B4F07F
:105770008CAEBDEF2BF0C2EF2BF00001E96BE92BF3
:10578000C4EF2BF00001E96BE933E9338C50E919E0
:105790007F0BE9198C6E01014269436944694569CF
:1057A0001E0E0001B56FE80E7B6ECC0E7A6E0A0EEF
:1057B000F727000EF823A090A190A192A08240505C
:1057C000D8B4E5EF2BF0E7EF2BF0EFEF2BF0C7515C
:1057D000C80DF3CFE1F1F4CFE2F1F4EF2BF0AF0E0F
:1057E0000101E26FC80EE16F00017A51D8B4FBEFFE
:1057F0002BF0FDEF2BF05CEF2CF04204D8A403EF6C
:105800002CF005EF2CF02EEF2CF0715109E13F0E3A
:10581000705DD8A00EEF2CF010EF2CF01FEF2CF0E5
:105820005EEC66F01F0E2616000E27161F0E2624AD
:105830000101E16F000E2720E26F5CEF2CF0405079
:10584000D8A425EF2CF027EF2CF05CEF2CF0EA0E1B
:105850000101E26F600EE16F5CEF2CF04150D8A4C3
:1058600034EF2CF036EF2CF03EEF2CF04050D8B453
:105870003CEF2CF03EEF2CF046EF2CF0C751C80D5A
:10588000F3CFE1F1F4CFE2F15CEF2CF0C751E96F17
:10589000EA6BD00EE903F3CFEBF0F4CFECF0EA03C0
:1058A000F350EC27070EE903F350EC27EBC0E1F1CE
:1058B000ECC0E2F15CEF2CF08D8812000001C10514
:1058C000D8A465EF2CF067EF2CF082EF2CF0BF51DD
:1058D0001F0B0009D8A46FEF2CF071EF2CF082EFB2
:1058E0002CF0628F030EC019D8A479EF2CF07BEF57
:1058F0002CF080EF2CF0010E0101C36F82EF2CF031
:105900000101C36B0001C151D8A489EF2CF08BEFCA
:105910002CF0F5EF2DF0BF511F0B020AD8A493EF26
:105920002CF095EF2CF0F5EF2DF0C3510F0B000983
:10593000D8B49DEF2CF09FEF2CF0F5EF2DF0C35174
:105940000F0BD26F030ED261A8EF2CF0AAEF2CF050
:10595000F5EF2DF0200EBE19D8A4B1EF2CF0B3EF67
:105960002CF0F5EF2DF0628FC3BFB9EF2CF0BBEF39
:105970002CF0D8EF2CF0C3510F0BD26FD251020D87
:105980001C0EF324D96E010EF420DA6EDECFD7F0B0
:10599000DDCFD8F0C3510F0BD26FD36B500ED22591
:1059A000D96E010ED321DA6EDF50D66FF3EF2CF0F3
:1059B000C3510F0BD26FD251020D160EF324D96EC4
:1059C000010EF420DA6EDECFD7F0DDCFD8F0C35170
:1059D0000F0BD26FD36B530ED225D96E010ED3218C
:1059E000DA6EDF50D66FD6B1F8EF2CF0FAEF2CF06C
:1059F000FDEF2CF0D795FEEF2CF0D785C3BF03EF5A
:105A00002DF005EF2DF016EF2DF0C3510F0BD26FD7
:105A1000D251020D1C0EF324D96E010EF420DA6E61
:105A2000D7C0DEFFD8C0DDFF25EF2DF0C3510F0B2F
:105A3000D26FD251020D160EF324D96E010EF4204E
:105A4000DA6ED7C0DEFFD8C0DDFF030EC019D8A4C0
:105A50002CEF2DF02EEF2DF062EF2DF0D7C0D9FFF7
:105A6000D8C0DAFFDFAE37EF2DF039EF2DF05AEF67
:105A70002DF0C3BF3EEF2DF040EF2DF04EEF2DF097
:105A8000C3510F0BD26FD36B500ED225D96E010EBE
:105A9000D321DA6E0101DF825AEF2DF0C3510F0BD3
:105AA000D26FD36B530ED225D96E010ED321DA6E8D
:105AB0000101DF82D7C0D9FFD8C0DAFF840EDF1220
:105AC000F5EF2DF0040ED71BD7C0D9FFD8C0DAFFF1
:105AD000DFAE6DEF2DF06FEF2DF08BEF2DF0D7C017
:105AE000D9FFD8C0DAFF7F0EDF16D7C0D9FFD8C0E4
:105AF000DAFF000EDB8C000ECD6F050ECC6FD7C029
:105B0000CEF0D8C0CFF0000ED16F020ED06FAAEC4D
:105B10005DF091EF2DF0D7C0D9FFD8C0DAFF000EAD
:105B2000DB8C040E0001D71BD6B399EF2DF09BEF51
:105B30002DF0A6EF2DF0D7C0D9FFD8C0DAFFDFAE29
:105B4000A4EF2DF0A6EF2DF0DEEF2DF0C3BFABEFED
:105B50002DF0ADEF2DF0BBEF2DF0C3510F0BD26F39
:105B6000D36B500ED225D96E010ED321DA6E01010E
:105B7000DF92C7EF2DF0C3510F0BD26FD36B530ED3
:105B8000D225D96E010ED321DA6E0101DF92D7C082
:105B9000D9FFD8C0DAFF3B0EDF16000E0001CD6F33
:105BA000050ECC6FD7C0CEF0D8C0CFF0000ED16FAD
:105BB000020ED06FAAEC5DF0E4EF2DF0D7C0D9FF54
:105BC000D8C0DAFF3B0EDF160001C3510F0BD26FB6
:105BD000D36B4C0ED225D46F0F0ED321D56FD4C00A
:105BE000D9FFD5C0DAFFFE0EDF1612000101FF6FEC
:105BF000030E1F6E0D0E206EFB0E00016E25216E32
:105C0000FF0E6F21226EFCEC64F0EB0E1A6E0B0E91
:105C10001B6E030E1C6E0D0E1D6E000E1F6E040E0D
:105C20001E6E06EC67F01AC06CF01BC06DF0040E1F
:105C300000016C27000E6D23030E6C27000E6D23F0
:105C4000FE0E6E251A6E0C0E6F211B6ED70E1C6E8B
:105C5000010E1D6E48EC5CF00009D8B432EF2EF056
:105C600034EF2EF082EF2EF00001906B87EF2EF0D4
:105C70000101FF5142EC24F0D0EF2EF0D7EC34F0CC
:105C8000D0EF2EF058EC45F0D0EF2EF0F8EC45F0C8
:105C9000D0EF2EF047EC32F0D0EF2EF0DCEC3DF000
:105CA000D0EF2EF0010E9A6FD0EF2EF0010E996F0B
:105CB000D0EF2EF0010E986FD0EF2EF0FFC1B1F1B2
:105CC000D0EF2EF0FFC1A7F0D0EF2EF00101FF5171
:105CD00059EC5FF0D0EF2EF00101FF5168EC6DF050
:105CE000D0EF2EF01CEC4AF0D0EF2EF0A6EC59F0DD
:105CF000D0EF2EF015EC6DF0D0EF2EF0F5EC6CF04F
:105D0000D0EF2EF04E0EE8CFEEFBD0EF2EF02DEEC2
:105D100006F0DF50410AD8B43EEF2EF0030AD8B4A3
:105D200038EF2EF0010AD8B44AEF2EF0070AD8B4A3
:105D300076EF2EF0020AD8B472EF2EF00C0AD8B427
:105D40007EEF2EF0040AD8B45EEF2EF0010AD8B42C
:105D500066EF2EF01F0AD8B442EF2EF0030AD8B433
:105D60007AEF2EF0070AD8B446EF2EF0030AD8B423
:105D700056EF2EF00F0AD8B44EEF2EF0020AD8B428
:105D800052EF2EF0320AD8B462EF2EF0100AD8B4D7
:105D90006CEF2EF0020AD8B45AEF2EF082EF2EF0FC
:105DA000EF0E216E0B0E226E050E0401F86F000E31
:105DB000F96FEB0EF85DFA6F0B0EF959FB6F0001EE
:105DC0006C510401FA25236E00016D510401FB2181
:105DD000246E030E256ED1EC5AF0EB0E1F6E0B0EE7
:105DE000206EEB0E00016C5D216E0B0E6D59226E64
:105DF000FCEC64F06CC01AF06DC01BF0D70E1C6E8A
:105E0000010E1D6E000E1F6E040E1E6E06EC67F076
:105E1000040E00016C27000E6D236CC0D9FF6DC00D
:105E2000DAFF0D0EDF6E6C4B6D2BC905D8A41BEF8E
:105E30002FF01DEF2FF020EF2FF0000EE8CFEBFB3F
:105E40006CC0DDF06DC0DEF0FFC1DFF052EC5DF044
:105E5000020E00019919D8B430EF2FF032EF2FF075
:105E60004DEF2FF0020E9819D8B439EF2FF03BEF19
:105E70002FF04DEF2FF0020E9A19D8B442EF2FF009
:105E800044EF2FF04DEF2FF0030E9B19D8A44BEFEA
:105E90002FF04DEF2FF079EF2FF0020E0101FF19D7
:105EA000D8A455EF2FF057EF2FF068EF2FF0A3B8DD
:105EB0005CEF2FF05EEF2FF057EF2FF09C0E0401F8
:105EC000F86FD70EE82EFED7F82FFCD779EF2FF01A
:105ED00043EC3BF098EC33F00001B851D8A473EFD9
:105EE0002FF075EF2FF068EF2FF0000EF86F1E0EF9
:105EF000F76F12004550040D000EF324D96E020E08
:105F0000F420DA6EDECFF3F2DECFF4F2DECFF5F27C
:105F1000DECFF6F24550D8A490EF2FF092EF2FF09D
:105F2000BEEF2FF00201F651F51109E1100EF45DFC
:105F3000D8A09DEF2FF09FEF2FF0A9EF2FF0000ECC
:105F4000F36F000EF46F000EF56F000EF66FD6EFD4
:105F50002FF0F651F51106E1F405D8B0B2EF2FF0AD
:105F6000B4EF2FF0B6EF2FF09FEF2FF00D0EF35F91
:105F7000000EF45BF55BF65BD6EF2FF0070E020127
:105F8000F565C5EF2FF0C7EF2FF0C9EF2FF09FEFAA
:105F90002FF0F651F51106E1F405D8B0D2EF2FF04D
:105FA000D4EF2FF0D6EF2FF09FEF2FF0000E2F6ED3
:105FB000000E306E000E316E4550080DF3CF31F0FB
:105FC0008B90030EC96E9EA6E8EF2FF0EAEF2FF03C
:105FD000E3EF2FF09E9631C0C9FF9EA6F2EF2FF09F
:105FE000F4EF2FF0EDEF2FF09E9630C0C9FF9EA684
:105FF000FCEF2FF0FEEF2FF0F7EF2FF09E962FC063
:10600000C9FF9EA606EF30F008EF30F001EF30F048
:106010009E96C9689EA60FEF30F011EF30F00AEFA0
:1060200030F09E960201F769F8693BEF30F0F851C5
:10603000C918F86FC968F839F00BF819F86FF83912
:10604000E842070BF819F26FF2390F0BF71900014C
:10605000F66F0201F839E842F80B0001F619020167
:10606000F86FF2C2F7F29EA638EF30F03AEF30F058
:1060700033EF30F09E960201F307000EF45BF55B00
:10608000F65BF3290AE1F42908E1F52906E1F6298E
:10609000D8A44DEF30F04FEF30F017EF30F08B8099
:1060A000F71FF851FF0AF86FF70E1A6E020E1B6EFB
:1060B000D70E1C6E010E1D6ECBEC47F0455038EC30
:1060C00061F00009D8B467EF30F069EF30F08BEF82
:1060D00030F04550D8A46FEF30F071EF30F07AEF28
:1060E00030F001018505D8B478EF30F07AEF30F068
:1060F0008BEF30F04550D8B480EF30F082EF30F0C5
:10610000E0EF30F001018405D8A489EF30F08BEF87
:1061100030F0E0EF30F04550D8A491EF30F093EF3D
:1061200030F0BAEF30F00101ED05D8A49AEF30F06D
:106130009CEF30F0EAEF30F00001A451D8A4A3EFB7
:1061400030F0A5EF30F0B2EF30F06F0ED16F2B0EC4
:10615000D26F000ED36F000ED46FEBEC30F0050E53
:106160000101B76F010E0001A46F040E426E7B6B3C
:10617000EAEF30F00101EC05D8A4C1EF30F0C3EF35
:1061800030F0EAEF30F00001A351D8A4CAEF30F0AC
:10619000CCEF30F0D9EF30F0D70ED16F2A0ED26F9E
:1061A000000ED36F000ED46FEBEC30F0050E010142
:1061B000B76F010E0001A36F040E426EEAEF30F0DC
:1061C0004550D8A4E6EF30F0E8EF30F0EAEF30F0D9
:1061D00019EC16F0120034C01AF035C01BF0D1C013
:1061E0001CF0D2C01DF03AEC65F034C01AF035C096
:1061F0001BF0000E1D6E000E1C6EEBEC6AF01AC058
:1062000034F01BC035F00001D351D8B40AEF31F09F
:106210000CEF31F018EF31F034C01AF035C01BF03C
:10622000300E1C6E040E1D6E3AEC65F02CEF32F051
:106230003C0ED419D8A41FEF31F021EF31F0B0EFAC
:1062400031F034C021F035C022F0010EFA25236E62
:10625000246A000E2422020E256ED1EC5AF021C0D1
:1062600034F022C035F034C0D9FF35C0DAFF200E3B
:10627000DF6E344A352A34C0D9FF35C0DAFF3A0E12
:10628000DF6E344A352A34C0D9FF35C0DAFF200E1C
:10629000DF6E344A352A100E0001FA25D96EDA6A0B
:1062A000010EDA226A0EFA25E16EE26A020EE2229D
:1062B000DE50E65CD8B05FEF31F061EF31F09FEF78
:1062C00031F034C021F035C022F06A0EFA25D96EC3
:1062D000DA6A020EDA22DF50D56FD551236E246AB6
:1062E000020E256ED1EC5AF021C034F022C035F0F8
:1062F00034C0D9FF35C0DAFF3C0EDF6E344A352A90
:1063000034C021F035C022F0100E0001FA25D96EFC
:10631000DA6A010EDA22DF50D56FD551236E246A76
:10632000020E256ED1EC5AF021C034F022C035F0B7
:1063300034C0D9FF35C0DAFFDF6A2CEF32F034C049
:10634000D9FF35C0DAFFDF6A34C01AF035C01BF060
:106350001C0E1C6E2C0E1D6E3AEC65F02CEF32F00C
:10636000640ED419D8A4B7EF31F0B9EF31F02CEFA7
:1063700032F034C021F035C022F0C751D56FD66B52
:10638000D890D537D637FF0ED525236EFF0ED621F0
:10639000246E020E256ED1EC5AF021C034F022C0DA
:1063A00035F034C0D9FF35C0DAFF200EDF6E344A35
:1063B000352A34C0D9FF35C0DAFF3A0EDF6E344AD1
:1063C000352A34C0D9FF35C0DAFF200EDF6E344ADB
:1063D000352A0001D86B16EF32F034C021F035C0F9
:1063E00022F0000ED825D96EDA6A010EDA22DF50CB
:1063F000D56FD551236E246A030E256ED1EC5AF069
:1064000021C034F022C035F034C0D9FF35C0DAFFE6
:106410002C0EDF6E344A352A34C0D9FF35C0DAFF7E
:10642000200EDF6E344A352A0001D82BC751020DE9
:10643000D851D56FD66BF350D55DD651800AD76F42
:10644000F450800AD759D8A028EF32F02AEF32F062
:10645000EDEF31F098EF31F034C01AF035C01BF099
:106460002B0E1C6E2C0E1D6E3AEC65F034C01AF02B
:1064700035C01BF0000E1D6E000E1C6EEBEC6AF0BA
:106480001AC034F01BC035F06BEC4DF012000A0E50
:106490001A6E0D0E1B6E000E1D6E2E0E1C6EEBEC9A
:1064A0006AF0010E1A240001E46F000E1B20E56F54
:1064B000E4C0D9FFE5C0DAFF690EDE18D8A463EFA7
:1064C00032F065EF32F08BEF32F0440ED16F2A0ECE
:1064D000D26F010ED36F000ED46FEBEC30F0000ED4
:1064E0002F6E000E306E000E316E2FC01AF030C0CD
:1064F0001BF031C01CF0000E1D6E030E1E6EE9EC89
:1065000062F000C23AF101C23BF102C23CF103C2A7
:106510003DF17DEF33F0E4C0D9FFE5C0DAFF6C0E4A
:10652000DE18D8A496EF32F098EF32F03EEF33F059
:10653000080ED16F2A0ED26F010ED36F000ED46FEA
:10654000EBEC30F0000E000165252F6E100E662179
:10655000306E000E6721316EF00E3016800E345C06
:10656000DD6F080E3558DE6FDDC03AF1DEC03BF15D
:106570000101000E3BBFFF0E3C6F3D6F3C2B000E38
:106580003A5F100E3B5B000E3C5B000E3D5B66C04D
:10659000DDF00F0E0001DD17DD51DF6FDE6BDEC0B9
:1065A000E0F0DFC0E1F0000EE1BFFF0EE26FE36F4D
:1065B000E05101013A270001E15101013B230001B3
:1065C000E25101013C230001E35101013D232FC0B1
:1065D0001AF030C01BF031C01CF0000E1D6E030E0F
:1065E0001E6EE9EC62F003010029D8B4FAEF32F034
:1065F000FCEF32F004EF33F0700E316402EF33F051
:1066000004EF33F07DEF33F0000E2F6E000E306E8E
:10661000700E316E000E01013A6F000E3B6F000EDE
:106620003C6F000E3D6F66C03BF1800E345C000194
:10663000DD6F080E3558DE6FDF6BDEBFDF07DF5121
:10664000E06FDD5101013A270001DE5101013B23DA
:106650000001DF5101013C230001E05101013D2314
:106660002FC01AF030C01BF031C01CF0000E1D6EA0
:10667000030E1E6EE9EC62F07DEF33F0E4C0D9FF4B
:10668000E5C0DAFF720EDE18D8A449EF33F04BEF05
:1066900033F069EF33F0000E0101716F000E706F7F
:1066A000000E736F000E726F000E3A6F000E3B6F9C
:1066B000000E3C6F000E3D6FEA0E0001D16F290EF7
:1066C000D26F010ED36F000ED46FEBEC30F07DEF84
:1066D00033F0000E01013A6F000E3B6F000E3C6F6D
:1066E000000E3D6F260E0001D16F2A0ED26F010EF3
:1066F000D36F000ED46FEBEC30F06CC0CCF06DC0FB
:10670000CDF03AC1CEF03BC1CFF03CC1D0F03DC19D
:10671000D1F0060E0001D26F73EC52F0CCC06CF0D9
:10672000CDC06DF0270E0101E46F100EE36F120073
:106730000001BE51D8A49FEF33F0A1EF33F0B7EFC3
:1067400033F0656A0F015C6B160E5F6F9F0E5D6F15
:106750007B0E5C6FADEF33F0658665A6B2EF33F06C
:10676000B4EF33F0ACEF33F0010E0001BE6FBE05A5
:10677000D8A4BDEF33F0BFEF33F0CEEF33F065BAFE
:10678000C4EF33F0C6EF33F0CEEF33F0626A0F019F
:106790005C6B5C815C89020E0001BE6F62A4D3EF6A
:1067A00033F0D5EF33F0E0EF33F00F015CA5DBEF12
:1067B00033F0DDEF33F0E0EF33F06294E0EC6BF0B8
:1067C00065A2E5EF33F0E7EF33F0EAEF33F0A1989D
:1067D000D6EF34F062A0EFEF33F0F1EF33F0FFEFDC
:1067E00033F00F015CA1F7EF33F0F9EF33F0FFEF77
:1067F00033F0FDEC4FF0040E0001BE6F629062A812
:1068000004EF34F006EF34F011EF34F00F015CA91F
:106810000CEF34F00EEF34F011EF34F037EC6BF096
:10682000629862AC16EF34F018EF34F044EF34F0B5
:106830000F015CAD1EEF34F020EF34F02FEF34F099
:10684000000E0001CD6F730ECC6F000ECE6F000EE8
:10685000CF6F000ED16F010ED06FAAEC5DF0629C7D
:106860000101C051D8B437EF34F039EF34F03AEFCA
:1068700034F0C007C051D8A440EF34F042EF34F0F8
:1068800044EF34F065EC58F062AA49EF34F04BEF76
:1068900034F055EF34F00F015CAB51EF34F053EFAF
:1068A00034F055EF34F01FEC6AF062A25AEF34F086
:1068B0005CEF34F073EF34F00F015CA362EF34F05F
:1068C00064EF34F073EF34F07F0E0001CD6FCC69CC
:1068D000000ECE6F000ECF6F000ED16F010ED06F85
:1068E000AAEC5DF0636A040E0001BE617AEF34F039
:1068F0007CEF34F07FEF34F0A198D6EF34F00F0145
:106900005CA785EF34F087EF34F0D5EF34F0000169
:10691000DC6B62A68EEF34F090EF34F0D5EF34F0FC
:1069200064CFCAF0CA31E832E8320F0BBB6F62960F
:10693000CAB59DEF34F09FEF34F0A9EF34F0500E5C
:10694000BB25D96EDA6A010EDA220101DF70B1EFE0
:1069500034F0530EBB25D96EDA6A010EDA2201013A
:10696000DF700001BB51D8A4B8EF34F0BAEF34F0B7
:10697000BEEF34F0D0EC54F0CBEF34F0000ECD6F1E
:10698000720ECC6FCA0ECE6FCF6B000ED16F000EA1
:10699000D06FAAEC5DF00001DC2B030EDC65D3EFB9
:1069A00034F0D5EF34F089EF34F0A1981200000EE6
:1069B00001014D6F000E4E6F000E4F6F0A0E1A6EE2
:1069C0000D0E1B6E000E1D6E2E0E1C6EEBEC6AF093
:1069D0001AC0DFF01BC0E0F0DFC0D9FFE0C0DAFF73
:1069E000DF6A0001DF4BE02BDFC01AF0E0C01BF0D4
:1069F000000E1D6E2D0E1C6EEBEC6AF0010E1A24BB
:106A00000001DB6F000E1B20DC6FDBC026F0DCC05A
:106A100027F0F7EC41F026C03AF127C03BF128C03F
:106A20003CF129C03DF1DBC01AF0DCC01BF0000EC8
:106A30001D6E2D0E1C6EEBEC6AF0010E1A24000187
:106A4000DD6F000E1B20DE6FDFC0D9FFE0C0DAFF74
:106A5000690EDE18D8A42FEF35F031EF35F080EF56
:106A600035F0460E0101756F500E746F0001A46B76
:106A70000101856B0001A56BA36BA26BA16BA06BE1
:106A8000C86BC851040D000EF324D96E020EF42019
:106A9000DA6E3AC1DEFF3BC1DEFF3CC1DEFF3DC125
:106AA000DEFFE16BDDC0D9FFDEC0DAFFC851040DA7
:106AB0002C0EF324D96F020EF420DA6FE151D925A0
:106AC000E16E000EDA21E26EDFCFE7FFDD4BDE2B59
:106AD000E12B030EE1656FEF35F071EF35F052EF0A
:106AE00035F07CEC4FF09E0E0001D16F2A0ED26F74
:106AF000010ED36F000ED46FEBEC30F00BEF36F0DD
:106B0000DFC0D9FFE0C0DAFF680EDE18D8A48BEF33
:106B100035F08DEF35F0A1EF35F0A56B0101866BF7
:106B2000750E4F6F010E00019B6F620ED16F2A0E22
:106B3000D26F010ED36F000ED46FEBEC30F00BEF81
:106B400036F0DFC0D9FFE0C0DAFF750EDE18D8A43A
:106B5000ACEF35F0AEEF35F0B3EF35F04E0EE8CFD9
:106B6000EEFB0BEF36F0460E0101756F500E746FA1
:106B70000001A36B0101846B70EC69F00001C86F28
:106B8000C851D8A4C6EF35F0C8EF35F0CAEF35F0DC
:106B9000AEEF35F0C851080DF3CF4FF1C851040DD9
:106BA000000EF324D96E020EF420DA6E3AC1DEFF35
:106BB0003BC1DEFF3CC1DEFF3DC1DEFFE16BDDC05E
:106BC000D9FFDEC0DAFFC851040D2C0EF324D96FB3
:106BD000020EF420DA6FE151D925E16E000EDA21C0
:106BE000E26EDFCFE7FFDD4BDE2BE12B030EE1652D
:106BF000FCEF35F0FEEF35F0DFEF35F07CEC4FF0D9
:106C0000800E0001D16F2A0ED26F010ED36F000EDD
:106C1000D46FEBEC30F04DC14AF14EC14BF14FC196
:106C20004CF10001946B120084BA19EF36F01BEF9F
:106C300036F050EF37F08D8C8D968D948D9884AA18
:106C400024EF36F026EF36F050EF37F0000E00015B
:106C5000F86F320EF76F30EF36F08D968D948D9879
:106C6000F751F811D8A437EF36F039EF36F02DEFA1
:106C700036F08D9CADB102D08D9601D08D8600018D
:106C8000AEB102D08D9401D08D840001AE51D8B444
:106C90004CEF36F04EEF36F056EF36F0AD51D8A44B
:106CA00054EF36F056EF36F064EF36F00001ADB138
:106CB00002D08D9601D08D860001AEB102D08D94A8
:106CC00001D08D8456EF36F0000EF86F320EF76F5C
:106CD00075EF36F0ADB102D08D9601D08D860001F2
:106CE000AEB102D08D9401D08D840001F751F8111E
:106CF000D8A47DEF36F07FEF36F06AEF36F08D885E
:106D000080EC6DF0000E0001F86F320EF76FF75156
:106D1000F811D8A48EEF36F090EF36F087EF36F00A
:106D20008D988E94000E736F830E726F7251731173
:106D3000D8A49DEF36F09FEF36F096EF36F0A86BB3
:106D4000380E0101F66FE4EC6CF028C526F0000E59
:106D50000001F86F1E0EF76FF751F811D8A4B3EFCA
:106D600036F0B5EF36F0ACEF36F0A86B4A0E010105
:106D7000F66FE4EC6CF005012851206E216A26C004
:106D800022F0D8902232D8902232225026C023F00E
:106D9000246A2326000E24222050235C2450800ADB
:106DA000256E2150800A2558D8B0D9EF36F0DBEF98
:106DB00036F0E3EF36F0180E2861E1EF36F0E3EF3E
:106DC00036F0E5EF36F0E3EF36F0030E0001F86F32
:106DD000E80EF76F3DEF37F00400000E396E020E3B
:106DE000386E000E376E000E366E000EE8CF03FDD3
:106DF0005A0EA96E8D8C36503710D8A402EF37F09A
:106E000004EF37F00DEF37F038503910D8A40BEFFE
:106E100037F00DEF37F0FBEF36F003CDE8FF5A0AFD
:106E2000D8A415EF37F017EF37F03DEF37F084AA0D
:106E30001CEF37F01EEF37F03DEF37F08D8C8B8E67
:106E40008B928D98000E396EA00E386E3850391026
:106E5000D8A42DEF37F02FEF37F026EF37F08D88DD
:106E6000000E396EA00E386E38503910D8A43BEFA2
:106E700037F03DEF37F034EF37F084BA42EF37F0B8
:106E800044EF37F04EEF37F00001F751F811D8A476
:106E90004CEF37F04EEF37F0ECEF36F04EEF37F0C7
:106EA0001200000E0001E16F000EE06F01018B5136
:106EB000D8B45DEF37F05FEF37F073EF38F00001D3
:106EC000A86B8E84000E736F040E726F7251731173
:106ED000D8A46DEF37F06FEF37F066EF37F08E9490
:106EE000000E736F830E726F72517311D8A47BEF13
:106EF00037F07DEF37F074EF37F0010EE26F000EE0
:106F0000D96F050EDA6FA851D927000EDA23E251A6
:106F1000D95DD96EDA51D8A0DA05DA6EDF50DB6FB1
:106F2000DB51E027000EE123E22B100EE2659BEF20
:106F300037F09DEF37F07FEF37F0D890E133E03353
:106F4000D890E133E033E0C01AF0E1C01BF096ECDA
:106F500066F00001DF6F490EDF65B1EF37F0B3EF88
:106F600037F0BCEF37F001018305D8A4BAEF37F052
:106F7000BCEF37F071EF38F00001DF51060F01016F
:106F8000F66FE4EC6CF0000E0001E16F000EE06FB4
:106F9000030EE26F000ED96F050EDA6FA851D927E4
:106FA000000EDA23E251D95DD96EDA51D8A0DA05A4
:106FB000DA6EDF50DB6FDB51E027000EE123E22BBE
:106FC000060EE265E6EF37F0E8EF37F0CAEF37F08C
:106FD000E0C01AF0E1C01BF096EC66F00001DE6F35
:106FE000100EFA25D96EDA6A010EDA22DFC0DFFF51
:106FF0006A0EFA25D96EDA6A020EDA22DEC0DFFFE7
:10700000DE51D96FDA6BDF51DB6FDC6B010EDB27F2
:10701000000EDC23D951DB5DDC51800ADD6FDA51D3
:10702000800ADD59D8B017EF38F019EF38F02DEF9E
:1070300038F0E15109E1800EE05DD8A022EF38F090
:1070400024EF38F02DEF38F001018305D8A42BEFA1
:1070500038F02DEF38F06BEF38F09C0E0001D16F57
:107060002B0ED26F000ED36F3C0ED46FEBEC30F0D2
:107070000001FA2B050EFA6540EF38F042EF38F0C8
:1070800060EF38F0A251D8A448EF38F04AEF38F05A
:1070900054EF38F0B10ED16F2B0ED26F000ED36FBC
:1070A000000ED46FEBEC30F0010E0001A26F040E65
:1070B000426E000E0101756F000E746F0001FA6BD5
:1070C0004450D8B466EF38F068EF38F06EEF38F01F
:1070D00045066EEF38F00001A26BFA6B380E010125
:1070E000F66F0001A86B1200030E000193657BEFA1
:1070F00038F07DEF38F06CEF39F0200EBE19D8A4CF
:1071000084EF38F086EF38F06CEF39F0B851D8A43E
:107110008CEF38F08EEF38F077EF39F0030E010185
:107120006625216E0D0E6721226E400E236E14EC33
:1071300057F00201FF6FFF51D8B4A1EF38F0A3EF71
:1071400038F057EF39F0010166516711D8A4ABEF61
:1071500038F0ADEF38F0AFEF38F09DEC6AF0020197
:10716000FF51010166250401FC6F000E010167213A
:107170000401FD6F00016E510401FC1909E10001D9
:107180006F510401FD19D8A4C8EF38F0CAEF38F0E8
:1071900015EF39F003CDE8FF0A0AD8A4D2EF38F092
:1071A000D4EF38F00EEF39F004CDE8FFA80AD8A4E8
:1071B000DCEF38F0DEEF38F00EEF39F005CDE8FF08
:1071C000330AD8A4E6EF38F0E8EF38F00EEF39F0E4
:1071D000030E4218D8B4EFEF38F0F1EF38F006EFB5
:1071E00039F0A39A380E0101F66F4204D8B4FBEFD0
:1071F00038F0FDEF38F006EF39F04050D8A403EF37
:1072000039F005EF39F006EF39F0B72B030E000126
:10721000F86FE80EF76F030EF6EC2DF0000E01018B
:10722000676F000E666F77EF39F00201FF510101C1
:1072300066250401FC6F000E010167210401FD6F4A
:1072400000016E510401FC5D00016F510401FD5904
:10725000D8A02DEF39F02FEF39F031EF39F00EEFE4
:1072600039F003CDE8FF0A0AD8A439EF39F03BEF33
:1072700039F00EEF39F00201FF5101016627000ECF
:107280006723180E665D010E6759D8A04AEF39F0E2
:107290004CEF39F055EF39F000019B6B996B9A6B0D
:1072A000986BA6EC59F077EF39F077EF39F00001E1
:1072B000F751F811D8A45FEF39F061EF39F055EFCD
:1072C00039F0030E4218D8A468EF39F06AEF39F0AC
:1072D00055EF39F04CEF39F0030E4218D8A473EF94
:1072E00039F075EF39F077EF39F04CEF39F01200E3
:1072F000A388A3B87EEF39F080EF39F079EF39F049
:10730000000E376E000E366E000E396E400E386E6F
:107310008CEF39F0E2EC4CF0FF0E3624D96E0C0EF7
:107320003720DA6E4F0EDE18D8A499EF39F09BEFB4
:1073300039F0C8EF39F0000E3624D96E0D0E372023
:10734000DA6E4B0EDE18D8A4A8EF39F0AAEF39F0A8
:10735000C8EF39F0010E3624D96E0D0E3720DA6EE3
:107360000D0EDE18D8A4B7EF39F0B9EF39F0C8EF39
:1073700039F0020E3624D96E0D0E3720DA6E0A0E61
:10738000DE18D8B4C6EF39F0C8EF39F0D1EF39F0D4
:1073900038503910D8A4CFEF39F0D1EF39F08AEF57
:1073A00039F038503910D8B4D8EF39F0DAEF39F075
:1073B0005BEF3AF000019251D8A4E1EF39F0E3EF2E
:1073C00039F010EF3AF0FD0E3624D96E0C0E37204E
:1073D000DA6EDF6A030E1A6E0D0E1B6E000E1D6E46
:1073E0003A0E1C6EEBEC6AF0010E1A24216E000EB0
:1073F0001B20226EB00E1A6E020E1B6E21C01CF0F6
:1074000022C01DF03AEC65F0B00E1A6E020E1B6E33
:10741000290E1C6E2C0E1D6E3AEC65F057EF3AF0FB
:107420009205D8A416EF3AF018EF3AF03BEF3AF095
:10743000FC0E3624D96E0C0E3720DA6EDF6A030E8E
:107440001A6E0D0E1B6E000E1D6E220E1C6EEBECE6
:107450006AF0010E1A24216E000E1B20226EB00E5F
:107460001A6E020E1B6E21C01CF022C01DF03AECF9
:1074700065F057EF3AF0090E9219D8A442EF3AF0AE
:1074800044EF3AF04AEF3AF0020E936F0101B96906
:1074900057EF3AF00B0E9219D8A451EF3AF053EF90
:1074A0003AF057EF3AF0040E936F57EF3AF00001BD
:1074B000922B5DEF3AF00201B06B120000017651A1
:1074C0007711D8A466EF3AF068EF3AF071EF3AF02E
:1074D00074517511D8B46FEF3AF071EF3AF0B2EF22
:1074E0003AF0560E4318D8A478EF3AF07AEF3AF013
:1074F00082EF3AF0020EC96F00017607D8A0770735
:107500002AEF3BF0520E4318D8A489EF3AF08BEFE4
:107510003AF02AEF3BF00101A805D8A492EF3AF027
:1075200094EF3AF0AAEF3AF000018651D8B49BEFFD
:107530003AF09DEF3AF0A3EF3AF0040EC96F010163
:10754000A86B2AEF3BF0030EC96F010E0101A86F73
:107550007CEF3AF0050E0001C96F010E0101A86F22
:107560007CEF3AF09605D8A4B8EF3AF0BAEF3AF0CB
:107570002AEF3BF0560E4318D8A4C1EF3AF0C3EF00
:107580003AF0DEEF3AF062C11AF063C11BF060C15D
:107590001CF061C11DF085C01EF083C01FF081C0CA
:1075A00020F080C021F07DC022F0020E50EC60F08F
:1075B00000017607D8A0770728EF3BF0520E43185A
:1075C000D8A4E5EF3AF0E7EF3AF026EF3BF086512A
:1075D000D8B4EDEF3AF0EFEF3AF008EF3BF06AC0C5
:1075E0001AF06BC01BF068C01CF069C01DF084C0AD
:1075F0001EF082C01FF07FC020F07EC021F07CC052
:1076000022F0040E50EC60F00101A86B28EF3BF073
:107610006AC01AF06BC01BF068C01CF069C01DF096
:1076200084C01EF082C01FF07FC020F07EC021F019
:107630007CC022F0030E50EC60F000017607D8A069
:107640007707010E0101A86F28EF3BF0CEEC66F042
:107650000001966B0001F751F811D8A432EF3BF00E
:1076600034EF3BF042EF3BF0CEEC66F0560E4318A1
:10767000D8A43DEF3BF03FEF3BF042EF3BF0010E73
:107680000101F06F1200010178517911D8B44BEF6C
:107690003BF04DEF3BF060EF3BF078C1D9FF79C193
:1076A000DAFFDFBE56EF3BF05AEF3BF0216A212AAA
:1076B0005BEF3BF0216A2150226E236A64EF3BF0BE
:1076C000000E236E000E226E22502310D8B46BEFF2
:1076D0003BF06DEF3BF06FEF3BF022EF3CF0030E21
:1076E0000001B819D8A477EF3BF079EF3BF07AEFBF
:1076F0003BF0B86BB851D8A480EF3BF082EF3BF081
:1077000084EF3BF022EF3CF0020EB819D8A48BEFC7
:107710003BF08DEF3BF0A1EF3BF0010E1A6E000E37
:107720001B6E000E1C6E000E1D6E020EA1EC56F0BC
:107730001AC078F11BC079F1030E0001B86F22EF77
:107740003CF0B805D8A4A7EF3BF0A9EF3BF022EF3F
:107750003CF0400EB765AFEF3BF0B1EF3BF0B5EF5B
:107760003BF0400E256EB7EF3BF0B7C025F025503B
:10777000B75DB76FB00E01017C6F040E7D6F25C041
:1077800024F0BB51D8A4C7EF3BF0C9EF3BF0F3EFB7
:107790003BF0DAEF3BF07EC1D9FF7FC1DAFF7CC15D
:1077A000E1FF7DC1E2FFDFCFE7FF7C4B7D2B7E4B0E
:1077B0007F2B24062450D8A4E0EF3BF0E2EF3BF00F
:1077C000CBEF3BF0FBEF3BF07EC1D9FF7FC1DAFF8F
:1077D0007CC1E1FF7DC1E2FFDFCFE7FF7C4B7D2B6A
:1077E0007E4B7F2B24062450D8A4F9EF3BF0FBEF0F
:1077F0003BF0E4EF3BF00001B751D8A402EF3CF0BE
:1078000004EF3CF013EF3CF0400E2518D8A40BEF2A
:107810003CF00DEF3CF011EF3CF0020EB86F13EFAF
:107820003CF0030EB86F010E1A6EB00E1B6E040E04
:107830001C6E25C01DF0020EA1EC56F01AC078F1A6
:107840001BC079F112000001DC6B4450D8B42BEF5F
:107850003CF02DEF3CF001EF3DF0DD6B8FEF3CF0A5
:107860007A51D8B436EF3CF038EF3CF068EF3CF09A
:10787000620EDD25D96EDA6A020EDA22DF50D8A454
:1078800044EF3CF046EF3CF08EEF3CF07951DD19CF
:10789000D8B44DEF3CF04FEF3CF08EEF3CF0000ED3
:1078A000DD25D96EDA6A010EDA22FA0EDF605BEFAF
:1078B0003CF05DEF3CF064EF3CF0000EDD25D96E4E
:1078C000DA6A010EDA22DF2A010EDC6F8EEF3CF05D
:1078D000DD51D8A46EEF3CF070EF3CF08EEF3CF041
:1078E000620EDD25D96EDA6A020EDA22DF50D8A4E4
:1078F0007CEF3CF07EEF3CF08EEF3CF0000EDD259F
:10790000D96EDA6A010EDA22FA0EDF608AEF3CF0F5
:107910008CEF3CF064EF3CF05DEF3CF0DD2BC751A9
:10792000020DDD51D96FDA6BF350D95DDA51800A5F
:10793000DB6FF450800ADB59D8A0A1EF3CF0A3EF35
:107940003CF030EF3CF0DC51D8A4A9EF3CF0ABEFB9
:107950003CF0C9EF3CF08C51D8A4B1EF3CF0B3EF50
:107960003CF0C9EF3CF04150D8B4B9EF3CF0BBEF6C
:107970003CF0C8EF3CF00101B72B040E4218D8A42C
:10798000C4EF3CF0C6EF3CF0C8EF3CF08B82426A9B
:10799000416A00018C51D8B4D0EF3CF0D2EF3CF0FA
:1079A000EFEF3CF04150D8A4D8EF3CF0DAEF3CF0D8
:1079B000EFEF3CF0020E7819D8A4E1EF3CF0E3EFD2
:1079C0003CF0EDEF3CF0260ED16F2B0ED26F000E87
:1079D000D36F000ED46FEBEC30F0010E416E00015E
:1079E000DD6B620EDD25D96EDA6A020EDA22DF6AFD
:1079F000DD2B070EDD65FFEF3CF001EF3DF0F1EF11
:107A00003CF01200226E2250D8B409EF3DF00BEF8B
:107A10003DF02DEF3DF01DBE12EF3DF010EF3DF0BB
:107A20002DEF3DF01AC01EF01BC01FF01CC020F04F
:107A30001DC021F01E1E1F1E201E211E1E2A000E0C
:107A40001F22202221221EC024F01FC025F020C0AA
:107A500026F021C027F035EF3DF01AC024F01BC0FE
:107A600025F01CC026F01DC027F01A501B101C105A
:107A70001D10D8A43EEF3DF040EF3DF04AEF3DF041
:107A8000000E1A6E000E1B6E000E1C6E000E1D6E98
:107A9000DBEF3DF0960E236E54EF3DF0232AD89095
:107AA0002732263225322432000E24141E6E000E98
:107AB00025141F6E000E2614206EFE0E2714216E54
:107AC0001E501F1020102110D8A469EF3DF06BEF5D
:107AD0003DF04EEF3DF079EF3DF0232A010E2426D4
:107AE000000E252226222722D89027322632253240
:107AF0002432000E24141E6E000E25141F6E000E7C
:107B00002614206EFF0E2714216E1E501F10201009
:107B10002110D8A48EEF3DF090EF3DF06DEF3DF0D9
:107B200098EF3DF02306D8902436253626362736A2
:107B300026BE9DEF3DF09FEF3DF0A7EF3DF0020E1A
:107B40002360A5EF3DF0A7EF3DF092EF3DF023B0AD
:107B5000ACEF3DF0AEEF3DF0AFEF3DF0269ED8909C
:107B6000233223C01EF01F6A206A216A1EC021F042
:107B7000206A1F6A1E6A1E5024121F5025122050B0
:107B80002612215027122250D8B4C9EF3DF0CBEF76
:107B90003DF0D3EF3DF01DBED2EF3DF0D0EF3DF014
:107BA000D3EF3DF0278E24C01AF025C01BF026C06D
:107BB0001CF027C01DF012000001D26B000EE8CFB0
:107BC0000EFD0A0E1A6E0D0E1B6EC9EC4BF01AC09C
:107BD000D0F01BC0D1F00101E3510001D0190BE13D
:107BE0000101E4510001D119D8B4F9EF3DF0FBEFE8
:107BF0003DF0B0EF3EF0D0C0E3F1D1C0E4F16CC095
:107C000021F06DC022F0D0C023F0D1C024F0040ECA
:107C1000256ED1EC5AF021C06CF022C06DF06CC022
:107C2000D9FF6DC0DAFF2D0EDF6E00016C4B6D2B9E
:107C300001013A513B113C113D11D8B422EF3EF005
:107C400024EF3EF0B4EF3EF0000E0001D225D96ED5
:107C5000DA6A030EDA22DF50D8A431EF3EF033EFB8
:107C60003EF03DEF3EF06CC0D9FF6DC0DAFF400E34
:107C7000DF6E6C4B6D2B4BEF3EF0000ED225D96EB4
:107C8000DA6A030EDA226CC0E1FF6DC0E2FFDFCFDB
:107C9000E7FF39EF3EF0D22B01013A07000E3B5BC4
:107CA0003C5B3D5B0001D251D8B459EF3EF05BEF35
:107CB0003EF067EF3EF001013A513B113C113D119E
:107CC000D8A465EF3EF067EF3EF024EF3EF0000EE3
:107CD0002F26010E3022000E3122700E316473EF18
:107CE0003EF075EF3EF07BEF3EF0000E2F6E000E83
:107CF000306E700E316E2FC01AF030C01BF031C0E4
:107D00001CF0000E1D6E030E1E6EE9EC62F0010108
:107D10003D513C1106E13B05D8B091EF3EF093EFA9
:107D20003EF0AAEF3EF0700E315CD8A09AEF3EF024
:107D30009CEF3EF0AAEF3EF0000E1A6E030E1B6E93
:107D4000800E1C6E080E1D6E010E1F6E000E1E6E44
:107D500006EC67F06CC064F16DC065F1B4EF3EF005
:107D600064C16CF065C16DF01200030E00019365F3
:107D7000BCEF3EF0BEEF3EF078EF3FF038503910E8
:107D8000D8A4C5EF3EF0C7EF3EF0D0EF3EF036503E
:107D90003710D8A4CEEF3EF0D0EF3EF0DBEF3EF050
:107DA000110E361806E13704D8A4D9EF3EF0DBEF08
:107DB0003EF03FEF3FF0020E3624D96E0D0E372015
:107DC000DA6E0D0EDE18D8A4E8EF3EF0EAEF3EF0D2
:107DD00057EF3FF003CDE8FF0A0AD8A4F2EF3EF0D8
:107DE000F4EF3EF039EF3FF09DEC6AF004CDE8FF90
:107DF000A80AD8A4FEEF3EF000EF3FF039EF3FF0C5
:107E000005CDE8FF330AD8A408EF3FF00AEF3FF0B2
:107E100039EF3FF0020E4218D8B411EF3FF013EFE4
:107E20003FF031EF3FF04A0E0101F66F4204D8B443
:107E30001CEF3FF01EEF3FF031EF3FF04050D8A471
:107E400024EF3FF026EF3FF031EF3FF006CDE8FFA3
:107E50004A0AD8B42EEF3FF030EF3FF031EF3FF059
:107E6000B72B030E0001F86FE80EF76F020EF6EC69
:107E70002DF0000E376E000E366E57EF3FF0F751C3
:107E8000F811D8A446EF3FF048EF3FF057EF3FF02E
:107E9000020E4218D8A44FEF3FF051EF3FF057EFDA
:107EA0003FF09B6B996B9A6B986BA6EC59F0425024
:107EB000D8A45DEF3FF05FEF3FF08BEF3FF0C0ECF9
:107EC0006BF08BEF3FF00101B951D8A46AEF3FF09E
:107ED0006CEF3FF08BEF3FF048EC55F08BEF3FF04D
:107EE00090EC5BF08BEF3FF0C9EC69F08BEF3FF06B
:107EF0009351000AD8B463EF3FF0010AD8B470EF91
:107F00003FF0030AD8B48BEF3FF0010AD8B474EF06
:107F10003FF08BEF3FF01200ECEC5BF085BA93EF93
:107F20003FF095EF3FF097EF3FF014EC36F088EC20
:107F30006DF0AAEC67F039EC6CF00009D8A4A3EF5F
:107F40003FF0A5EF3FF09BEF3FF07BEC51F0BBEC37
:107F500055F00DEC5AF086EC57F08D8C0201B06BA9
:107F60000101B969FDEC4FF00400B2EC65F0C2EC20
:107F700021F05FEC40F098EC33F0CEEF3FF01DECD9
:107F80006CF0E5EF3FF026EC66F0E5EF3FF013EC28
:107F900044F0E5EF3FF0426AE5EF3FF04250000A5F
:107FA000D8B4C7EF3FF0010AD8B4BFEF3FF0030ADF
:107FB000D8B4E5EF3FF0010AD8B4E5EF3FF0070A87
:107FC000D8B4C3EF3FF0CBEF3FF0B5EC3EF074EC2C
:107FD00038F0020E00019019D8A4F1EF3FF0F3EF52
:107FE0003FF0FAEF3FF0A3A8F8EF3FF0FAEF3FF0D1
:107FF0000BEF40F0030E9019D8A401EF40F003EF0F
:1080000040F00DEF40F0B851D8A409EF40F00BEF6D
:1080100040F00DEF40F004EC5FF043EC3BF000016A
:10802000F85107E10F0EF75DD8B019EF40F01BEFE4
:1080300040F023EF40F0B8EC63F0FBEC63F05BEC56
:108040006DF041EC69F0E2EC4CF0A0B22AEF40F0A8
:108050002CEF40F0B4EF3FF0050E00019319D8A4C7
:1080600034EF40F036EF40F03DEF40F084AA02D00C
:108070008D8801D08D98B4EF3FF0040E9319D8A4E9
:1080800044EF40F046EF40F05AEF40F084AA4BEF47
:1080900040F050EF40F00401FE6BFE2B52EF40F039
:1080A0000401FE6BFE3B8D50FE19EF0BFE198D6E29
:1080B000B4EF3FF08D98B4EF3FF095EF11F0000171
:1080C000C951D8B466EF40F068EF40F02AEF41F0B4
:1080D0009751D8A46EEF40F070EF40F0A7EF40F05A
:1080E000898881EC6CF062EC48F06AC1E2F06BC107
:1080F000E3F0F7EC57F00001C951040D000EF32432
:10810000D96E020EF420DA6EDECF3AF1DECF3BF10B
:10811000DECF3CF1DECF3DF1000E2F6E000E306E53
:10812000000E316EC951080DF3CF31F02FC01AF097
:1081300030C01BF031C01CF0000E1D6E030E1E6E11
:10814000E9EC62F0010E0001976F2AEF41F00101A6
:108150003D513C113B1107E1210E3A5DD8B0B3EF20
:1081600040F0B5EF40F0F5EF40F0000E2F241A6E0E
:108170001B6A030E1B223AC11CF015EC68F00009C3
:10818000D8B4C5EF40F0C7EF40F02AEF41F08E843D
:108190000001976B830E0101DD250001726F000E57
:1081A0000101DE210001736FC96B76517711D8A4EC
:1081B000DCEF40F0DEEF40F02AEF41F07451751132
:1081C000D8A4E5EF40F0E7EF40F02AEF41F0AC6BC8
:1081D000400EFC6F500EFB6F020E0101F26F020E9B
:1081E000F16F0001A96B2AEF41F0000E2F241A6EE7
:1081F0001B6A030E1B22200E1C6E15EC68F0000992
:10820000D8B405EF41F007EF41F02AEF41F0200E1E
:1082100001013A5F000E3B5B3C5B3D5B200E2F266D
:10822000000E3022000E31222F50D8A41AEF41F058
:108230001CEF41F02AEF41F02FC01AF030C01BF0C4
:1082400031C01CF0000E1D6E030E1E6EE9EC62F0D4
:108250002AEF41F01200000E0001ED6F000EEC6FEE
:10826000EE6BA851D8A437EF41F039EF41F0F6EFAB
:1082700041F04204D8A43FEF41F041EF41F0A4EFB8
:1082800041F076517711D8A448EF41F04AEF41F020
:1082900053EF41F074517511D8B451EF41F053EFE1
:1082A00041F07CEF41F0EE6B000EEE25D96EDA6AFC
:1082B000050EDA22DF50E76FE751EC27000EED23C1
:1082C000EE2B1F0EEE6567EF41F069EF41F054EFC2
:1082D00041F0ECC0E7F0EDC0E8F0D890E833E733C8
:1082E000D890E833E733D890E833E733E7C0EAF0D3
:1082F000E8C0EBF0BCEF41F08E84000EEE25D96EA5
:10830000DA6A050EDA22DF50E76FE751EC27000E3C
:10831000ED23EE2BEE51D8A490EF41F092EF41F017
:108320007DEF41F0ECC0E7F0EDC0E8F0060EE96F3C
:10833000D890E833E733E92F98EF41F0E7C0EAF04F
:10834000E8C0EBF0BCEF41F08E84000EEE25D96E54
:10835000DA6A050EDA22DF50E76FE751EC27000EEC
:10836000ED23EE2BEE51D8A4B8EF41F0BAEF41F077
:10837000A5EF41F092EF41F0EAC01AF0EBC01BF01C
:1083800096EC66F00001AB6FFAEC5CF04250D8B4AA
:10839000CCEF41F0CEEF41F0E1EF41F0000176513A
:1083A0007711D8A4D6EF41F0D8EF41F0E9EF41F0D2
:1083B00074517511D8A4DFEF41F0E1EF41F0E9EF1E
:1083C00041F0EAC0E2F0EBC0E3F0F7EC57F0EDEF7C
:1083D00041F0EAC06AF1EBC06BF10001A851D8B4DA
:1083E000F4EF41F0F6EF41F0EDEF41F01200000E36
:1083F0000001D26F000ED36F000ED46F000ED56F48
:10840000D16B05EF42F0264A272A26C0D9FF27C0A4
:10841000DAFF200EDE18D8B410EF42F012EF42F06F
:1084200003EF42F026C0D9FF27C0DAFFDF5000017A
:10843000CC6FF70ECC27040ECC6521EF42F023EF72
:1084400042F003EF42F026C0D9FF27C0DAFF2D0E1D
:10845000DE18D8A42EEF42F030EF42F036EF42F0B3
:10846000010ED16F264A272A77EF42F026C0D9FFA6
:1084700027C0DAFF2B0EDE18D8A441EF42F043EFFD
:1084800042F077EF42F032EF42F026C0D9FF27C02A
:10849000DAFFDF50CC6FD00ECC25CD6FCE6BFF0E48
:1084A000CE23CF6BCEBFCF07CF51D06FD2C01AF043
:1084B000D3C01BF0D4C01CF0D5C01DF00A0E1E6E38
:1084C000000E1F6E000E206E000E216EE0EC67F0B5
:1084D0000001CD511A5CD26FCE511B58D36FCF51D2
:1084E0001C58D46FD0511D58D56F32EF42F026C0C2
:1084F000D9FF27C0DAFFDF50CC6FD00ECC27090E92
:10850000CC6585EF42F087EF42F045EF42F0D15164
:10851000D8A48DEF42F08FEF42F0AAEF42F0D2C024
:10852000CCF0D3C0CDF0D4C0CEF0D5C0CFF0CC1FAE
:10853000CD1FCE1FCF1FCC2B000ECD23CE23CF239C
:10854000CCC026F0CDC027F0CEC028F0CFC029F097
:10855000B2EF42F0D2C026F0D3C027F0D4C028F04A
:10856000D5C029F01200560E4318D8A4BAEF42F035
:10857000BCEF42F006EF43F00101AA51D8A4C3EFCB
:1085800042F0C5EF42F002EF43F09E51D8B4CBEF7A
:1085900042F0CDEF42F0E4EF42F062C11AF063C165
:1085A0001BF060C11CF061C11DF085C01EF083C0CE
:1085B0001FF081C020F080C021F07DC022F0010EAC
:1085C00050EC60F0FDEF42F062C11AF063C11BF0A5
:1085D00060C11CF061C11DF085C01EF083C01FF09A
:1085E00081C020F080C021F07DC022F0020E50EC4E
:1085F00060F000017607D8A07707010E0101AA6F8D
:1086000068EF43F0CEEC66F068EF43F0520E43188B
:10861000D8A40DEF43F00FEF43F002EF43F0010158
:10862000A951D8B416EF43F018EF43F028EF43F008
:10863000A951D8B41EEF43F020EF43F002EF43F00E
:108640009D51D8B426EF43F028EF43F002EF43F0FA
:1086500000018651D8B42FEF43F031EF43F04AEFD9
:1086600043F06AC01AF06BC01BF068C01CF069C010
:108670001DF084C01EF082C01FF07FC020F07EC0BD
:1086800021F07CC022F0040E50EC60F00101A86BD8
:1086900066EF43F06AC01AF06BC01BF068C01CF0B4
:1086A00069C01DF084C01EF082C01FF07FC020F0A2
:1086B0007EC021F07CC022F0030E50EC60F000017F
:1086C0007607D8A07707010E0101A86F010EA96FE8
:1086D00012000001AA6B010E0101AB6FAA6BA96B1E
:1086E000560E4318D8A477EF43F079EF43F0C5EF67
:1086F00043F0F051D8A47FEF43F081EF43F0AAEFAD
:1087000043F000018751D8B488EF43F08AEF43F07B
:10871000AAEF43F001019E51D8B491EF43F093EFDB
:1087200043F0AAEF43F062C11AF063C11BF060C1CD
:108730001CF061C11DF085C01EF083C01FF081C018
:1087400020F080C021F07DC022F0010E50EC60F0DE
:1087500010EF44F062C11AF063C11BF060C11CF05D
:1087600061C11DF085C01EF083C01FF081C020F0E4
:1087700080C021F07DC022F0020E50EC60F00001BC
:108780007607D8A0770710EF44F0520E4318D8A40C
:10879000CCEF43F0CEEF43F00EEF44F000018651F2
:1087A000D8B4D5EF43F0D7EF43F0F0EF43F06AC011
:1087B0001AF06BC01BF068C01CF069C01DF084C0CB
:1087C0001EF082C01FF07FC020F07EC021F07CC070
:1087D00022F0040E50EC60F00101A86B10EF44F0A1
:1087E0006AC01AF06BC01BF068C01CF069C01DF0B5
:1087F00084C01EF082C01FF07FC020F07EC021F038
:108800007CC022F0030E50EC60F000017607D8A087
:108810007707010E0101A86F10EF44F0CEEC66F06F
:108820000101F06B120000017B51D8B41AEF44F043
:108830001CEF44F02EEF44F00101E151E211D8A405
:1088400024EF44F026EF44F02EEF44F0000E000138
:10885000E86F050EBBEC2AF023EC3CF00001F75169
:10886000F811D8A436EF44F038EF44F0A7EF44F005
:10887000A0804050D8A43FEF44F041EF44F0A3EF74
:1088800044F063EF44F07AEC2FF0A2EF44F0AFEC49
:108890005EF0A2EF44F051EC37F0A2EF44F02FEC81
:1088A00063F0A2EF44F086EC57F0A2EF44F057ECEF
:1088B0004CF0A2EF44F0C0EC6CF0A2EF44F014ECEA
:1088C00062F0A2EF44F04550000AD8B443EF44F000
:1088D000010AD8B443EF44F0030AD8B443EF44F09C
:1088E000010AD8B443EF44F0070AD8B443EF44F088
:1088F000010AD8B443EF44F0030AD8B443EF44F07C
:10890000010AD8B443EF44F00F0AD8B447EF44F05B
:10891000010AD8B44BEF44F0030AD8B44FEF44F047
:10892000010AD8B453EF44F0070AD8B457EF44F023
:10893000010AD8B45BEF44F0030AD8B4A2EF44F0C4
:108940005FEF44F0452AE5C1F7F0E6C1F8F0445086
:10895000D8B4ADEF44F0AFEF44F0B6EF44F02BECF9
:1089600041F0A1EC5CF04AEC6AF08E941200800EAB
:108970000001BF19D8A4BFEF44F0C1EF44F057EF96
:1089800045F0C00E626F48EF45F0DA0E606F2B0EB7
:10899000616F000E646F120E636F57EF45F0C151A7
:1089A000020D820EF324F66E240EF420F76EF86AA0
:1089B000000EF8220900F5CF60F00A00F5CF61F053
:1089C000020E60251A6E000E61211B6E1AC0F6FFA2
:1089D0001BC0F7FF000EF86E0F0EF76403D00800FF
:1089E000F55005D0F6CFE1FFF7CFE2FFE7500001E9
:1089F000636F030E60251A6E000E61211B6E1AC094
:108A0000F6FF1BC0F7FF000EF86E0F0EF76403D0E1
:108A10000800F55005D0F6CFE1FFF7CFE2FFE750B1
:108A20000001646F57EF45F0030EC1611AEF45F086
:108A30001CEF45F045EF45F0C151020D7C0EF324CB
:108A4000F66E240EF420F76EF86A000EF822090084
:108A5000F5CF60F00A00F5CF61F060C0F6FF61C0AD
:108A6000F7FF000EF86E0F0EF76403D00800F55004
:108A700005D0F6CFE1FFF7CFE2FFE7501A6E1A50AC
:108A80000001636F646B57EF45F0626B57EF45F081
:108A9000C251010AD8B4C5EF44F0030AD8B4CFEFED
:108AA00044F0010AD8B414EF45F045EF45F0120048
:108AB0000A0E1A6E0D0E1B6EC9EC4BF01AC0F2F4C2
:108AC0001BC0F3F40401000EF3BFFF0EF46FF56F4B
:108AD0000A0E1A6E0D0E1B6E000E1D6E2D0E1C6EF4
:108AE000EBEC6AF0010E1A240401F06F000E1B205B
:108AF000F16FEF0E00016E250401F66FFF0E00010D
:108B00006F210401F76FF2C4FAF2F3C4FBF2020121
:108B1000F96B01014A510201F92501014D6F4B51D9
:108B20000201FA2101014E6F4C510201FB210101AA
:108B30004F6F4DC11FF04EC120F04FC121F0F0C466
:108B400022F0F1C423F0F6C424F0D3EC58F0040171
:108B5000F6510201F96F0401F7510201FA6FFB6B44
:108B6000FC6BF95101013A5F0201FA5101013B5BD3
:108B70000201FB5101013C5B0201FC5101013D5B23
:108B80003A513B113C113D11D8A4C9EF45F0CBEF50
:108B900045F0E4EF45F000019B05D8A4D2EF45F085
:108BA000D4EF45F0D8EF45F0020E9B6FE4EF45F0AF
:108BB000080E01014F61DFEF45F0E1EF45F0E4EF12
:108BC00045F0456A7AEC2FF06CC021F06DC022F0C0
:108BD000010E0401F225236E000EF321246E040E13
:108BE000256ED1EC5AF021C06CF022C06DF012005D
:108BF0000A0E1A6E0D0E1B6EC9EC4BF01AC0FAF27B
:108C00001BC0FBF20A0E1A6E0D0E1B6E000E1D6EBF
:108C10002D0E1C6EEBEC6AF0010E1A240201FC6FA3
:108C2000000E1B20FD6F00016E51EF0F0201F96F66
:108C3000FE6B31EF46F0FCC2D9FFFDC2DAFF000E39
:108C400000019425E16EE26A030EE222DFCFE7FF26
:108C50000201FC4BFD2B0001942BE1EC68F00201BA
:108C6000FE2BF951FE5DD8A038EF46F03AEF46F002
:108C70001BEF46F0000E00019425D96EDA6A030E50
:108C8000DA220D0EDF6E942BE1EC68F0000E00018D
:108C90009425D96EDA6A030EDA220A0EDF6E942B5F
:108CA000E1EC68F001013A513B113C113D11D8A4AF
:108CB0005CEF46F05EEF46F083EF46F04DC11FF0EB
:108CC0004EC120F04FC121F0000E226E030E236E24
:108CD00094C024F0D3EC58F0000E01014D27010E92
:108CE0004E23000E4F2300019B05D8A47AEF46F0D7
:108CF0007CEF46F080EF46F0020E9B6F83EF46F06C
:108D0000456A7AEC2FF00201FA4BFB2B6CC021F084
:108D10006DC022F0FAC223F0FBC224F0040E256ECF
:108D2000D1EC5AF021C06CF022C06DF01200EB0EB5
:108D30000001E66F0B0EE76F4050D8B4A2EF46F08B
:108D4000A4EF46F033EF47F070517111D8A4ABEFA8
:108D500046F0ADEF46F033EF47F0E56B07EF47F035
:108D6000D80EE525D96EDA6A020EDA22E6C0E1FFF6
:108D7000E7C0E2FFDFCFE7FFE64BE72BE6C0D9FF16
:108D8000E7C0DAFF090EDF6EE64BE72BE6C021F005
:108D9000E7C022F0620EE525D96EDA6A020EDA2209
:108DA000DF50E26FE251236E246A030E256ED1EC90
:108DB0005AF021C0E6F022C0E7F0E6C0D9FFE7C0D4
:108DC000DAFF090EDF6E0001E64BE72BE6C021F06B
:108DD000E7C022F0000EE525D96EDA6A010EDA222C
:108DE000DF50E26FE251236E246A030E256ED1EC50
:108DF0005AF021C0E6F022C0E7F0E6C0D9FFE7C094
:108E0000DAFF090EDF6E0001E64BE72BE52BC751B9
:108E1000020DE551E26FE36BF350E25DE351800A2E
:108E2000E46FF450800AE459D8A019EF47F01BEF23
:108E300047F0B0EF46F0E6C0D9FFE7C0DAFF0D0E0D
:108E4000DF6EE64BE72BE6C0D9FFE7C0DAFF0A0E7C
:108E5000DF6EE64BE72BE6C0DDF0E7C0DEF040C09A
:108E6000DFF052EC5DF01200216EA388A3B83BEF57
:108E700047F03DEF47F036EF47F0000E376E000E3B
:108E8000366E000E396E100E386E49EF47F0E2EC88
:108E90004CF0375009E1030E365CD8A052EF47F092
:108EA00054EF47F063EF47F0020E3624D96E0D0EF3
:108EB0003720DA6E2150DE18D8B461EF47F063EF47
:108EC00047F06CEF47F038503910D8A46AEF47F0FC
:108ED0006CEF47F047EF47F038503910D8B473EFD4
:108EE00047F075EF47F0C5EF47F000019151D8A466
:108EF0007CEF47F07EEF47F09BEF47F0020E362401
:108F0000D96E0D0E3720DA6EDF6AB00E1A6E020EC1
:108F10001B6E0C0E1C6E0D0E1D6E3AEC65F0B00E45
:108F20001A6E020E1B6E290E1C6E2C0E1D6E3AEC74
:108F300065F0C1EF47F09105D8A4A1EF47F0A3EF8A
:108F400047F0B6EF47F0020E3624D96E0D0E3720EB
:108F5000DA6EDF6AB00E1A6E020E1B6E090E1C6E00
:108F60000D0E1D6E3AEC65F0C1EF47F0040E91193D
:108F7000D8A4BDEF47F0BFEF47F0C1EF47F0050EB3
:108F8000936F0001912BCAEF47F00201B06B060E00
:108F90000001936F12001AC0D9FF1BC0DAFFDF5027
:108FA000F00B1E6E1E3A0F0E1E160A0E1E60DBEF31
:108FB00047F0DDEF47F0E8EF47F01E50300F1CC0E0
:108FC000D9FF1DC0DAFFDF6E1C4A1D2AF1EF47F002
:108FD0001E50370F1CC0D9FF1DC0DAFFDF6EE4EF53
:108FE00047F01AC0D9FF1BC0DAFFDF500F0B1E6E0F
:108FF0001A4A1B2A0A0E1E6000EF48F002EF48F0E2
:109000000DEF48F01E50300F1CC0D9FF1DC0DAFF15
:10901000DF6E1C4A1D2A16EF48F01E50370F1CC089
:10902000D9FF1DC0DAFFDF6E09EF48F01AC0D9FF83
:109030001BC0DAFFDF50F00B1E6E1E3A0F0E1E161D
:109040000A0E1E6026EF48F028EF48F033EF48F094
:109050001E50300F1CC0D9FF1DC0DAFFDF6E1C4A46
:109060001D2A3CEF48F01E50370F1CC0D9FF1DC011
:10907000DAFFDF6E2FEF48F01AC0D9FF1BC0DAFF0E
:10908000DF500F0B1E6E1A4A1B2A0A0E1E604BEF92
:1090900048F04DEF48F058EF48F01E50300F1CC01C
:1090A000D9FF1DC0DAFFDF6E1C4A1D2A61EF48F0B0
:1090B0001E50370F1CC0D9FF1DC0DAFFDF6E54EF02
:1090C00048F012000001A951AC25256EFB51FC5D52
:1090D000D8B06DEF48F06FEF48F0ACEF48F0FC51BE
:1090E000FD5DD8B076EF48F078EF48F07CEF48F0BF
:1090F000FCC0ACF08BEF48F0FD51FB5DD8B083EFC6
:1091000048F085EF48F089EF48F0FBC0ACF08BEFFA
:1091100048F0FDC0ACF0AA51ACC020F0216A202676
:10912000000E2122FB51226E236A2050225C235024
:10913000800A246E2150800A2458D8B0A2EF48F04B
:10914000A4EF48F0A8EF48F0FBC0ACF0AEEF48F059
:10915000AA51AC27AEEF48F0FCC0ACF07B51D8B4BC
:10916000B4EF48F0B6EF48F0D8EF48F04150D8A43B
:10917000BCEF48F0BEEF48F0D8EF48F0D890793116
:109180008D19D8B4C6EF48F0C8EF48F0D8EF48F0D2
:1091900001019051D8B4CFEF48F0D1EF48F0D5EFAE
:1091A00048F08FC1ACF0D8EF48F08F510001AC27E8
:1091B0002550206E216A0001AC51A925226EE86A73
:1091C000D8B0E82AA9BFE806236E2050221809E18A
:1091D00021502318D8B4EFEF48F0F1EF48F0F7EF43
:1091E00048F0A951AC2574EC67F032EC6DF0120038
:1091F00020EE01F03E50D9263F50DA22DF501B6EA0
:109200001B5001010B5D000E0C59D8B00AEF49F05C
:109210000CEF49F00EEF49F00BC11BF01B500B5D3A
:109220000B6F0C51D8A00C050C6F1A6A27EF49F090
:10923000C40E1A24D96EDA6A010EDA2208C1E1FFDF
:1092400009C1E2FFDFCFE7FF084B092B1A2A1B50A9
:109250001A5CD8A02EEF49F030EF49F018EF49F032
:109260000B510C11D8B437EF49F039EF49F066EFE4
:1092700049F020EE01F03C50D9263D50DA22080E8C
:10928000DF6E20EE02F03C50D9263D50DA22C40EAB
:10929000DE6E010EDD6E3EC0D9FF3FC0DAFFDFBCDF
:1092A00054EF49F056EF49F05EEF49F03CC0D9FF6A
:1092B0003DC0DAFFC80EDF6E8AEF49F03CC0D9FF2F
:1092C0003DC0DAFF880EDF6E8AEF49F020EE01F034
:1092D0003C50D9263D50DA22080EDF6E20EE02F017
:1092E0003C50D9263D50DA22BF0EDE6E000EDD6EF8
:1092F0003CC0D9FF3DC0DAFF840EDF6E0A9F00013B
:10930000BA51D8A486EF49F088EF49F08AEF49F0C6
:1093100065EC58F012006598000162BF92EF49F0C9
:1093200094EF49F0CFEF49F001010AAF9AEF49F00D
:109330009CEF49F0AFEF49F0020E0001BC6F010154
:10934000BC51D8A4A6EF49F0A8EF49F0AAEF49F024
:1093500083EC61F00101BE6BBF6B1BEF4AF020EEA6
:1093600001F03C50D9263D50DA22080EDF6E20EE87
:1093700002F03C50D9263D50DA22BF0EDE6E000EC0
:10938000DD6E3CC0D9FF3DC0DAFF8C0EDF6E16C12A
:10939000D9FF17C1DAFF840EDF6E1BEF4AF0BFAFB3
:1093A000D4EF49F0D6EF49F0F3EF49F0010EBC6F6E
:1093B0000101BD51D8A4DFEF49F0E1EF49F0E3EF3F
:1093C00049F083EC61F00101BE6BBF6B0001BA5143
:1093D000D8A4EDEF49F0EFEF49F01BEF4AF065EC50
:1093E00058F01BEF4AF0020EBC6F20EE01F03C502B
:1093F000D9263D50DA22080EDF6E20EE02F03C50F6
:10940000D9263D50DA22BF0EDE6E000EDD6E3CC066
:10941000D9FF3DC0DAFF840EDF6E0101BE6BBF6B6A
:109420000001BA51D8A417EF4AF019EF4AF01BEF28
:109430004AF0EFEF49F01200070E1C6E070EADEC7C
:109440006CF00101896F1C2A1C50ADEC6CF001011D
:10945000886F1C2A1C50ADEC6CF00101876F1C2A30
:109460001C2A1C04ADEC6CF00101866F8651D8A457
:109470003CEF4AF03EEF4AF040EF4AF00001A56BA6
:109480001C2A1C04ADEC6CF00101856F8551D8A439
:109490004CEF4AF04EEF4AF050EF4AF00001A46B57
:1094A0001C2A1C04ADEC6CF00101846F8451D8A41B
:1094B0005CEF4AF05EEF4AF060EF4AF00001A36B08
:1094C0001C2A1C04ADEC6CF00101836F8351D8A4FD
:1094D0006CEF4AF06EEF4AF070EF4AF00001A26BB9
:1094E0001C2A1C04ADEC6CF00101826F8251D8A4DF
:1094F0007CEF4AF07EEF4AF080EF4AF00001A16B6A
:109500001C2A1C04ADEC6CF00101816F8151D8A4C0
:109510008CEF4AF08EEF4AF090EF4AF00001A06B1A
:109520001C2A1C04ADEC6CF00101806F8051D8A4A2
:109530009CEF4AF09EEF4AF09FEF4AF0416A000E1E
:10954000756F000E746F050E0001FA6F000E0101B9
:10955000E66F030EE56F1200080E1A6E00016451EB
:1095600007E1080E635DD8B0B8EF4AF0BAEF4AF0F1
:10957000D2EF4AF063C01AF0BD51D8A4C2EF4AF04E
:10958000C4EF4AF0C8EF4AF0010EBD6FD2EF4AF0C7
:10959000BD05D8A4CEEF4AF0D0EF4AF0D2EF4AF0A2
:1095A000020EBD6F1A50635D636F6451D8A06405ED
:1095B000646F010120EE01F01651D9261751DA220D
:1095C0001AC0DFFFC40E3A6E010E3B6E000162B19D
:1095D000ECEF4AF0EEEF4AF032EF4BF00CEF4BF0CD
:1095E00060C0F6FF61C0F7FF000EF86E3AC0D9FF09
:1095F0003BC0DAFF0F0EF76403D00800F55005D02A
:10960000F6CFE1FFF7CFE2FFE750DF6E0001604BDE
:10961000612B3A4A3B2A1A061A50D8A412EF4BF093
:1096200014EF4BF0F0EF4AF03AEF4BF060C0F6FF6A
:1096300061C0F7FF000EF86E3AC0D9FF3BC0DAFFF9
:109640000F0EF76403D00800F55005D0F6CFE1FF08
:10965000F7CFE2FFE750DF6E0001604B612B3A4A23
:109660003B2A1A061A50D8A438EF4BF03AEF4BF0C9
:1096700016EF4BF012000101B651D8A442EF4BF0A7
:1096800044EF4BF0C8EF4BF00001A605D8A44BEF18
:109690004BF04DEF4BF072EF4BF08DA652EF4BF0CD
:1096A00056EF4BF01A6A1A2A57EF4BF01A6A1A460D
:1096B0001A461A468D501A18F70B1A188D6E8DA679
:1096C00064EF4BF068EF4BF01A6A1A2A69EF4BF01F
:1096D0001A6A1A461A468D501A18FB0B1A188D6E04
:1096E000C5EF4BF0A005D8B478EF4BF07AEF4BF014
:1096F00092EF4BF0A505D8B480EF4BF082EF4BF022
:1097000092EF4BF0A405D8B488EF4BF08AEF4BF002
:1097100092EF4BF0A305D8A490EF4BF092EF4BF0F3
:10972000ABEF4BF08DA697EF4BF09BEF4BF01A6A27
:109730001A2A9CEF4BF01A6A1A461A461A468D509E
:109740001A18F70B1A188D6E8DA602D08D8401D0D1
:109750008D94C5EF4BF04104D8B4B1EF4BF0B3EFAB
:109760004BF0C3EF4BF0A205D8B4B9EF4BF0BBEF11
:109770004BF0C3EF4BF0A105D8A4C1EF4BF0C3EF02
:109780004BF0C5EF4BF08D868D84640E0101B66FF2
:109790001200000E216E000E206E1F6AD2EF4BF0F9
:1097A0001A4A1B2A1AC0D9FF1BC0DAFF200EDE1886
:1097B000D8B4DDEF4BF0DFEF4BF0D0EF4BF01AC039
:1097C000D9FF1BC0DAFFDF501C6EF70E1C26040EFB
:1097D0001C64EDEF4BF0EFEF4BF0D0EF4BF01AC005
:1097E000D9FF1BC0DAFF2D0EDE18D8A4FAEF4BF01C
:1097F000FCEF4BF002EF4CF0010E1F6E1A4A1B2AD1
:109800002CEF4CF01AC0D9FF1BC0DAFF2B0EDE186C
:10981000D8A40DEF4CF00FEF4CF02CEF4CF0FEEF16
:109820004BF00A0E2002F3CF1CF0F4CF1DF0210202
:10983000F3501D261AC0D9FF1BC0DAFFDF501E6E81
:109840001E501C5E000E1D5A300E1C24206E000E91
:109850001D20216EFEEF4BF01AC0D9FF1BC0DAFFAE
:10986000DF501C6ED00E1C26090E1C643AEF4CF023
:109870003CEF4CF011EF4CF01F50D8A442EF4CF0ED
:1098800044EF4CF052EF4CF020C01CF021C01DF012
:109890001C1E1D1E1C4A1D2A1CC01AF01DC01BF0D8
:1098A00056EF4CF020C01AF021C01BF0120000014E
:1098B000DC6B4450D8B45FEF4CF061EF4CF0E1EF5B
:1098C0004CF07B51D8B467EF4CF069EF4CF0E1EF0E
:1098D0004CF0DD6B7DEF4CF0000EDD25D96EDA6AC1
:1098E000010EDA22030EDF6478EF4CF07AEF4CF0D1
:1098F0007CEF4CF0010EDC6FDD2BC751020DDD510A
:10990000D96FDA6BF350D95DDA51800ADB6FF4500E
:10991000800ADB59D8A08FEF4CF091EF4CF06CEF40
:109920004CF0DC51D8A497EF4CF099EF4CF0AAEF33
:109930004CF08C51D8A49FEF4CF0A1EF4CF0AAEF63
:109940004CF001018051D8B4A8EF4CF0AAEF4CF0D4
:10995000E1EF4CF04150D8A4B0EF4CF0B2EF4CF036
:10996000E1EF4CF0010E416E8B0E0001D16F290E1C
:10997000D26F000ED36F640ED46FEBEC30F0F20EAA
:109980000001D16F2A0ED26F000ED36F000ED46F7C
:10999000EBEC30F000017805D8A4D1EF4CF0D3EF18
:1099A0004CF0D7EF4CF0040E426EE1EF4CF0260E77
:1099B000D16F2B0ED26F000ED36F000ED46FEBEC75
:1099C00030F012000101B851D8A4E9EF4CF0EBEFF0
:1099D0004CF06AEF4DF0B751D8B4F1EF4CF0F3EF23
:1099E0004CF06AEF4DF076517711D8A4FAEF4CF0B5
:1099F000FCEF4CF01DEF4DF00A0E0001B66F8988A8
:109A000081EC6CF00101F65132EC6DF0840E1A6EAF
:109A1000240E1B6E2C0E1C6E15EC68F00009D8B4D9
:109A200014EF4DF016EF4DF06AEF4DF0000E01010E
:109A3000776F2C0E766F6AEF4DF00001B651D8B4F7
:109A400024EF4DF026EF4DF05FEF4DF08C0E01014D
:109A5000765D030E7759D8B030EF4DF032EF4DF010
:109A60004BEF4DF0840E76251A6E240E77211B6E77
:109A7000200E1C6E15EC68F00009D8B442EF4DF0D2
:109A800044EF4DF06AEF4DF0200E01017627000EF5
:109A900077236AEF4DF0840E76251A6E240E772117
:109AA0001B6E120E1C6E15EC68F00009D8B45BEF4B
:109AB0004DF05DEF4DF06AEF4DF016EF4DF08998E7
:109AC0000A0E0101B86FB707000E776F000E766FB0
:109AD0006AEF4DF01200800E286E090E296E285094
:109AE000345C29503558D8A078EF4DF07AEF4DF01E
:109AF000C3EF4DF0000E1A6E030E1B6E800E1C6E2F
:109B0000080E1D6E010E1F6E000E1E6E06EC67F035
:109B100065C01FF066C020F067C021F0000E226E05
:109B2000030E236E000E246ED3EC58F0800E1A6ED6
:109B3000080E1B6E800E1C6E090E1D6EF4EC69F093
:109B4000800E1A6E080E1B6E000E1D6E000E1C6E2F
:109B5000EBEC6AF01AC034F01BC035F0000E0001C7
:109B60006527010E6623000E6723700E6765BBEF45
:109B70004DF0BDEF4DF0C3EF4DF0000E656F000EE0
:109B8000666F700E676F3550080802E13450800828
:109B9000D8B0CDEF4DF0CFEF4DF0F0EF4DF0000E1F
:109BA0001A6E030E1B6E800E1C6E080E1D6E800E4C
:109BB000345C1E6E080E35581F6E06EC67F065C0EB
:109BC0001FF066C020F067C021F0000E226E030E69
:109BD000236E800E286E2850345C246ED3EC58F02F
:109BE0009FEC60F012000001E735E835296E29503E
:109BF000D8A4FDEF4DF0FFEF4DF009EF4EF0000E51
:109C0000E56F000EE66F000EE76F000EE86F76EF6F
:109C10004EF0E5C0E9F0E6C0EAF0E7C0EBF0E8C0DE
:109C2000ECF0200E19EF4EF0D890EC33EB33EA3322
:109C3000E933E82E14EF4EF0E951286EE78FFF0E5E
:109C4000E517FF0EE617FF0EE717000EE817960E52
:109C5000295E29BE30EF4EF02EEF4EF046EF4EF06B
:109C60002950800A970FD8B038EF4EF03AEF4EF0F7
:109C70003CEF4EF0FFEF4DF0D890E833E733E6339A
:109C8000E533293E3CEF4EF05EEF4EF01F0E2964A7
:109C90004CEF4EF04EEF4EF056EF4EF0FFEF4DF022
:109CA000D890E537E637E737E83729062950D8A4B2
:109CB0005CEF4EF05EEF4EF050EF4EF02850D8B40F
:109CC00064EF4EF066EF4EF06EEF4EF0E81FE71FC8
:109CD000E61FE56D000EE623E723E823E5C0E5F087
:109CE000E6C0E6F0E7C0E7F0E8C0E8F012000001E7
:109CF000D46BD0C021F0D1C022F0000E8E25D96ED9
:109D0000DA6A060EDA22DF50D36FD351236E246A4B
:109D1000030E256ED1EC5AF021C0D0F022C0D1F054
:109D2000D0C0D9FFD1C0DAFF090EDF6E0001D04BE1
:109D3000D12B8E51040D800EF324D96E060EF42023
:109D4000DA6EDECFD5F0DECFD6F0DECFD7F0DECFC5
:109D5000D8F08E2BD0C01AF0D1C01BF0D851A2EC95
:109D600062F01AC0D0F01BC0D1F0D0C01AF0D1C040
:109D70001BF00001D751A2EC62F01AC0D0F01BC05A
:109D8000D1F0D0C01AF0D1C01BF00001D651A2EC26
:109D900062F01AC0D0F01BC0D1F0D0C01AF0D1C010
:109DA0001BF00001D551A2EC62F01AC0D0F01BC02C
:109DB000D1F0D0C0D9FFD1C0DAFF0D0EDF6E0001A7
:109DC000D04BD12BD0C0D9FFD1C0DAFF0A0EDF6E45
:109DD000D04BD12B8E9FD42B0F0ED465F2EF4EF0CB
:109DE000F4EF4EF079EF4EF00101A407D0C0D0F0AF
:109DF000D1C0D1F012009C0EF66EDA0EF76E000E96
:109E0000F86E02EED8F010EE1AF00900F5CFEEFF72
:109E1000E550E150FAE1A60EF66ED90EF76E000E8F
:109E2000F86E01EEDDF010EE22F00900F5CFEEFF46
:109E3000E550E150FAE11C0EF66EDB0EF76E000EF7
:109E4000F86E00EEF7F010EE09F00900F5CFEEFF26
:109E5000E550E150FAE106EE80F014EE00F0EE6A13
:109E6000E550E150FCE1E250FAE10AEE80F013EE39
:109E70009BF0EE6AE550E150FCE1E250FAE106EEBB
:109E800000F0800EEE6AE806FDE105EE00F011EE4E
:109E900000F0EE6AE550E150FCE1E250FAE103EE39
:109EA00000F011EE00F0EE6AE550E150FCE1E25006
:109EB000FAE102EE00F0D80EEE6AE806FDE101EEEE
:109EC00000F0DD0EEE6AE806FDE104EE30F0C00EB3
:109ED000EE6AE806FDE100EE60F06C0EEE6AE80660
:109EE000FDE100EE2BF01B0EEE6AE806FDE1469068
:109EF000469200018CEF3FF0020E0001D56F030E79
:109F0000D66FD46BCF6BD451040D2C0EF324276E77
:109F1000020EF420286ECF512724D96E000E28207F
:109F2000DA6ED5C0E1FFD6C0E2FFDFCFE7FFD54B49
:109F3000D62BCF2B030ECF65A0EF4FF0A2EF4FF043
:109F400083EF4FF0D42B0A0ED465A9EF4FF0ABEF9F
:109F50004FF082EF4FF0D46BD451040D000EF32478
:109F6000D96E020EF420DA6EDECFD0F0DECFD1F063
:109F7000DECFD2F0DECFD3F0D5C0D9FFD6C0DAFF26
:109F8000D3C0DFFFD54BD62BD5C0D9FFD6C0DAFF63
:109F9000D2C0DFFFD54BD62BD5C0D9FFD6C0DAFF54
:109FA000D1C0DFFFD54BD62BD5C0D9FFD6C0DAFF45
:109FB000D0C0DFFFD54BD62BD42B0A0ED465E3EFF0
:109FC0004FF0E5EF4FF0ACEF4FF0000ECC6FF00E1E
:109FD000CD6F070ECE6FCCC01FF0CDC020F0CEC02D
:109FE00021F0000E226E030E236E000E276E275006
:109FF000D55D246ED3EC58F01200A098636A626AB3
:10A000000F014C6B160E5F6F9F0E5D6F7B0E5C6FCA
:10A010001A6A1A50040D000EF324D96E040EF420AF
:10A02000DA6EDE6ADE6ADE6ADD6A1A2A0B0E1A64EE
:10A030001CEF50F01EEF50F009EF50F0658C0F014F
:10A040005E6B6598659C2EEF50F062960001626B26
:10A0500001010A6B000E0C6F000E0B6F62B633EF3E
:10A0600050F035EF50F025EF50F0010E0101BF6FB9
:10A07000010EBE6FBD6BBC6BC26B1A6A1A50020D2B
:10A08000160EF324D96E010EF420DA6EDE6ADD6A54
:10A090001A50020D1C0EF324D96E010EF420DA6E54
:10A0A000DE6ADD6A530E1A24D96EDA6A010EDA22EC
:10A0B000DF6A500E1A24D96EDA6A010EDA22DF6ADC
:10A0C0001A2A020E1A6467EF50F069EF50F03EEF63
:10A0D00050F0080E0101166F040E176F160E0F01D7
:10A0E0004C6F000E0401036FBF0E026F080E016F6C
:10A0F000840E006F0001CB6BBE6B12000001BF39F4
:10A10000E832030B0009D8B488EF50F08AEF50F022
:10A11000CDEF50F0FCEF50F0628F080EBE6FFCEFF9
:10A1200050F0B7EC44F0FCEF50F031EC5BF0FCEF9A
:10A1300050F0CB0E606F616B6281010E636F628FB6
:10A14000FCEF50F0DEEC53F0FCEF50F05EEC2CF046
:10A15000FCEF50F0DB0EC325606F616B010E6123D5
:10A160009CEF50F0628FDB0EC325D96EDA6A010EC8
:10A17000DA22C1C0DFFFFCEF50F0000ECD6F020EFF
:10A18000CC6F000ECE6F000ECF6F000ED16F000EA1
:10A19000D06FAAEC5DF0FCEF50F0C051000AD8B4CB
:10A1A000A2EF50F0010AD8B4A6EF50F0020AD8B4DA
:10A1B000A6EF50F0060AD8B48CEF50F0030AD8B4DA
:10A1C00091EF50F0010AD8B4BDEF50F00F0AD8B4A7
:10A1D00099EF50F0010AD8B495EF50F0030AD8B4C3
:10A1E000AAEF50F0010AD8B4B2EF50F0070AD8B481
:10A1F000FCEF50F0FCEF50F01200296A43EF51F0F1
:10A2000023C0D9FF24C0DAFF2550210D800EF3248E
:10A21000266E0A0EF420276E29502624E16E000EC9
:10A220002720E26EDFCFE7FF234A242A2550210DA5
:10A23000800EF324266E0A0EF420276E2950262461
:10A24000D96E000E2720DA6E5C0EDE18D8A42BEF34
:10A2500051F02DEF51F030EF51F0296A39EF51F004
:10A26000200E296036EF51F038EF51F039EF51F000
:10A27000292A23C020F024C021F0C4EC6AF020C0B9
:10A2800023F021C024F023C0D9FF24C0DAFF2E0E12
:10A29000DE18D8B44EEF51F050EF51F06EEF51F0A0
:10A2A00023C0D9FF24C0DAFF200EDF605AEF51F03F
:10A2B0005CEF51F000EF51F06EEF51F02550210DA1
:10A2C000800EF324266E0A0EF420276E29502624D1
:10A2D000D96E000E2720DA6EDF6A292A1F0E296444
:10A2E00074EF51F076EF51F05EEF51F023C023F0A0
:10A2F00024C024F01200000E0001CC6FF00ECD6FD0
:10A30000070ECE6FCCC01AF0CDC01BF0CEC01CF033
:10A31000000E1D6E030E1E6EE9EC62F0020E0001CF
:10A32000D46F030ED56FD66BCF6BD4C0D9FFD5C019
:10A33000DAFFD651040D2C0EF324206E020EF42009
:10A34000216ECF512024E16E000E2120E26EDFCF7E
:10A35000E7FFD44BD52BCF2B030ECF65B2EF51F0D7
:10A36000B4EF51F095EF51F0D62B0A0ED665BBEF46
:10A3700051F0BDEF51F094EF51F0D66BD4C0D9FF3E
:10A38000D5C0DAFFDF50D36FD44BD52BD4C0D9FF63
:10A39000D5C0DAFFDF50D26FD44BD52BD4C0D9FF54
:10A3A000D5C0DAFFDF50D16FD44BD52BD4C0D9FF45
:10A3B000D5C0DAFFDF50D06FD44BD52BD651040D6A
:10A3C000000EF324D96E020EF420DA6ED0C0DEFF48
:10A3D000D1C0DEFFD2C0DEFFD3C0DEFFD62B0A0E17
:10A3E000D665F5EF51F0F7EF51F0BEEF51F01200E6
:10A3F00025C0D1F0000E0001CD6F000ECE6F000E13
:10A40000CF6F000ED06F4DEF52F023C0D9FF24C0A4
:10A41000DAFFDF50CC6F234A242ACCC027F00F0E7E
:10A4200027162750CD27000ECE23CF23D023400E52
:10A43000CC651DEF52F01FEF52F025EF52F0090EE0
:10A44000CD27000ECE23CF23D023D107D151D8B4AE
:10A450002CEF52F02EEF52F037EF52F0040ED8905E
:10A46000CD37CE37CF37D037E82E2FEF52F0260436
:10A47000D8A43DEF52F03FEF52F04DEF52F023C021
:10A4800020F024C021F0C4EC6AF020C023F021C0E9
:10A4900024F023C032F024C033F00001D151D8A4FD
:10A4A00054EF52F056EF52F005EF52F062EF52F0D7
:10A4B000040ED890CD37CE37CF37D037E82E59EFAE
:10A4C00052F0252A070E256468EF52F06AEF52F029
:10A4D00058EF52F0CDC023F0CEC024F0CFC025F00D
:10A4E000D0C026F012000001DC6B80EF52F0CCC02F
:10A4F000D9FFCDC0DAFF300EDF6ECC4BCD2BDC2B7D
:10A50000FF0ED225D36FD46BFF0ED423DC51D56F51
:10A51000D66BD351D55DD651800AD76FD451800AFE
:10A52000D759D8A096EF52F098EF52F077EF52F04B
:10A53000010ECC25D86F000ECD21D96FCEC01AF0F8
:10A54000CFC01BF0D0C01CF0D1C01DF00A0E1E6E93
:10A55000000E1F6E000E206E000E216E74EC63F074
:10A560001AC0DAF01BC0DBF0CEC01AF0CFC01BF06F
:10A57000D0C01CF0D1C01DF00A0E1E6E000E1F6E62
:10A58000000E206E000E216EACEC5FF01AC0CEF013
:10A590001BC0CFF01CC0D0F01DC0D1F0300E0001A8
:10A5A000DA27000EDB23CCC0D9FFCDC0DAFFDAC03A
:10A5B000DFFFCC07D8A0CD07CE51CF11D011D111DC
:10A5C000D8A4E5EF52F0E7EF52F09EEF52F0D8C07A
:10A5D000CCF0D9C0CDF012000101AB51D8A4F3EFFB
:10A5E00052F0F5EF52F0FBEF52F0B3C043F0ECEC59
:10A5F00060F064EF53F043500001B319D8A403EFA7
:10A6000053F005EF53F05FEF53F0C951D8A40BEFAF
:10A6100053F00DEF53F064EF53F0735107E1840EE4
:10A62000725DD8B016EF53F018EF53F01AEF53F0F5
:10A6300089988E9472057311D8A421EF53F023EFFB
:10A6400053F02CEF53F0A86BA851D8B42AEF53F075
:10A650002CEF53F024EF53F072517311D8A433EF61
:10A6600053F035EF53F064EF53F09051D8B43BEF13
:10A6700053F03DEF53F041EF53F03DEC59F064EFF0
:10A6800053F076517711D8A448EF53F04AEF53F0C6
:10A6900053EF53F074517511D8B451EF53F053EF99
:10A6A00053F05BEF53F0A851D8A459EF53F05BEF90
:10A6B00053F053EF53F02BEC41F03DEF53F08998FA
:10A6C000B3C043F0FEEC5FF012000101AB51D8A41F
:10A6D0006CEF53F06EEF53F074EF53F0B3C043F0F0
:10A6E00069EC43F0DDEF53F043500001B319D8A4F7
:10A6F0007CEF53F07EEF53F0D8EF53F0C951D8A45C
:10A7000084EF53F086EF53F0DDEF53F0735107E120
:10A71000840E725DD8B08FEF53F091EF53F093EF4A
:10A7200053F089988E9472057311D8A49AEF53F060
:10A730009CEF53F0A5EF53F0A86BA851D8B4A3EF4A
:10A7400053F0A5EF53F09DEF53F072517311D8A45D
:10A75000ACEF53F0AEEF53F0DDEF53F09051D8B4BF
:10A76000B4EF53F0B6EF53F0BAEF53F05EEC3AF0BB
:10A77000DDEF53F076517711D8A4C1EF53F0C3EF5A
:10A7800053F0CCEF53F074517511D8B4CAEF53F0B5
:10A79000CCEF53F0D4EF53F0A851D8A4D2EF53F03C
:10A7A000D4EF53F0CCEF53F02BEC41F0B6EF53F075
:10A7B0008998B3C043F0B3EC42F012000101C46BBE
:10A7C000C56B36EF54F0628F0101C305D8A4EBEFDF
:10A7D00053F0EDEF53F047EF54F0C48347EF54F0DC
:10A7E000628F47EF54F0628FC3BFF9EF53F0FBEF76
:10A7F00053F00CEF54F0C3510F0B1A6E1A50020DA8
:10A800001C0EF324D96E010EF420DA6EDECF1BF09D
:10A81000DDCF1CF01BEF54F0C3510F0B1A6E1A5012
:10A82000020D160EF324D96E010EF420DA6EDECF7F
:10A830001BF0DDCF1CF01BC0D9FF1CC0DAFFDFAE60
:10A8400024EF54F026EF54F047EF54F01BC0D9FF2B
:10A850001CC0DAFFDFA42FEF54F031EF54F047EFC4
:10A8600054F0010E0101C46F47EF54F00001BF51D5
:10A870001F0B000AD8B4E3EF53F0010AD8B4F0EF8D
:10A8800053F0030AD8B4F3EF53F047EF54F000014C
:10A8900062AF4DEF54F04FEF54F056EF54F0C40E4A
:10A8A000606F010E616F6281020E636F1200000122
:10A8B000BF511F0BE806D8B460EF54F062EF54F0BC
:10A8C00064EF54F0CFEF54F0BF39E832030BE806E1
:10A8D000D8B46DEF54F06FEF54F071EF54F0CFEF48
:10A8E00054F0C351D8B477EF54F079EF54F0B8EF87
:10A8F00054F0C305D8B47FEF54F081EF54F0B8EFB3
:10A9000054F0CFEF54F0D00E606F020E616F000E66
:10A91000646F080E636F6281628FCFEF54F0D00EC8
:10A92000606F020E616F8CEF54F0C5C00BF1C6C0B2
:10A930000CF1CC0E0101086F010E096F000E0D6FB6
:10A94000000E0E6F000E0F6F0A8FCFEF54F0CC0E7B
:10A95000606F010E616F000E646F070E636FC10EB2
:10A96000626FCFEF54F0C1C0BAF1628FCFEF54F0F5
:10A97000C051000AD8B483EF54F0010AD8B48FEF65
:10A9800054F0210AD8B495EF54F0010AD8B4A7EFD7
:10A9900054F0030AD8B4B3EF54F0CFEF54F01200E0
:10A9A0002D0E0101C06FCAC0D9F0FD0E0001D917EC
:10A9B000D8A4DDEF54F0DFEF54F03BEF55F0CAC000
:10A9C000D9F0D890D9333F0ED917D951040D000EC4
:10A9D000F3243E6E040EF4203F6E3EC03CF03FC0B8
:10A9E0003DF0040E3C1A3EC0D9FF3FC0DAFFDF3015
:10A9F000E8320F0B0D0AD8A400EF55F002EF55F026
:10AA000037EF55F0DB6B20EE02F03E50D9263F5079
:10AA1000DA22DECFD9F0DDCFDAF0D9C0D9FFDAC043
:10AA2000DAFFDB51BF0FE16EE26ADFCFE7FF20EE16
:10AA300002F03E50D9263F50DA22DE2A000EDD22F7
:10AA4000DB2B070EDB6527EF55F029EF55F003EF01
:10AA500055F020EE02F03E50D9263F50DA22BF0ECC
:10AA6000DE6E000EDD6E7DEC64F047EF55F04AECD3
:10AA700068F047EF55F0CA51FD0B040AD8A443EF24
:10AA800055F045EF55F047EF55F02EEC56F012001B
:10AA90000A0E0101B96F0001916BEB0E1A6E0B0EDD
:10AAA0001B6EFD0E1C6E2B0E1D6EF4EC69F00D0E70
:10AAB00034EC47F0EB0E1A6E0B0E1B6EF50E1C6E8F
:10AAC0002B0E1D6EF4EC69F00D0E34EC47F0EB0E1E
:10AAD0001A6E0B0E1B6EC60E1C6E2B0E1D6EF4EC4A
:10AAE00069F03A0E34EC47F0EB0E1A6E0B0E1B6E4B
:10AAF000EC0E1C6E2B0E1D6EF4EC69F03A0E34EC6D
:10AB000047F0EB0E1A6E0B0E1B6E260E1C6E2C0EF3
:10AB10001D6EF4EC69F0EB0E1A6E0B0E1B6EF70E49
:10AB20001C6E010E1D6E000E1F6E080E1E6ECDEC0B
:10AB300061F0EB0E1A6E0B0E1B6EE00E1C6E020E19
:10AB40001D6E3AEC65F0EB0E1A6E0B0E1B6E2B0EA3
:10AB50001C6E2C0E1D6E3AEC65F04B0E34EC47F07B
:10AB6000330EAB6E7D6A630E0001926F000E376E7E
:10AB7000000E366E1200000E206EE00E216E070EE3
:10AB8000226E20C01AF021C01BF022C01CF0000E63
:10AB90001D6E030E1E6EE9EC62F0000E236E030EB6
:10ABA000246E23C0D9FF24C0DAFFDF500101716F8A
:10ABB000234A242A23C0D9FF24C0DAFFDF50706F54
:10ABC000234A242A702906E17129D8A4EAEF55F016
:10ABD000ECEF55F0F0EF55F0000E716F000E706F56
:10ABE00070C172F171C173F123C0D9FF24C0DAFFC3
:10ABF000DF500001676F234A242A23C0D9FF24C0F5
:10AC0000DAFFDF50666F234A242A23C0D9FF24C00D
:10AC1000DAFFDF50656F234A242A710E676113EF54
:10AC200056F015EF56F01DEF56F0700E67611BEFF2
:10AC300056F01DEF56F025EF56F0000E656F000E32
:10AC4000666F700E676F020E986F23C0D9FF24C025
:10AC5000DAFFDF509F6F234A242A120016C1D9FF62
:10AC600017C1DAFF0101000EDFBC010E1B6E040EDE
:10AC7000161B080E0001BE19D8A441EF56F043EF91
:10AC800056F056EF56F0C1C05EFF0F015E51D8B4CA
:10AC90004CEF56F04EEF56F053EF56F0100E000109
:10ACA000BE6F56EF56F0040E0001BE6FBC05D8A46F
:10ACB0005CEF56F05EEF56F095EF56F0010120EE96
:10ACC00002F01651D9261751DA22C40EDE6E010E9B
:10ACD000DD6EACEC4AF0020E0001BD19D8A473EF92
:10ACE00056F075EF56F07DEF56F016C1D9FF17C13B
:10ACF000DAFF840EDF6EA0EF56F01B50D8A483EF6E
:10AD000056F085EF56F08DEF56F016C1D9FF17C1FA
:10AD1000DAFFC80EDF6EA0EF56F016C1D9FF17C1DB
:10AD2000DAFF880EDF6EA0EF56F001010AAF9BEF4D
:10AD300056F09DEF56F09EEF56F00A9F0001BC6B57
:10AD400012001E6E1A50D8B4A8EF56F0AAEF56F0B3
:10AD5000B8EF56F01E50020D160EF324D96E010EF8
:10AD6000F420DA6EDECF1FF0DDCF20F0C4EF56F016
:10AD70001E50020D1C0EF324D96E010EF420DA6E63
:10AD8000DECF1FF0DDCF20F01F502010D8A4CBEF76
:10AD900056F0CDEF56F0D3EF56F0000E1A6E000EBF
:10ADA0001B6E13EF57F020EE02F01F50D9262050F3
:10ADB000DA221BC0DEFF1CC0DDFF20EE01F01F50B9
:10ADC000D9262050DA221DC0DFFF1FC0D9FF20C0C6
:10ADD000DAFF400EDF161FC0D9FF20C0DAFF880E51
:10ADE000DF121A50D8B4F7EF56F0F9EF56F005EF2E
:10ADF00057F01E50020D160EF324D96E010EF420EA
:10AE0000DA6E040EDF1A0FEF57F01E50020D1C0E03
:10AE1000F324D96E010EF420DA6E040EDF1A1FC07F
:10AE20001AF020C01BF012000001B96B01017A5129
:10AE30007B11D8B41EEF57F020EF57F033EF57F0E7
:10AE40007AC1D9FF7BC1DAFFDFBE29EF57F02DEFC2
:10AE500057F0246A242A2EEF57F0246A2450256ED6
:10AE6000266A37EF57F0000E266E000E256E25502D
:10AE70002610D8A43EEF57F040EF57F083EF57F07D
:10AE8000010120EE01F07A51D9267B51DA222350BC
:10AE9000DE5CD8B04EEF57F050EF57F058EF57F058
:10AEA00020EE01F07A51D9267B51DA22DF50236E51
:10AEB0000001B96B6BEF57F0700EB925D96EDA6AE5
:10AEC000020EDA22B9512124E16E000E2220E26E38
:10AED000DFCFE7FFB92B2350B95DD8A072EF57F051
:10AEE00074EF57F05CEF57F0000E1A6E700E1B6E89
:10AEF000020E1C6E400E1D6E020EA1EC56F01AC022
:10AF00007AF11BC07BF10001B95112004550D8A461
:10AF10008CEF57F08EEF57F0A7EF57F0D0B693EFC6
:10AF200057F095EF57F0A3EF57F000019F2B860ED7
:10AF3000D16F2B0ED26F000ED36F000ED46FEBECDF
:10AF400030F0F6EF57F000019F6BF6EF57F04450EA
:10AF5000D8A4ADEF57F0AFEF57F0EAEF57F001018B
:10AF6000EB05D8A4B6EF57F0B8EF57F0F6EF57F06F
:10AF7000925100019F5DD8B0C0EF57F0C2EF57F07B
:10AF8000CBEF57F001018105D8A4C9EF57F0CBEF03
:10AF900057F0F6EF57F00001A051D8A4D2EF57F0C8
:10AFA000D4EF57F0DEEF57F0AD0ED16F290ED26F10
:10AFB000000ED36F000ED46FEBEC30F0010E0001E9
:10AFC000A06F040E426E000E0101756F000E746FCB
:10AFD000F6EF57F000019F51D8B4F1EF57F0F3EFBF
:10AFE00057F0F6EF57F09F079FEC60F01200EB0E62
:10AFF0000001E56F0B0EE66F0101B151D8B403EF0C
:10B0000058F005EF58F064EF58F0E5C021F0E6C0C5
:10B0100022F0E2C023F0E3C024F0040E256ED1EC50
:10B020005AF021C0E5F022C0E6F0E5C0D9FFE6C045
:10B03000DAFF090EDF6E0001E54BE62BF00E216E04
:10B040000B0E226EABC023F0246A020E256ED1ECEB
:10B050005AF021C0E5F022C0E6F0E5C0D9FFE6C015
:10B06000DAFF090EDF6E0001E54BE62BF30E216ED1
:10B070000B0E226EA951AC2574EC67F00001E46F51
:10B08000E451236E246A020E256ED1EC5AF021C0E1
:10B09000E5F022C0E6F0E5C0D9FFE6C0DAFF0D0E0C
:10B0A000DF6E0001E54BE62BE5C0D9FFE6C0DAFF15
:10B0B0000A0EDF6EE54BE62BE5C0DDF0E6C0DEF004
:10B0C000B1C1DFF052EC5DF012000101BF51D8A414
:10B0D0006CEF58F06EEF58F0D2EF58F0010EBF6FE2
:10B0E000BE51D8A476EF58F078EF58F0D2EF58F070
:10B0F000010EBE6F020E0001BC19D8A482EF58F0F9
:10B1000084EF58F094EF58F0010120EE01F0165151
:10B11000D9261751DA22DF6A16C1D9FF17C1DAFF23
:10B12000C80EDF6ED2EF58F0BC05D8A49AEF58F0E5
:10B130009CEF58F0D2EF58F00101C16B20EE01F006
:10B140003E50D9263F50DA22080EDF6E20EE02F084
:10B150003E50D9263F50DA22BF0EDE6E000EDD6E65
:10B160003EC0D9FF3FC0DAFF840EDF6E010EC16F13
:10B1700020EE01F03C50D9263D50DA22080EDF6E59
:10B1800020EE02F03C50D9263D50DA22BF0EDE6E92
:10B19000000EDD6E3CC0D9FF3DC0DAFF800EDF6ED1
:10B1A000D2EF58F0120024C026F020C025F00F0E78
:10B1B0002516D8A4DEEF58F0E0EF58F0E8EF58F08D
:10B1C0001FC01BF020C01CF021C01DF03DEC64F03E
:10B1D000060E40EC6DF08B90020EC96E9EA6F3EF4A
:10B1E00058F0F5EF58F0EEEF58F09E9621C0C9FFE9
:10B1F0009EA6FDEF58F0FFEF58F0F8EF58F09E963E
:10B2000020C0C9FF9EA607EF59F009EF59F002EFE1
:10B2100059F09E961FC0C9FF9EA611EF59F013EF7B
:10B2200059F00CEF59F09E9622C0D9FF23C0DAFFE7
:10B23000DF50C96E224A232A26069EA622EF59F025
:10B2400024EF59F01DEF59F09E962650D8A42BEF0D
:10B2500059F02DEF59F014EF59F08B80F00E00D01B
:10B26000E82EFDD739EC6CF00009D8A43AEF59F07C
:10B270003CEF59F02EEF59F01200560E4318D8A4A7
:10B2800044EF59F046EF59F064EF59F00001765160
:10B290007711D8A44EEF59F050EF59F059EF59F00B
:10B2A00074517511D8B457EF59F059EF59F060EF58
:10B2B00059F0060EC96F7607D8A07707A5EF59F0A9
:10B2C000CEEC66F0A5EF59F0520E4318D8A46BEF00
:10B2D00059F06DEF59F0A5EF59F000017651771153
:10B2E000D8A475EF59F077EF59F080EF59F0745109
:10B2F0007511D8B47EEF59F080EF59F084EF59F012
:10B30000070EC96F5BEF59F09605D8A48AEF59F084
:10B310008CEF59F05BEF59F05AC11AF05BC11BF08A
:10B3200056C11CF057C11DF099C11EF097C11FF006
:10B3300094C120F093C121F07CC022F0070E50ECA4
:10B3400060F00001966B5BEF59F012000101B72B22
:10B35000010EF56F010EF06F000E0001F86F1E0E6A
:10B36000F76F456AA605D8A4B8EF59F0BAEF59F0BF
:10B37000C3EF59F0040E426E000E0101756F000E0E
:10B38000746FC5EF59F0426A8B820001876B01012F
:10B390009C6B8E94000E676F000E666F000199051E
:10B3A000D8A4D5EF59F0D7EF59F0D9EF59F0020EE4
:10B3B000996F9A05D8A4DFEF59F0E1EF59F0E3EF68
:10B3C00059F0020E9A6F9805D8A4E9EF59F0EBEF07
:10B3D00059F0EDEF59F0020E986F9B05D8A4F3EFEA
:10B3E00059F0F5EF59F0F6EF59F09B6B020E9B19EF
:10B3F000D8A4FDEF59F0FFEF59F001EF5AF0030E1A
:10B400009B6F0101B16B0001A76B406A0101A76B43
:10B41000A66BA38AA190A0801200800E346E080E45
:10B42000356E65C01AF066C01BF067C01CF0000ED8
:10B430001D6E030E1E6EE9EC62F0090E030100653D
:10B4400024EF5AF026EF5AF069EF5AF00029D8B4E9
:10B450002CEF5AF02EEF5AF069EF5AF0800E1A6E68
:10B46000080E1B6E000E1C6E030E1D6E010E1F6E6D
:10B47000000E1E6E06EC67F0800E1A6E080E1B6E34
:10B48000000E1D6E1C68EBEC6AF01AC034F01BC095
:10B4900035F034503510D8B450EF5AF052EF5AF01E
:10B4A00065EF5AF0800E256E080E266EFF0E2526DB
:10B4B000000E26222550345C26503558D8A063EF64
:10B4C0005AF065EF5AF069EF5AF0800E346E080EAC
:10B4D000356E34C0D9FF35C0DAFFDF6A12001A6E4C
:10B4E000290E1B6EA0EF5AF0C40E1B6ECFEF5AF060
:10B4F000A00E1B6ECFEF5AF07C0E1B6ECFEF5AF0F2
:10B500005F0E1B6ECFEF5AF04E0E1B6ECFEF5AF050
:10B51000440E1B6ECFEF5AF03C0E1B6ECFEF5AF06D
:10B52000360E1B6ECFEF5AF0300E1B6ECFEF5AF077
:10B530002D0E1B6ECFEF5AF0290E1B6ECFEF5AF077
:10B540001A500A0AD8B474EF5AF0050AD8B478EF42
:10B550005AF01B0AD8B47CEF5AF00D0AD8B480EF29
:10B560005AF0070AD8B484EF5AF03D0AD8B488EFED
:10B570005AF00B0AD8B48CEF5AF0050AD8B490EF01
:10B580005AF01F0AD8B494EF5AF0050AD8B498EFCD
:10B590005AF00B0AD8B49CEF5AF0CFEF5AF01B5078
:10B5A00012000001CE6BDEEF5AF021C0D9FF22C09D
:10B5B000DAFF300EDF6E214A222ACE2BFF0E252421
:10B5C000266E276AFF0E2722CE51286E296A265042
:10B5D000285C2950800A2A6E2750800A2A58D8A051
:10B5E000F4EF5AF0F6EF5AF0D5EF5AF0010E21249D
:10B5F000CC6F000E2220CD6F23C01AF024C01BF0A8
:10B60000000E1D6E0A0E1C6E7EEC68F01A500001D2
:10B61000CF6F23C01AF024C01BF0000E1D6E0A0E5F
:10B620001C6EECEC65F01AC023F01BC024F0300E49
:10B630000001CF2721C0D9FF22C0DAFFCFC0DFFF32
:10B640002106D8A0220623502410D8A42AEF5BF0AC
:10B650002CEF5BF0FCEF5AF0CCC021F0CDC022F013
:10B6600012000001628F2A6A2A50040D000EF32492
:10B67000D96E040EF420DA6EDE6ADE6ADE6ADD6AF6
:10B680002A2A0B0E2A6447EF5BF049EF5BF034EF98
:10B690005BF0658C2A6A530E2A24D96EDA6A010E91
:10B6A000DA22DF6A500E2A24D96EDA6A010EDA2213
:10B6B000DF6A2A2A020E2A6460EF5BF062EF5BF019
:10B6C0004BEF5BF0659C080E0101166F040E176FBF
:10B6D000000E3E6E040E3F6E3EC03CF03FC03DF09B
:10B6E000C1C0CBF00001CB51D8A479EF5BF07BEF68
:10B6F0005BF07FEF5BF0100EBE6F8FEF5BF0000E24
:10B70000CD6F010ECC6FCB0ECE6FCF6B000ED16F15
:10B71000010ED06FAAEC5DF0200E0001BE6F12008A
:10B72000EB0E1A6E0B0E1B6E00019251130D220EC2
:10B73000F3241C6E280EF4201D6EF4EC69F0020E4A
:10B7400000019219D8A4A7EF5BF0A9EF5BF0E9EF35
:10B750005BF0EB0E1A6E0B0E1B6E2E0E1C6E2C0E7B
:10B760001D6E3AEC65F0EB0E1A6E0B0E1B6E260E7C
:10B770001C6E2C0E1D6E3AEC65F0EB0E1A6E0B0E65
:10B780001B6EF70E1C6E010E1D6E000E1F6E080E56
:10B790001E6ECDEC61F0EB0E1A6E0B0E1B6EE00E02
:10B7A0001C6E020E1D6E3AEC65F0EB0E1A6E0B0E5F
:10B7B0001B6E2E0E1C6E2C0E1D6E3AEC65F0EB0E01
:10B7C0001A6E0B0E1B6E2B0E1C6E2C0E1D6E3AECA1
:10B7D00065F078EC39F01200020E1B6E580E1A6EEE
:10B7E000400E9B6E1A06D8A01B061A2806E11B28DD
:10B7F000D8A4FDEF5BF0FFEF5BF0F2EF5BF0810EA2
:10B80000C06E896A0F0E926E190E8A6E200E936EAC
:10B810006B0E8B6E100E946E8C6A200E956E1C0E45
:10B820008D6EA00E966E040E8E6E780E976E020EC2
:10B830008F6E040E986EC088980EC16EF70EC26EA1
:10B84000C098BE0EC16E2D0EC26E800ED56E910ECA
:10B85000CD6E040EB66E810E796E400EC76EA10ECF
:10B86000C66E240EA86E900E9C6E080E7C6E670E3F
:10B87000AB6E7D6AC282200EF26E800EF16E010EFA
:10B88000A06EA268A568D08EF28CF28EA38A1200F8
:10B89000206A1CC0D9FF1DC0DAFF1C4A1D2A1AC02D
:10B8A000E1FF1BC0E2FF1A4A1B2ADE50E618D8A4AB
:10B8B0005CEF5CF05EEF5CF09FEF5CF01CC0D9FFCA
:10B8C0001DC0DAFF1C4A1D2A1AC0E1FF1BC0E2FF9F
:10B8D0001A4A1B2ADE50E618D8A471EF5CF073EF09
:10B8E0005CF09FEF5CF01CC0D9FF1DC0DAFF1C4A62
:10B8F0001D2A1AC0E1FF1BC0E2FF1A4A1B2ADE50B4
:10B90000E618D8A486EF5CF088EF5CF09FEF5CF05F
:10B910001CC0D9FF1DC0DAFF1C4A1D2A1AC0E1FF56
:10B920001BC0E2FF1A4A1B2ADE50E618D8A49BEF80
:10B930005CF09DEF5CF09FEF5CF0010E206E2050FC
:10B940001200EB0E0001E26F0B0EE36FA751D8B4AB
:10B95000ACEF5CF0AEEF5CF0F7EF5CF00101B251E0
:10B96000D8B4B5EF5CF0B7EF5CF0F7EF5CF0E2C095
:10B9700021F0E3C022F0B0C023F0246A030E256E4C
:10B98000D1EC5AF021C0E2F022C0E3F0E2C0D9FFCE
:10B99000E3C0DAFF090EDF6E0001E24BE32BE2C0E9
:10B9A00021F0E3C022F0AFC023F0246A030E256E1D
:10B9B000D1EC5AF021C0E2F022C0E3F0E2C0D9FF9E
:10B9C000E3C0DAFF0D0EDF6E0001E24BE32BE2C0B5
:10B9D000D9FFE3C0DAFF0A0EDF6EE24BE32BE2C0D1
:10B9E000DDF0E3C0DEF0A7C0DFF052EC5DF0010156
:10B9F000B26B12000001AB51FD5DD8B002EF5DF0FB
:10BA000004EF5DF029EF5DF00101F2511A6E1B6A3F
:10BA10000001FD51ABC01CF01D6A1C5E000E1D5ADA
:10BA20001A501C5C1D50800A1E6E1B50800A1E5846
:10BA3000D8A01DEF5DF01FEF5DF025EF5DF0010177
:10BA4000F2510001FD2751EF5DF0ABC0FDF051EF69
:10BA50005DF0FD51AB5DD8B030EF5DF032EF5DF0E1
:10BA600051EF5DF00101F1511A6E1B6A0001AB51FB
:10BA7000FDC01CF01D6A1C5E000E1D5A1A501C5C95
:10BA80001D50800A1E6E1B50800A1E58D8A04BEF16
:10BA90005DF04DEF5DF025EF5DF00101F15100012A
:10BAA000FD5F1200EB0E0001DD5DE06F0B0EDE5955
:10BAB000E16F030EDF19D8A460EF5DF062EF5DF077
:10BAC0009AEF5DF0E1BF6EEF5DF0E15109E18D0E9F
:10BAD000E05DD8A06EEF5DF070EF5DF090EF5DF08F
:10BAE000EB0E1A6E0B0E1B6E8C0E1C6E97EC6CF030
:10BAF00043EC3BF098EC33F00001B851D8A483EF4D
:10BB00005DF085EF5DF078EF5DF0770E1A6E0C0E4C
:10BB10001B6EE051740F1C6E97EC6CF0A9EF5DF09A
:10BB2000EB0E1A6E0B0E1B6EE0C01CF097EC6CF067
:10BB3000A9EF5DF0020EDF19D8A4A1EF5DF0A3EF2D
:10BB40005DF0A9EF5DF0DDC0D9FFDEC0DAFFDF6A8E
:10BB5000A3881200C8EF5DF099EC6DF001EF5EF084
:10BB60009BEC6DF001EF5EF09AEC6DF001EF5EF092
:10BB700093EC6DF001EF5EF09CEC6DF001EF5EF088
:10BB800096EC6DF001EF5EF09DEC6DF001EF5EF074
:10BB9000CCC028F0CDC029F02950000AD8B4D7EF86
:10BBA0005DF07F0AD8B4FAEF5DF001EF5EF0285047
:10BBB000010AD8B4B8EF5DF0030AD8B4BCEF5DF069
:10BBC000010AD8B4C0EF5DF0060AD8B401EF5EF008
:10BBD000770AD8B401EF5EF0010AD8B4ACEF5DF09B
:10BBE000070AD8B4B4EF5DF0010AD8B4B0EF5DF045
:10BBF00001EF5EF02850FF0AD8B4C4EF5DF001EF0A
:10BC00005EF01200216E000E226E040E236E1A509A
:10BC10001B6E1C6AD8901B361C3621501D6E1E6A86
:10BC2000D8901D361E36D8901D361E361B501D244A
:10BC30001F6E1C501E20206ED8901F362036D890C4
:10BC40001F3620361F5022262050232222C0D9FF23
:10BC500023C0DAFFDF9E1A50D8A431EF5EF033EF35
:10BC60005EF041EF5EF02150020D1C0EF324D96E00
:10BC7000010EF420DA6E22C0DEFF23C0DDFF4DEF9F
:10BC80005EF02150020D160EF324D96E010EF42041
:10BC9000DA6E22C0DEFF23C0DDFF22C0D9FF23C041
:10BCA000DAFFDF9C20EE04F02250D9262350DA225E
:10BCB000DF8C1200010E1C6E82EF5EF032C0D9FFE5
:10BCC00033C0DAFFE00E1C24E16EE26A020EE222CB
:10BCD000DE50E618D8B46FEF5EF071EF5EF073EFF0
:10BCE0005EF00001926B32C0D9FF33C0DAFFE00E84
:10BCF0001C24E16EE26A020EE222DFCFE7FF324A45
:10BD0000332A1C2A32C0D9FF33C0DAFF0D0EDE18E9
:10BD1000D8B48DEF5EF08FEF5EF097EF5EF0100E0F
:10BD20001C6495EF5EF097EF5EF05EEF5EF0E00E64
:10BD30001C24D96EDA6A020EDA22DF50D8B4A3EFDF
:10BD40005EF0A5EF5EF0A7EF5EF00001926BE00EF3
:10BD50001C24D96EDA6A020EDA22DF6A1200000EA3
:10BD60001A6E200E1B6E000E1C6ECE0E1E6EF00E96
:10BD70001D6E74EC6AF01AC0D9F01BC0DAF0010134
:10BD8000EE05D8A4C6EF5EF0C8EF5EF003EF5FF0FB
:10BD9000F00EF66EEE0EF76E000EF86E0900F5501E
:10BDA0000001D91908E10900F550DA19D8A4DBEF30
:10BDB0005EF0DDEF5EF0E6EF5EF001018605D8A4EF
:10BDC000E4EF5EF0E6EF5EF003EF5FF00001A551F7
:10BDD000D8A4EDEF5EF0EFEF5EF0F9EF5EF00C0E41
:10BDE000D16F2B0ED26F000ED36F000ED46FEBEC21
:10BDF00030F0010E0001A56F040E426E000E01012D
:10BE0000756F000E746F1200EB0E0001E46F0B0EE5
:10BE1000E56F4050D8B40FEF5FF011EF5FF01DEF0A
:10BE20005FF0E4C0D0F0E5C0D1F077EC4EF0D0C0C8
:10BE3000E4F0D1C0E5F03DEF5FF08E518FC0E2F04D
:10BE4000E36BE25F000EE35BE3BF32EF5FF0E351D1
:10BE500007E1100EE25DD8B030EF5FF032EF5FF037
:10BE600011EF5FF08E518F5DD8B039EF5FF03BEF8F
:10BE70005FF03DEF5FF011EF5FF0E4C0DDF0E5C093
:10BE8000DEF090C0DFF052EC5DF04050D8B44BEFE4
:10BE90005FF04DEF5FF058EF5FF00101A451D8A4BF
:10BEA00054EF5FF056EF5FF058EF5FF00001906BDA
:10BEB0001200286E0A0E236E0D0E246E060E256EDD
:10BEC000000E266EF8EC51F023C036F124C037F195
:10BED00025C038F126C039F1110E236E0D0E246EE7
:10BEE000060E256E000E266EF8EC51F023C032F1DE
:10BEF00024C033F125C034F126C035F1010136519B
:10BF0000371138113911D8B488EF5FF08AEF5FF03C
:10BF10008CEF5FF0010EA76F3251331134113511E0
:10BF2000D8B495EF5FF097EF5FF099EF5FF0010EF7
:10BF3000A66F28C090F04050D8B4A1EF5FF0A3EFF7
:10BF40005FF0A7EF5FF0080EA46FA9EF5FF00001AC
:10BF50008F6B8FC08EF01200000E236E000E246EC9
:10BF6000000E256E000E266E1E501F102010211090
:10BF7000D8B4BDEF5FF0BFEF5FF0F5EF5FF0010EFB
:10BF8000226EC9EF5FF0D8901E361F36203621365C
:10BF9000222A21AECEEF5FF0D0EF5FF0C3EF5FF06B
:10BFA000D89023362436253626361E501A5C1F506C
:10BFB0001B5820501C5821501D58D8A0E2EF5FF0AC
:10BFC000E4EF5FF0EDEF5FF01E501A5E1F501B5A5A
:10BFD00020501C5A21501D5A2380D89021322032E3
:10BFE0001F321E32222ED0EF5FF023C01AF024C081
:10BFF0001BF025C01CF026C01DF01200560E431881
:10C00000D8A405EF60F007EF60F02FEF60F00101BA
:10C010009B51D8B40EEF60F010EF60F02BEF60F0A2
:10C02000000E1B6E010E1A6E000E1D6E640E1C6E4D
:10C030009AC11EF098C11FF096C120F095C121F061
:10C040007DC022F0060E50EC60F000017607D8A00B
:10C0500077074FEF60F0CEEC66F04FEF60F0520ED6
:10C060004318D8A436EF60F038EF60F02BEF60F0A3
:10C070005AC11AF05BC11BF056C11CF057C11DF02C
:10C0800099C11EF097C11FF094C120F093C121F017
:10C090007CC022F0070E50EC60F025EF60F012003B
:10C0A000236E0001C951D8B458EF60F05AEF60F028
:10C0B00064EF60F0976B000E01013A6F000E3B6F6A
:10C0C000000E3C6F000E3D6F23C0C9F01EC0FCF097
:10C0D0001FC0FBF020C0F2F121C0F1F122C0A9F095
:10C0E0000001AC6B8A51D8B478EF60F07AEF60F061
:10C0F0008DEF60F01A501B10D8B481EF60F083EF21
:10C1000060F089EF60F01AC076F01BC077F09EEF08
:10C1100060F0766977699EEF60F01C501D10D8B40E
:10C1200094EF60F096EF60F09CEF60F01CC074F04C
:10C130001DC075F09EEF60F0746975691200000E05
:10C140000001CF6F030ED06FCFC0D9FFD0C0DAFF90
:10C1500071C1DFFFCF4BD02BCFC0D9FFD0C0DAFFEA
:10C1600070C1DFFFCF4BD02BCFC0D9FFD0C0DAFFDB
:10C1700067C0DFFFCF4BD02BCFC0D9FFD0C0DAFFD5
:10C1800066C0DFFFCF4BD02BCFC0D9FFD0C0DAFFC6
:10C1900065C0DFFFCF4BD02BCFC0D9FFD0C0DAFFB7
:10C1A0009FC0DFFFCF4BD02B000ECC6FE00ECD6FCA
:10C1B000070ECE6FCCC01FF0CDC020F0CEC021F056
:10C1C000000E226E030E236E000E276E2750CF5DE9
:10C1D000246ED3EC58F012000001AA6B010E01018D
:10C1E000AB6F560E4318D8A4F8EF60F0FAEF60F08A
:10C1F00015EF61F05CC11AF05DC11BF058C11CF075
:10C2000059C11DF09AC11EF098C11FF096C120F0CF
:10C2100095C121F07DC022F0060E50EC60F00001C7
:10C220007607D8A0770737EF61F0520E4318D8A4ED
:10C230001CEF61F01EEF61F035EF61F05AC11AF0AA
:10C240005BC11BF056C11CF057C11DF099C11EF017
:10C2500097C11FF094C120F093C121F07CC022F05F
:10C26000070E50EC60F00FEF61F0CEEC66F01200BC
:10C270001C6E1B6A1C50040D2C0EF324D96E020E8A
:10C28000F420DA6E0101D751DE18D8A44AEF61F02C
:10C290004CEF61F081EF61F01C50040D2D0EF32482
:10C2A000D96E020EF420DA6EDE50D819D8A45BEFF6
:10C2B00061F05DEF61F081EF61F01C50040D2E0E16
:10C2C000F324D96E020EF420DA6EDE50D919D8A408
:10C2D0006CEF61F06EEF61F081EF61F01C50040DC6
:10C2E0002F0EF324D96E020EF420DA6EDE50DA1926
:10C2F000D8A47DEF61F07FEF61F081EF61F0010E76
:10C300001B6E1B5012000101BD6BBC6B020E0001C5
:10C31000BC19D8A48EEF61F090EF61F0AAEF61F044
:10C3200020EE01F03C50D9263D50DA22080EDF6E97
:10C3300020EE02F03C50D9263D50DA22C40EDE6ECB
:10C34000010EDD6E3CC0D9FF3DC0DAFFC80EDF6EC6
:10C35000CCEF61F06351C55D6451C659D8B0B3EFFD
:10C3600061F0B5EF61F0B9EF61F0C5C063F0C6C030
:10C3700064F0ACEC4AF0010120EE02F01651D9262F
:10C380001751DA22C40EDE6E010EDD6E16C1D9FF22
:10C3900017C1DAFFC80EDF6E12001AC020F01BC0F2
:10C3A00021F0D5EF61F0204A212A20C0D9FF21C019
:10C3B000DAFFDF50D8A4DFEF61F0E1EF61F0D3EFF7
:10C3C00061F0EAEF61F0204A212A1C4A1D2A1E066C
:10C3D000D8A01F061E501F10D8B4F1EF61F0F3EF84
:10C3E00061F005EF62F01CC0D9FF1DC0DAFF20C06C
:10C3F000E1FF21C0E2FFDFCFE7FFE750D8A403EF62
:10C4000062F005EF62F0E3EF61F01E501F10D8A458
:10C410000CEF62F00EEF62F013EF62F020C0D9FF74
:10C4200021C0DAFFDF6A12004450D8A41AEF62F08C
:10C430001CEF62F053EF62F000017B51D8B423EFA0
:10C4400062F025EF62F051EF62F0510E0101E15D03
:10C45000C30EE259D8A02FEF62F031EF62F053EF34
:10C4600062F0010E416E00017A51D8B43AEF62F0E9
:10C470003CEF62F042EF62F08BC0E1F10101E26B50
:10C4800053EF62F0AF0E0101E26FC80EE16F0001E1
:10C490007951640DF3500101E127F450E22353EF89
:10C4A00062F00101B72BDFC1E5F1E0C1E6F1010E59
:10C4B000446E4568120023C0D1F024C0D2F0200E93
:10C4C0002518D8B466EF62F068EF62F071EF62F0A1
:10C4D00026502518D8A46FEF62F071EF62F09DEF3F
:10C4E00062F00001D36B32C0D9FF33C0DAFFD35101
:10C4F000CC0FE16EE26ADFCFE7FF324A332A32C067
:10C5000020F033C021F0C4EC6AF020C032F021C02A
:10C5100033F00001D32B030ED36591EF62F093EF5C
:10C5200062F073EF62F0D06BCC0E1A6E1B6AC9EC2E
:10C530004BF01AC0D1F01BC0D2F0D1C023F0D2C052
:10C5400024F012001D6E1D50F00B1E6E1E3A0F0ED1
:10C550001E160A0E1E60AFEF62F0B1EF62F0BCEF84
:10C5600062F01E50300F1AC0D9FF1BC0DAFFDF6E19
:10C570001A4A1B2AC5EF62F01E50370F1AC0D9FFA6
:10C580001BC0DAFFDF6EB8EF62F01D500F0B1E6E9E
:10C590000A0E1E60CEEF62F0D0EF62F0DBEF62F0C9
:10C5A0001E50300F1AC0D9FF1BC0DAFFDF6E1A4AC7
:10C5B0001B2AE4EF62F01E50370F1AC0D9FF1BC0D0
:10C5C000DAFFDF6ED7EF62F01AC01AF01BC01BF063
:10C5D00012001F6A8B90030EC96E9EA6F2EF62F0E6
:10C5E000F4EF62F0EDEF62F09E961CC0C9FF9EA6CC
:10C5F000FCEF62F0FEEF62F0F7EF62F09E961BC078
:10C60000C9FF9EA606EF63F008EF63F001EF63F049
:10C610009E961AC0C9FF9EA610EF63F012EF63F05A
:10C620000BEF63F09E96C9689EA619EF63F01BEFAF
:10C6300063F014EF63F09E961DC0D9FF1EC0DAFFB1
:10C64000C9CFDFFF1D4A1E2A1F2A1F50D8A42BEF77
:10C6500063F02DEF63F013EF63F08B8012000101A4
:10C660008A51D8B436EF63F038EF63F073EF63F0BC
:10C670004404D8A43EEF63F040EF63F048EF63F06A
:10C68000F551D8B446EF63F048EF63F050EF63F034
:10C690008205D8A44EEF63F050EF63F06FEF63F0C4
:10C6A0000001A151D8A457EF63F059EF63F063EF95
:10C6B00063F03F0ED16F2B0ED26F000ED36F000EC2
:10C6C000D46FEBEC30F0010E0001A16F040E426E4E
:10C6D000000E0101756F000E746F71EF63F00001C1
:10C6E000A16B0101F56B12001E501F1020102110CC
:10C6F000D8B47DEF63F07FEF63F0AFEF63F0010E2E
:10C70000226E89EF63F0D8901E361F362036213610
:10C71000222A21AE8EEF63F090EF63F083EF63F097
:10C720001E501A5C1F501B5820501C5821501D5879
:10C73000D8A09DEF63F09FEF63F0A7EF63F01E506A
:10C740001A5E1F501B5A20501C5A21501D5AD89057
:10C75000213220321F321E32222E90EF63F01AC097
:10C760001AF01BC01BF01CC01CF01DC01DF01200F5
:10C77000020E00019819D8A4C0EF63F0C2EF63F075
:10C78000FAEF63F0000E01014D6F000E4E6F700E58
:10C790004F6F4DC11BF04EC11CF04FC11DF03DEC61
:10C7A00064F0000E01014D27100E4E23000E4F23A2
:10C7B000700E4F65DEEF63F0E0EF63F0C9EF63F0FA
:10C7C000800E346E080E356E000EE8CF80F8000E35
:10C7D0000001656F000E666F700E676FCC0ED16F33
:10C7E000290ED26F010ED36F000ED46FEBEC30F038
:10C7F0000001986B1200020E00019A19D8A403EFF1
:10C8000064F005EF64F03CEF64F005EC6DF00101BD
:10C81000AC07AC29D8A40FEF64F011EF64F024EF5B
:10C8200064F08DA816EF64F01AEF64F01B6A1B2AFF
:10C830001BEF64F01B6A1B3A8D501B18EF0B1B1883
:10C840008D6E320E0101AC6F020E1C6E380E1B6E27
:10C85000AD0EE82EFED71B2EFCD71C2EFAD70000FB
:10C86000040039EC6CF00009D8A439EF64F03BEF18
:10C8700064F007EF64F0FF001200060E40EC6DF06C
:10C880008B90200EC96E9EA648EF64F04AEF64F0CC
:10C8900043EF64F09E961DC0C9FF9EA652EF64F060
:10C8A00054EF64F04DEF64F09E961CC0C9FF9EA645
:10C8B0005CEF64F05EEF64F057EF64F09E961BC08F
:10C8C000C9FF9EA666EF64F068EF64F061EF64F064
:10C8D0009E968B809C0E1E6ED70EE82EFED71E2EC7
:10C8E000FCD7000039EC6CF00009D8A47AEF64F0B2
:10C8F0007CEF64F06AEF64F012000001BD6BBA6B6C
:10C900000101BD6BBC6BC16B0001BC6B16C1D9FFD3
:10C9100017C1DAFF7F0EDF16040E0101161B16C1C8
:10C92000D9FF17C1DAFF7F0EDF16040E161B3CC0BD
:10C93000D9FF3DC0DAFF7F0EDF160001626B000EEB
:10C94000646F000E636F01010A6B000E0C6F000E26
:10C950000B6F7EEC50F0000E0001CD6F030ECC6F1C
:10C96000000ECE6F000ECF6F000ED16F000ED06F95
:10C97000AAEC5DF08BEC49F012000001D16F0001D0
:10C98000D26B32C0D9FF33C0DAFFD251CC0FE16E87
:10C99000E26ADFCFE7FF324A332A32C020F033C0E9
:10C9A00021F0C4EC6AF020C032F021C033F0000165
:10C9B000D22B030ED265DFEF64F0E1EF64F0C1EF3C
:10C9C00064F0D06BD151256E266ACC0E1A6E1B6AAC
:10C9D000C9EC4BF025501A02F3CF27F0F4CF28F022
:10C9E0001B02F350282626501A02F350282627C08F
:10C9F00023F028C024F01200256826681FEF65F098
:10CA00001FC0D9FF20C0DAFFDF50236E2650231845
:10CA1000266E2638F00B2618266E2638E842070BBD
:10CA20002618246E24380F0B2518236E2638E8426A
:10CA3000F80B2318266E24C025F01F4A202A210651
:10CA4000D8A02206212806E12228D8A42AEF65F0E2
:10CA50002CEF65F000EF65F0251E2650FF0A266ECC
:10CA6000250E1A6E1B6AD70E1C6E010E1D6ECBECC6
:10CA700047F01200000E1F6E000E1E6E42EF65F0B2
:10CA80001E4A1F2A1E501A24D96E1F501B20DA6E10
:10CA9000DF50D8A44EEF65F050EF65F040EF65F041
:10CAA00056EF65F01E4A1F2A1C4A1D2A1CC0F6FFBD
:10CAB0001DC0F7FF000EF86E1E501A24D96E1F50CD
:10CAC0001B20DA6E0F0EF76403D00800F55005D076
:10CAD000F6CFE1FFF7CFE2FFE750DF6EDF50D8A4DB
:10CAE00074EF65F076EF65F052EF65F012001AC052
:10CAF0001FF094EF65F01D06D8A01E061BC0D9FFDD
:10CB00001CC0DAFF1B4A1C2A1F2A1F04E16EE26ABE
:10CB1000DFCFE7FFE750D8A490EF65F092EF65F024
:10CB200094EF65F0A4EF65F01D501E10D8A49BEFA4
:10CB300065F09DEF65F07BEF65F0A4EF65F01F50A9
:10CB4000D96EDA6ADF6A1F2A1D06D8A01E061D28C4
:10CB500006E11E28D8A4AFEF65F0B1EF65F09FEFB6
:10CB600065F012000101E951EA11D8A4BAEF65F0AD
:10CB7000BCEF65F0EBEF65F00001A651D8A4C3EF60
:10CB800065F0C5EF65F0CFEF65F0570ED16F2B0E56
:10CB9000D26F000ED36F000ED46FEBEC30F0010EAD
:10CBA0000001A66F4204D8A4D8EF65F0DAEF65F073
:10CBB000DCEF65F0CEEC66F04250D8A4E2EF65F011
:10CBC000E4EF65F0EBEF65F0040E426E000E01013C
:10CBD000756F000E746F1200000E206E000E1F6E37
:10CBE0001C501D10D8B4F7EF65F0F9EF65F021EF98
:10CBF00066F0010E1E6E01EF66F0D8901C361D36F1
:10CC00001E2A1DAE06EF66F008EF66F0FDEF65F038
:10CC1000D8901F3620361C501A5C1D501B58D8A0C7
:10CC200014EF66F016EF66F01BEF66F01C501A5E0C
:10CC30001D501B5A1F80D8901D321C321E2E08EF2B
:10CC400066F01FC01AF020C01BF012004150D8B48B
:10CC50002CEF66F02EEF66F04BEF66F000017B5193
:10CC6000D8B435EF66F037EF66F050EF66F00101AB
:10CC7000E151E211D8A43FEF66F041EF66F050EFCA
:10CC800066F0000E0001E86F050EBBEC2AF023EC05
:10CC90003CF050EF66F0EA0E0101E26F600EE16FCA
:10CCA000010174517511D8A458EF66F05AEF66F07F
:10CCB0005BEF66F08B923BEC4BF01200D3C11AF0A5
:10CCC000D4C11BF0D5C11CF0D6C11DF02D0E1E6EB7
:10CCD0007F0E1F6E950E206E4C0E216EE0EC67F0FD
:10CCE000010E1A240101D36F000E1B20D46F000E19
:10CCF0001C20D56F000E1D20D66FD3C1CCF0D4C13F
:10CD0000CDF0D5C1CEF0D6C1CFF0120E8EEF66F0C9
:10CD10000001D890CF33CE33CD33CC33E82E88EF1B
:10CD200066F0CCC026F0CDC027F01200FF0E010146
:10CD30009F251C6E1D6AFF0E1D22730E1C24F66EAD
:10CD4000240E1D20F76EF86A000EF8220800F5CFB9
:10CD50001EF01F6A1F50020D2F0EF324F66E240ED4
:10CD6000F420F76EF86A000EF8220900F5501A5CFC
:10CD70000900F5501B58D8A0C0EF66F0C2EF66F06E
:10CD8000CCEF66F01E2A1F2A210E1F64CAEF66F040
:10CD9000CCEF66F0AAEF66F01E5012000001C96BDE
:10CDA0000101AB6B0001976B89988E94AC6B426A62
:10CDB000400EFC6F500EFB6F020E0101F26F020E6F
:10CDC000F16F0001A96B7A51D8B4E9EF66F0EBEF8F
:10CDD00066F0F8EF66F08BC0E1F10101E26B2C0E1A
:10CDE000E127010EE223300E0201D86F05EF67F054
:10CDF000AF0E0101E26FC80EE16F00017951640DC1
:10CE0000F3500101E127F450E22312001CC023F08B
:10CE10001DC024F01AC021F01BC022F02CEF67F0D7
:10CE200023C0F6FF24C0F7FF000EF86E0F0EF76464
:10CE300003D00800F55005D0F6CFE1FFF7CFE2FFB1
:10CE4000E750206E234A242A21C0D9FF22C0DAFFEE
:10CE500020C0DFFF214A222A1E06D8A01F061E2856
:10CE600006E11F28D8A437EF67F039EF67F010EF1D
:10CE700067F01AC01AF01BC01BF0120044EF67F0F5
:10CE80001A4A1B2A1C4A1D2A1CC0D9FF1DC0DAFFE2
:10CE90001AC0E1FF1BC0E2FFDE50E618D8A453EF32
:10CEA00067F055EF67F061EF67F01AC0D9FF1BC05C
:10CEB000DAFFDF50D8A45FEF67F061EF67F040EF73
:10CEC00067F01AC0D9FF1BC0DAFFDF501E6E1CC00E
:10CED000D9FF1DC0DAFFDF501F6E1F501E5C1A6E97
:10CEE0001B6AD8A01B0612001B6E1BC01AF0380E5E
:10CEF0000101F9617EEF67F080EF67F08CEF67F07A
:10CF0000540E1B6486EF67F088EF67F096EF67F0CA
:10CF1000540E1A6E96EF67F0620E1B6492EF67F084
:10CF200094EF67F096EF67F0620E1A6E4204D8A491
:10CF30009CEF67F09EEF67F0A8EF67F08D05D8A42F
:10CF4000A4EF67F0A6EF67F0A8EF67F0280E1A6E5F
:10CF50001A501200040EF66EF76AF86A0900F5CF4F
:10CF60002BF10900F5CF2AF10900F5CF2DF10900C9
:10CF7000F5CF2CF101012A390F0B0F0B300FF76F92
:10CF80002A510F0B300FF86F2B390F0B0F0B300F8F
:10CF9000F96F2B510F0B300FFA6F2C390F0B0F0B52
:10CFA000300FFB6F2C510F0B300FFC6F2D390F0B17
:10CFB0000F0B300FFD6F2D510F0B300FFE6F120056
:10CFC000000E226E000E236E000E246E000E256EE3
:10CFD0001AA0EDEF67F0EFEF67F0F7EF67F01E5084
:10CFE00022261F5023222050242221502522D8906F
:10CFF0001E361F3620362136D8901D321C321B3289
:10D000001A321A501B101C101D10D8A40AEF68F019
:10D010000CEF68F0E8EF67F022C01AF023C01BF0B5
:10D0200024C01CF025C01DF012001D6A81AA1BEF50
:10D0300068F01DEF68F048EF68F08A961D6A3EEFD1
:10D0400068F01AC0F6FF1BC0F7FF000EF86E0F0E57
:10D05000F76403D00800F55005D0F6CFE1FFF7CF15
:10D06000E2FFE750C96E1A4A1B2A9EA63AEF68F003
:10D070003CEF68F035EF68F09E961D2A1C501D5C51
:10D08000D8A045EF68F047EF68F021EF68F08A8696
:10D090001D501200020E0001BC19D8A452EF68F016
:10D0A00054EF68F058EF68F0F8EC48F07DEF68F066
:10D0B000BC6B0101C151D8A460EF68F062EF68F069
:10D0C0007CEF68F020EE01F03C50D9263D50DA228A
:10D0D000080EDF6E20EE02F03C50D9263D50DA22D9
:10D0E000BF0EDE6E000EDD6E3CC0D9FF3DC0DAFF24
:10D0F0008C0EDF6E7DEF68F0C16B12001C501D10AE
:10D10000D8B485EF68F087EF68F0ABEF68F0010EF8
:10D110001E6E8FEF68F0D8901C361D361E2A1DAE8D
:10D1200094EF68F096EF68F08BEF68F01C501A5C93
:10D130001D501B58D8A09FEF68F0A1EF68F0A5EF35
:10D1400068F01C501A5E1D501B5AD8901D321C32BC
:10D150001E2E96EF68F01AC01AF01BC01BF01200CA
:10D16000010EC26EC282C2B2B8EF68F0BAEF68F0C8
:10D17000B3EF68F0D890C432C332D890C432C3320F
:10D18000C35001016E27C4506F230001B22BB29F20
:10D19000050EC26EC282C2B2D0EF68F0D2EF68F064
:10D1A000CBEF68F0D890C432C332D890C432C332C7
:10D1B000C35001016C27C4506D230001B12BB19FF6
:10D1C000120001013A513B113C113D11D8B4EBEF73
:10D1D00068F0EDEF68F0F2EF68F03A07000E3B5BA5
:10D1E0003C5B3D5B00019451D8A4F9EF68F0FBEF84
:10D1F00068F010EF69F04DC11FF04EC120F04FC133
:10D2000021F0000E226E030E236E000E246ED3EC6E
:10D2100058F0000E01014D27010E4E23000E4F2342
:10D220001200000E0101CC6F4B0ECD6F000ECE6FC1
:10D23000000ECF6FD06BD16B080ED26F0001B96BAF
:10D240001A0E246E010E11EC6BF01E0E246E020EEF
:10D2500011EC6BF0000E1A6E700E1B6E020E1C6E3F
:10D26000400E1D6E020EA1EC56F01AC07AF11BC0E2
:10D270007BF1000E0101786F000E796F0001B86B31
:10D280001200030E00019B19D8A449EF69F04BEF7F
:10D2900069F06FEF69F09B6B000E276EF10E286E40
:10D2A0007F0E296E000E1A6E030E1B6E140E1C6E7E
:10D2B0002C0E1D6E000E1F6E030E1E6E06EC67F028
:10D2C00027C01FF028C020F029C021F0000E226ED8
:10D2D000030E236E030E246ED3EC58F0FF001200F1
:10D2E000226A010E236E2350210D800EF324206E3E
:10D2F0000A0EF420216E20C01AF021C01BF00A0E85
:10D300001C6E0D0E1D6E3EEC67F01A501B10D8A45B
:10D310008CEF69F08EEF69F092EF69F023C022F094
:10D320009BEF69F0232A0A0E236499EF69F09BEFC3
:10D3300069F073EF69F02250120000019051D8A4F7
:10D34000A4EF69F0A6EF69F0AEEF69F04050D8B4F1
:10D35000ACEF69F0AEEF69F0C8EF69F0000E8F2511
:10D36000D96EDA6A060EDA22A5C1DFFF8F51040DED
:10D37000800EF324D96E060EF420DA6E2BC0DEFF89
:10D380002CC0DEFF2DC0DEFF2EC0DEFF8F2B8F9F57
:10D390001200EB0E1A6E0B0E1B6EBC0E1C6E2A0ECC
:10D3A0001D6EF4EC69F078EC39F0330EAB6E7D6AEB
:10D3B000040E246E0C0E236E340EE82EFED7232EA0
:10D3C000FCD7242EFAD7EB0E1A6E0B0E1B6E0D0E29
:10D3D0001C6E2C0E1D6EF4EC69F078EC39F0000E2A
:10D3E000376E000E366E12001AC020F01BC021F0FE
:10D3F0001C501E6E1D501F6E1C4A1D2A1EC0F6FFBB
:10D400001FC0F7FF000EF86E20C0D9FF21C0DAFF61
:10D41000204A212A0F0EF76403D00800F55005D0EA
:10D42000F6CFE1FFF7CFE2FFE750DF6EDF50D8A481
:10D430001CEF6AF01EEF6AF0F8EF69F012000F01BE
:10D440004CA125EF6AF027EF6AF048EF6AF03EC082
:10D45000D9FF3FC0DAFF800EDE18D8A432EF6AF0A1
:10D4600034EF6AF047EF6AF016C1D9FF17C1DAFF4F
:10D47000840EDE18D8A43FEF6AF041EF6AF047EF60
:10D480006AF03EC0D9FF3FC0DAFF8C0EDF6E4C91D0
:10D49000629A120000018951D8B451EF6AF053EF3B
:10D4A0006AF060EF6AF08751D8B459EF6AF05BEF29
:10D4B0006AF073EF6AF0010E0101AE6F73EF6AF06C
:10D4C0008851D8B466EF6AF068EF6AF073EF6AF0DB
:10D4D00001019C51D8B46FEF6AF071EF6AF073EFFD
:10D4E0006AF05BEF6AF01200000E206E000E1F6EF5
:10D4F0008BEF6AF01AC0F6FF1BC0F7FF1CC0F8FFE5
:10D500000800F5501F26000E2022010E1A26000EDC
:10D510001B22000E1C221D06D8A01E061D2806E197
:10D520001E28D8A496EF6AF098EF6AF07AEF6AF0B6
:10D530001FC01AF020C01BF01200220E1A6E070E38
:10D540001B6E0D0E1C6E000E1E6E030E1D6E77EC14
:10D5500065F0256A220E1A6E1B6AC9EC4BF01AC0E0
:10D560006EF01BC06FF000016F5107E1050E6E5D9C
:10D57000D8B0BDEF6AF0BFEF6AF0C3EF6AF0000EFB
:10D580006F6F050E6E6F12002150030802E12050EC
:10D59000FF08D8B0CEEF6AF0D0EF6AF0E6EF6AF09D
:10D5A000000E2F26010E3022000E31222FC01AF05D
:10D5B00030C01BF031C01CF0000E1D6E030E1E6E3D
:10D5C000E9EC62F0000E206E030E216E20C020F008
:10D5D00021C021F012001AC0D9FF1BC0DAFF1C5075
:10D5E000DE18D8A4F6EF6AF0F8EF6AF0FEEF6AF002
:10D5F0001AC01AF01BC01BF010EF6BF01AC0D9FF55
:10D600001BC0DAFF1A4A1B2ADF50D8A40AEF6BF0BE
:10D610000CEF6BF0EBEF6AF0000E1A6E000E1B6E53
:10D620001200276E24A417EF6BF019EF6BF01EEFBA
:10D630006BF0000E1A6E275002EC5EF024A223EF6E
:10D640006BF025EF6BF02AEF6BF0010E1A6E27508E
:10D6500002EC5EF04C0E2724256E266A0F0E262261
:10D6600025C0D9FF26C0DAFF24C0DFFF12000F015A
:10D670005C8562986582010E0101C26F000E000197
:10D68000CD6F750ECC6F000ECE6F000ECF6F000EFB
:10D69000D16F000ED06FAAEC5DF0200E0001BE1914
:10D6A000D8A455EF6BF057EF6BF059EF6BF0FDEC32
:10D6B0004FF0120085BA5FEF6BF061EF6BF06DEF2A
:10D6C0006BF00101F351D8B468EF6BF06AEF6BF0C7
:10D6D0007CEF6BF0F3077CEF6BF00101F351D8A402
:10D6E00074EF6BF076EF6BF079EF6BF0010E0001E9
:10D6F0009D6F050E0101F36F1200040EF66EF76ABE
:10D70000F86A2BC1F5FF0D002AC1F5FF0C00240EAD
:10D71000A66EF29E550EA76EAA0EA76EA682060EE4
:10D72000F66E2DC1F5FF0D002CC1F5FF0C00550E56
:10D73000A76EAA0EA76EA682F28EA6941200010E04
:10D740001C6E2F0E0101B325F66EF76A230EF72229
:10D75000F86A000EF8220800F5CF1BF01B50800A73
:10D760001A6EA051800A1A5CD8B0B9EF6BF0BBEF0B
:10D770006BF0BEEF6BF01C6A00019E6B1C50120038
:10D7800000019251D8A4C7EF6BF0C9EF6BF0DFEF47
:10D790006BF08D9C670EAB6E7D6A040E1B6E0C0EDB
:10D7A0001A6E340EE82EFED71A2EFCD71B2EFAD78F
:10D7B0008D8C0201B06B0101B9690001936B1200FD
:10D7C0000101C26B000E0001CD6F740ECC6F000E14
:10D7D000CE6F000ECF6F000ED16F000ED06FAAEC8F
:10D7E0005DF065920F015C95F7EF6BF0629462B4A7
:10D7F000FCEF6BF0FEEF6BF0F6EF6BF012001D6EBE
:10D800001DC01EF01B501A18D8A409EF6CF00BEFC6
:10D810006CF01BEF6CF032C0D9FF33C0DAFF4F0E53
:10D82000DE18D8B416EF6CF019EF6CF0010E1AEF99
:10D830006CF0000E1E6E1E50120000017B51D8B419
:10D8400024EF6CF026EF6CF036EF6CF00101E15143
:10D85000E211D8A42EEF6CF030EF6CF036EF6CF0E4
:10D86000000E0001E86F050EBBEC2AF052EC6CF0E4
:10D8700012008B90050EC96E9EA641EF6CF043EF2F
:10D880006CF03CEF6CF09E96C9689EA64AEF6CF077
:10D890004CEF6CF045EF6CF09E96C9CF1AF08B8080
:10D8A0001A50120000018951D8B459EF6CF05BEFA7
:10D8B0006CF05FEF6CF065EC53F069EF6CF0885141
:10D8C000D8B465EF6CF067EF6CF069EF6CF0ECECDE
:10D8D00052F012001D6E8A98020E74EC6DF01D500D
:10D8E00074EC6DF01B5074EC6DF01C5074EC6DF02A
:10D8F0008A8881AA7EEF6CF080EF6CF079EF6CF093
:10D90000120081AA86EF6CF088EF6CF081EF6CF06A
:10D91000000E1B6E040E1C6E000E6AEC6CF0080EFE
:10D920001B6E010E1C6E000E6AEC6CF01200000102
:10D93000B851D8A49EEF6CF0A0EF6CF0ACEF6CF097
:10D940001AC07EF11BC07FF11CC0B7F0010E0101AF
:10D95000BB6F010E0001B86F12001B6E030E1B247B
:10D96000D96EDA6A0D0EDA224F0EDE18D8B4BBEF8C
:10D970006CF0BEEF6CF0010EBFEF6CF0000E120009
:10D9800001017251705D73517159D8B0CAEF6CF0DA
:10D99000CCEF6CF0D2EF6CF072C170F173C171F129
:10D9A0009FEC60F012003002030060EA10270300D1
:10D9B0000500580201010101010102020540013880
:10D9C0003430303134303234010E0101B76FEBEFB7
:10D9D0006CF0E2EC4CF00101B751D8A4F2EF6CF01E
:10D9E000F4EF6CF0E9EF6CF012004204D8A4FBEF06
:10D9F0006CF0FDEF6CF001EF6DF0CEEC66F004EF33
:10DA00006DF0010E0001C96F1200060E40EC6DF0C2
:10DA10008B90600EC96E9EA610EF6DF012EF6DF048
:10DA20000BEF6DF09E968B801200010E0101AF6F1F
:10DA3000DFC1E5F1E0C1E6F1010E446E010E000127
:10DA4000736FF40E726F12001A6E1A04D8A42BEFC3
:10DA50006DF02DEF6DF030EF6DF04F0E31EF6DF09A
:10DA60004E0E12001E6E1E50FE0DF350C40F1F6EA0
:10DA70001FC01BF01FC01CF00B0E6AEC6CF01200F4
:10DA80001A6E8B901AC0C9FF9EA649EF6DF04BEF3E
:10DA90006DF044EF6DF09E968B8012003030303088
:10DAA000303030302D000000000000000000000089
:10DAB000000000000000020E00019919D8A463EFD5
:10DAC0006DF065EF6DF067EF6DF065EF6DF01200D2
:10DAD0001A6E00018F6B1AC040F0C751C80DF3CF0A
:10DAE000E1F1F4CFE2F112001A6E1AC0C9FF9EA64E
:10DAF0007CEF6DF07EEF6DF077EF6DF09E9612008B
:10DB00008B94280EE82EFED78B8481EC6CF01200EB
:10DB10008D948D9680EC6DF08D981200050029058E
:10DB200050403CFF02FF11EC69F0120057EC54F03A
:10DB3000120012001200120012001200FFFFFFFF7D
:10DB4000FFFFFFFFFFFFFFFFFFFFFFFFFFFFFFFFE5
:10DB5000FFFFFFFFFFFFFFFFFFFFFFFFFFFFFFFFD5
:10DB6000FFFFFFFFFFFFFFFFFFFFFFFFFFFFFFFFC5
:10DB7000FFFFFFFFFFFFFFFFFFFFFFFFFFFFFFFFB5
:02EEF000CEA6AC
:020000040001F9
:06FFF800A7F705FBF8F875
:00000001FF
